:100000000088012059090000550900005509000029
:1000100055090000550900005509000000000000C6
:100020000000000000000000000000005509000072
:1000300055090000000000005509000055090000A6
:100040005509000055090000550900005509000038
:100050005509000055090000550900005509000028
:100060005509000055090000550900005509000018
:100070005509000055090000550900005509000008
:1000800055090000550900005509000055090000F8
:1000900055090000550900005509000055090000E8
:1000A00055090000550900005509000055090000D8
:1000B00055090000550900005509000055090000C8
:1000C00055090000550900005509000055090000B8
:1000D00055090000550900005509000055090000A8
:1000E0005509000055090000000000000000000054
:1000F00000000000CD050000B10800001D0900004F
:10010000250900002D0900005509000055090000CF
:100110005509000055090000550900005509000067
:100120005509000055090000550900005509000057
:100130005509000055090000550900005509000047
:100140005509000055090000550900005509000037
:100150005509000055090000550900005509000027
:100160005509000055090000550900005509000017
:100170005509000055090000550900005509000007
:1001800055090000550900005509000055090000F7
:1001900055090000550900005509000055090000E7
:1001A00055090000550900005509000055090000D7
:1001B00055090000550900005509000055090000C7
:1001C00055090000550900005509000055090000B7
:1001D00055090000550900005509000055090000A7
:1001E0005509000055090000550900002D0F0000B9
:1001F0005509000055090000550900005509000087
:100200005509000055090000550900005509000076
:100210005509000055090000550900005509000066
:100220005509000055090000550900005509000056
:100230005509000055090000550900005509000046
:100240005509000055090000550900005509000036
:100250005509000055090000550900005509000026
:10026000550900000348044B834202D0034B03B1FD
:1002700018477047E4460200E44602000000000010
:100280000548064B1B1AD90F01EBA301491002D0F8
:10029000034B03B118477047E4460200E4460200EE
:1002A0000000000010B5064C237843B9FFF7DAFFD1
:1002B000044B13B10448AFF300800123237010BD39
:1002C0007800002000000000E446020008B5044B5E
:1002D0001BB104490448AFF30080BDE80840CFE7F4
:1002E000000000007C000020E446020070B50D46CE
:1002F0001646044610B1081E18BF01200549064BDA
:10030000342298472368324629462046BDE870408B
:10031000184700BF4863010055060000430904491F
:1003200000F01F0001224033824041F82320704733
:1003300000E100E07723584302300323B0FBF3F0E1
:1003400070477723584302300323B0FBF3F04FF498
:100350007A735843704770470139FDD8704700BF22
:10036000F0B505681DB90F4BBDE8F0401847D1F84E
:1003700008C02C460026C2F1010ED4E90137934291
:1003800095BFDB1973449B1ADB199C4507D9236879
:10039000264613B9044B3046E6E71C46EDE7A54276
:1003A000E1D0F7E715060000410600002DE9F0470F
:1003B000D0E90465037E0136DA07044606611FD4DE
:1003C000037E9B071CD4DFF84480DFF8449000F1E3
:1003D0001407CDB16B68AA68F31A934214D3384658
:1003E000C0472B7C012B04D16E603246294638462B
:1003F000C847D4F814A0EB68284698475546E8E764
:10040000237E43F002032376BDE8F087490600000F
:100410006103000038B50D46044610B1081E18BF30
:1004200001203B220549064B9847064B29462046AA
:100430009847054B23600020206138BD5C630100B4
:1004400055060000810D0000AD03000038B50546DB
:10045000003818BF01200849084B53229847084B21
:1004600028469847044620B92846064B9847204618
:1004700038BD6FF01000FBE75C630100550600001B
:10048000D10E0000BD0E00002DE9F3410D460446DB
:1004900010B1081E18BF01201E49DFF890807A2293
:1004A000C047237E04F1140743F001032376294655
:1004B000194B38469847064660B1237E154903F02C
:1004C000FE03002023767F22C0476FF0110002B0A8
:1004D000BDE8F0812269114B6A6029463846984789
:1004E000237E03F0FE032376237E13F002030ED057
:1004F0000B4B01A89847237E03F0FD03237620468B
:10050000084B984701A8084B98473046DFE7184644
:10051000DDE700BF5C630100050600006103000029
:10052000490F0000ED0E0000570F000055060000B7
:10053000014B1860014B184794000020570300003E
:10054000054B10B51C68054B9847054B01462046E6
:10055000BDE81040184700BF94000020350300009C
:1005600059030000054B10B51C68054B9847054B17
:1005700001462046BDE81040184700BF9400002007
:1005800043030000590300000A4A13889BB210B5C8
:1005900043F4A0631380084B9847084B9847084BD7
:1005A0009847084B9847BDE81040074B40F6FF704E
:1005B000184700BF004000413D0A00005B060000F4
:1005C000990600005D060000350900000B4A93788B
:1005D00082B0DBB20193019B990705D5084B1B68DC
:1005E00013B1506802B01847019BDB0704D5044BD8
:1005F0005B680BB1014AF4E702B0704700000241AA
:1006000098000020006800B970478842FAD10120A4
:100610007047000038B5074B0446984780F001004A
:100620000D46054B05493922C0B2984723682B6017
:10063000256038BD05060000550600007363010003
:1006400003680B600160704703680BB11A680260B1
:100650001846704700B900BE704770470C4B0D4AF2
:100660005A63DA6B12F0060FFBD14FF402629A6301
:10067000022283F83020064AD36B9807FCD4044B3F
:100680001A6CD10702D41A6C9207F9D5704700BFD3
:10069000001000404D0E0100014B01225A717047BD
:1006A00000080040C3690B42FCD170470268034B4D
:1006B00042F0020202600321184700BFA5060000B5
:1006C0000268034B22F0020202600321184700BFB8
:1006D000A50600000160014B03211847A506000094
:1006E00070B50C4D06460FCD88B06C460FC495E82A
:1006F0000F0084E80F006A46002352F8041BB14241
:1007000002D1D8B208B070BD0133082BF5D100205A
:10071000F8E700BFAC63010008B5034B98478000C1
:100720002E3000F0FE0008BDE10600004109044A39
:1007300000F01F000123834042F82130704700BFC2
:1007400000E100E04309064900F01F0020330122C8
:10075000824041F82320BFF34F8FBFF36F8F704764
:1007600000E100E04309044900F01F00012260336A
:10077000824041F82320704700E100E070B5194B3A
:100780000446984728B11849184B40F26B220020C4
:100790009847E369164D174E13F0010F0DD1164B14
:1007A00003212046984723689B0703D5134B98479E
:1007B0000221A84705212046B04720460121A8472D
:1007C0000F49B0474FF4403363601F21A8470D4BDA
:1007D000A3604FF61143A3810023A373184684F846
:1007E000303070BDE1060000916301005506000045
:1007F000A5060000D5060000A5060000C106000001
:1008000004001040020070002DE9F743054600384F
:1008100018BF0120144B0C46CB2214499847144BA7
:10082000204698470646D8B9124BAC619C4208BF97
:10083000114BDFF8509008BF1D6020460F4BDFF8CA
:1008400048800F4F9847002405462B19D8B20190D5
:10085000C8470198C04701340198B847042CF4D127
:10086000304603B0BDE8F0835506000091630100F7
:100870007D07000000300040A8000020190700009C
:100880002D07000045070000650700008069014B47
:10089000184700BFAD0600008369996270478369FD
:1008A00001229A757047836902229A757047000089
:1008B000194B186810B58469237EDA0708D5A37D23
:1008C000DB0705D5012323750368BDE810401847F1
:1008D000237E990706D5A37D9A0703D502232375A6
:1008E0008368F2E7237E5B070CD5638B03F0370345
:1008F00013B1FF23638310BDA16A4368BDE81040B4
:10090000C9B21847237EDB09F5D080232376C3685C
:100910009847638B9BB2EDE7A8000020004B184777
:10092000B1080000004B1847B1080000004B184701
:10093000B1080000C30707D5044B054A1A6243F605
:10094000FD7259681142FCD1704700BF001C004085
:1009500007010100FEE7000018491948814210B55F
:100960000AD0184BDA1C121A22F00302C41EA3424A
:1009700038BF0022144B9847144B1548DA1C121A42
:10098000C11E22F00302994288BF0022114B0021B0
:100990009847114A114B22F07F029A60D3F88820C1
:1009A00042F47002C3F88820BFF34F8FBFF36F8FFC
:1009B0000B4B98470B4B9847FEE700BFE4460200FD
:1009C0000000002074000020B562010000C8002073
:1009D00078000020056301000000000000ED00E049
:1009E0004D620100E909000008B5024B024C98472E
:1009F000A047FDE7FD090000350A000010B5074BD0
:100A00009847074B9847074B9847074B9847074B22
:100A10009847BDE81040064B184700BF8905000005
:100A20000D1300006D120000A511000095120000CA
:100A3000B9130000004B184765140000064B42F242
:100A40008E329A8200229A75DA75DA6902F47C5243
:100A5000DA6101221A747047001400400023836297
:100A6000C3690BB108381847704700238362436A93
:100A70000BB108381847704770B50446054BA0F114
:100A800008052C309847236A1BB12846BDE8704002
:100A9000184770BDC90C000070B50E4615460446D7
:100AA00018B1D9B1101E18BF01200F4B0F4940F2E9
:100AB0003B129847B4F84420B4F84C309A420FD116
:100AC0000023A4F844300123236304F10800084BF9
:100AD000A664A4F84C509847284670BD0846E4E741
:100AE0006FF01B00F9E700BF55060000F563010039
:100AF0009F080000838FB0F844209A4210B5044646
:100B00000AD0026C591C8187D15C044B9847044B76
:100B10002046BDE810401847024BFAE7990800004C
:100B20009F080000A70800002DE9F7430E4617466E
:100B3000044618B1E9B1101E18BF01201049114B2D
:100B4000DFF850904FF4AC72984734340E4B01A844
:100B500098470E4B204698470D4B804601A8984772
:100B60000025A84501D0BD4205D1284603B0BDE807
:100B7000F0830846E2E771192046C8470135F0E7DF
:100B8000F563010055060000490F0000090D000043
:100B9000570F0000890C0000F8B50D4616461F4699
:100BA000044620B109B312B3181E18BF0120124920
:100BB000124B3A229847124B3A46314604F1340020
:100BC0009847B0B90F4B294604F10800984758B927
:100BD0000D4B63600D4B23600D4BA3600D4BE36029
:100BE0000D4B23610D4B6361F8BD0846DFE71046EE
:100BF000DDE76FF00C00F7E7F56301005506000034
:100C00004D0C000009080000290B0000990A0000A3
:100C1000F50A0000790A00005D0A00006B0A000076
:100C200010B50446003818BF01200549054B612264
:100C3000984704F10800044B9847002010BD00BFFE
:100C4000F5630100550600008D08000070B50E46E2
:100C50001446054618B189B1101E18BF0120084975
:100C6000084B28229847631E13EA040003BFC5E916
:100C70000130E8602E606FF00C0070BD0846EEE7B2
:100C8000126401005506000038B50D46044610B147
:100C9000081E18BF01200A4B0A4940229847D4E990
:100CA00002329A4209D0626813402268D35C2B70EA
:100CB000A3680133A360002038BD6FF00900FBE793
:100CC000550600001264010038B504460D460C4B71
:100CD0000C49512201209847E3686268134022685A
:100CE000D554D4E90121E368591A914288BF9A1A70
:100CF00003F1010388BFA260E360002038BD00BF9C
:100D0000550600001264010010B50549054B044664
:100D1000672201209847D4E90230C01A10BD00BFF5
:100D2000126401005506000003690B42FCD17047B4
:100D300070B5104D06460FCD88B06C460FC495E8CF
:100D40000F0084E80F006A46002052F8041BB142ED
:100D500002D130B908B070BD01300828F5D10020AB
:100D6000F8E700200449054B4FF49E7298474FF076
:100D7000FF30EFE74C6401003664010055060000C7
:100D80002DE9F843454B814608460C469847444BAD
:100D90004449C9F80C408D228046012098472369B8
:100DA000414A13F0010F11D10321204690472368D7
:100DB0009B0706D5236823F0020323609047022196
:100DC000904701232360032120469047374F142585
:100DD00005FB08750121204690476E6A26600321B5
:100DE000904795F82A30E37306F00C062B8DE380CC
:100DF000082E4FF0010323733AD1EB6AE361C0215F
:100E0000904700232362904701236372284B9C4242
:100E100004BF284BC3F80090142303FB0873B3F9F5
:100E20002230002B0DDB5A09012103F01F039940EA
:100E300002F12003204A42F82310BFF34F8FBFF383
:100E40006F8F142303FB0870B0F92230002B0CDBEA
:100E500003F01F015B099B0003F1604303F561434D
:100E600001228A40C3F880211A600020BDE8F8837F
:100E70002EB9AB8DA383C0219047E683C3E7042E30
:100E8000C2D195F82C302377C02190470023637797
:100E9000904795F82B30E3762021B4E7310D000020
:100EA0005506000036640100290D00004C64010065
:100EB00000380040AC00002000E100E0C06803689A
:100EC00043F0020303600321004B1847290D000083
:100ED00008B5C068034B032198470068C0F3400081
:100EE00008BD00BF290D00000020704710B50A4B57
:100EF000C0689847094B0A49044640F20F12012086
:100F000098470848084B142202FB0400BDE8104033
:100F100090F82200184700BF310D00005506000070
:100F2000366401004C6401001D030000054B186885
:100F3000C3689A7AD20703D501229A7203681847C8
:100F4000704700BFAC000020EFF31083036072B65F
:100F5000BFF35F8F7047BFF35F8F036883F3108821
:100F6000704700004309012200F01F00012902FA26
:100F700000F210D002291FD029BBDB0103F182430C
:100F800003F500435A6091B241F08041120C99621E
:100F900042F040420EE0DB0191B203F1824303F5DF
:100FA000004341F0804141F400315A6099620849A0
:100FB00041EA12429A627047DB0103F1824303F572
:100FC00000439A60DFE70349034B4622002018479D
:100FD000000002C0806401005506000030B54B1CC3
:100FE000C5B2184B00F01F044FEA50104FEAC01072
:100FF000034407D1234493F8402002F0FE0283F813
:10100000402030BD181903EB540390F8402002F043
:10101000FE0242F0010280F8402093F8302015F0E3
:10102000010FC9B219BF02F00F0242EA011202F029
:10103000F00201F00F0114BFD2B20A4383F830204E
:10104000DFE700BF0080004101294FEA501300F0A4
:101050001F000FD002291DD069BB00EBC31000F1A7
:10106000824000F5004090F8403003F0FB0380F828
:1010700040307047DB0103F1824303F500438140B8
:101080001844596090F8402042F0040280F8402053
:1010900099617047DB0103F1824303F500430122AC
:1010A000824018445A6090F8401041F0040180F8E2
:1010B00040105A6170470249024B892200201847AC
:1010C0008064010055060000530010B5540104F47B
:1010D000703403F47C73234302F00704520302F0DC
:1010E000E0522343134303EA010221EA0301826130
:1010F000416110BD38B5054C054B402565619847E9
:1011000080236361A361A56138BD00BF00800041F9
:10111000C91000002DE9F041074F884616461D46CC
:101120000024A54201DCBDE8F08136F814204146D8
:10113000B8470134F5E700BFF51000002DE9F84F7E
:101140004701154BDFF858A0884616465FFA87FB23
:10115000002528FA05F2D20719D5EC19E4B2204689
:10116000717898470BEB05090C4B3178204698476E
:1011700071684846D04704F01F016409E40104F196
:101180008244012204F500448A40034B6261013528
:10119000202DDED1BDE8F88F650F0000491000005A
:1011A000DD0F00002DE9F7434FF000096A46294B97
:1011B000CDF8009002254FF0FF342749DFF8A880D2
:1011C0008DF8015001200194984729460620234FAD
:1011D000234EC04749460620B84721460620B0475F
:1011E00029460420C04749460420B8472146042028
:1011F000B04729460320C04749460320B847214647
:101200000320B04729460520C04749460520B84776
:1012100021460520B04729460720C04749460720F8
:10122000B84721460720B04701216820C04729461A
:101230006820B84721466820B0470A4B40229A618F
:1012400010229A6108229A6180229A6103B0BDE857
:10125000F08300BF3D110000F7C3031C49100000DC
:10126000DD0F000000800041650F000070470000A6
:1012700010B4064CD4E90023501C43F10001C4E92A
:101280000001034B5DF8044B01201847B00000201B
:1012900035DA000070B51248124B134C9847134AC8
:1012A000536943F480435361114B4022C3F8A42097
:1012B000104B984704F11C0502460F490F4B284676
:1012C00098470123236123760D4A0E4B626104F196
:1012D00008012846984728460B4BBDE87040184740
:1012E00010E000E031050000B000002000080040E0
:1012F000001C0040E90E000000380040150400000A
:1013000071120000890400004D040000214B37B524
:101310004022C3F89C204322C3F88C201E4A1F4958
:1013200053691F4D43F4805353611E4A002302F159
:101330001004009320461023A8471B4B93F8D82095
:1013400002F0FE0242F0010283F8D82093F8BC209C
:1013500002F0F00242F0030283F8BC2093F8D92097
:1013600002F0FE0242F0010283F8D92093F8BC207B
:1013700002F00F0242F0300283F8BC2020460B4BF3
:1013800098470B490B4B0C22204603B0BDE8304078
:10139000184700BF001C0040000800400020014129
:1013A000990B0000E800002000800041210C0000A3
:1013B00000000020ED02000030B51A4B1A4C1B4D06
:1013C0008DB098471A4B984700221A4920464FF48F
:1013D0007F53A84701A8184B9847184B049301A8BE
:1013E000174B02949847174B00209847164B002143
:1013F00004469847154B1649054698470022114662
:101400002846144DA847144B002120469847232214
:1014100004465A21A8471149114B204698470DB060
:1014200030BD00BF2D1D0000480100209DD70000E9
:10143000E51400006C0100205DD700008916000053
:10144000BDD700007118000019470100C544010014
:10145000A8640100A1280000315901009C6401002A
:1014600035560100004B1847FDF90000094908B541
:1014700040234B61084B0246187818B92020486178
:1014800001211970054B064906489847014B402237
:101490009A6108BD008000410C000020F51000009A
:1014A000F7C3031C80800041094908B540234B6104
:1014B000084B0246187818B1202088610021197065
:1014C000054B064906489847014B40229A6108BDE2
:1014D000008000410C000020F5100000F7C3031C41
:1014E000808000412DE9F84300BF5F4F5F4E10241C
:1014F000BC613220B0477C6100BF3220B047BC6184
:101500003220B04700BF4FF040080A20C7F81480CF
:10151000B0470520C7F81880554D564CDFF860914C
:10152000B0470120A8471420B0470120A847142045
:10153000B0470120A8471420B047E220C7F8148024
:10154000A8472F20A0470320A0475420A047E02011
:10155000A8470120A047484B64209847E020A847AF
:101560000320A0470120B0470120A8470120B04731
:10157000E620A8470120A047CC20A047CC20A047C8
:10158000B020A8472820A0473C4E8020A047B04765
:10159000C8470138C0F30720A047B047C847013803
:1015A000C0B2A047DFF8DC90B047C8470138C0F3AD
:1015B0000720A047B047C8470138C0B2A047002065
:1015C000A047F020A8470320A0473A20A84755206D
:1015D000A047B420A8470220A0470D20A047002024
:1015E000A0472B20A0472820A0470020A04700208C
:1015F000A0470020A047B620A8470120A0471D20F3
:10160000A0470020A0470C20A0470920A0470020A9
:10161000A0470020A0472A20A8470020A04700207C
:10162000A0470120A047DF20A0472B20A84700208B
:10163000A0470020A0470120A0470F20A047292055
:10164000A847BE20A8470620A047FF20A0470120AA
:10165000A047FF20A0470020A0470120A047C7F8CF
:101660001880BDE8F88300BF0080004165050000D8
:101670006D140000A914000041050000FDD8000011
:1016800009D900002DD900002DE9F04FB1F904303F
:101690002DED028B002B08EE100A81B00D4690460E
:1016A000C0F28280B1F90630002B7DDB414FDFF8BC
:1016B00018A1B847D047B5F90030834274DAB8476B
:1016C000DFF808B1D847B5F90260B0426CDDB5F972
:1016D0000040B847D047B5F90430984224EAE47492
:1016E00026EAE67653DCB847D04700F1FF3AB84720
:1016F000D847B5F9063098424BDCB847D847471E63
:10170000DFF8CC90DFF8CCB02A20C847C4F307201C
:10171000D847E0B2D847CAF30720D8475FFA8AF023
:10172000D8472B20C847C6F30720D847F0B2D84780
:10173000C7F30720D847F8B2D8472C20C847AB8852
:101740002A8801339D1A1C4A1C4B1178ADB219B17D
:101750002021996100211170C4F1010440225A61D5
:101760001748DFF874B004EB0A03DFF870A09CB2EE
:101770006D00BE420FDD114B40229A6118EE100A37
:10178000104B01B0BDEC028BBDE8F04F18479A46F4
:10179000ADE71F46B4E74246234651460136D847D7
:1017A000A844074836B2E4E701B0BDEC028BBDE8BF
:1017B000F08F00BFFDD800000C0000200080004129
:1017C00080800041B9D9000009D900002DD900005E
:1017D0006D140000A914000015110000F7C3031CCC
:1017E000003818BF01207047F0B51B4BC3B0074647
:1017F00016469847E528044629D802AD0246174BFD
:101800003946284698472B1920222A5528225A70F3
:1018100030229A70124C7822DA70181D1C2226FA97
:1018200002F101F00F012144043AC97C00F8011BC8
:10183000111DF4D129221A7300225A73094B009505
:10184000BC220949094C0320A04743B0F0BD054B19
:101850000097BF22F5E700BF3963010031EC0000BB
:1018600019EB01003DEB01000FEA0100E9E800007F
:1018700037B5044670B9084B9847044650B9074B32
:1018800000930749074B084D2E220220A847204607
:1018900003B030BDE46BFAE7FDD8000080EB010037
:1018A00050EB0100F0EC0100E9E8000037B5044618
:1018B00070B9084B9847044650B9074B0093074945
:1018C000074B084D4B220220A847204603B030BDED
:1018D000246CFAE7FDD80000B9EB010050EB0100E1
:1018E00004ED0100E9E8000037B5044670B9084B83
:1018F0009847044650B9074B00930749074B084DDA
:101900005C220220A847204603B030BD646CFAE791
:10191000FDD80000F2EB010050EB01001AED0100D0
:10192000E9E8000070B5094D002428B964B12046EB
:10193000074BBDE87040184790F8343013F0200F83
:1019400018BF0446A847F0E770BD00BF252100007E
:10195000112800002DE9F347067D16F00106054623
:10196000884617465CD1C468DFF8C8A04FF001096B
:10197000002C4CD12B7DDB0601D4002E50D1B9F1C7
:10198000000F4DD02846C0470446002E3AD100280B
:1019900046D006464FF000092068D047024600288E
:1019A000E6D1EB68A3423BD01F4E7BB11868019291
:1019B000C36917219847EB68019A18680E21B04750
:1019C00001282DD1EB681868184B98472068EC6007
:1019D000C369002216219847EB68002218680D2180
:1019E000B04701281CD1EB681868114B9847EB6889
:1019F00018680E4B98472B6993B1284602B0BDE892
:101A0000F04718474FF00009002CC5D1B2E7214636
:101A10002846B847002E08BF2646B0420446F3D1F8
:101A200002B0BDE8F08700BF791F000085270000E5
:101A3000251900001D2600000148024B18211847F7
:101A40004886002005E60000014A0249024B18477B
:101A5000B5E60000A9E6000055190000014A024958
:101A6000024B1847D5E60000AFE60000551900000C
:101A700038B5037DC3F3001543F010030375044626
:101A80001B0754BF034B044B9847237D65F3041396
:101A9000237538BD491A00005D1A00002DE9F34195
:101AA0000D460446002836D0DFF8C480244EC047D7
:101AB00030BBAB6B73B1234B2846984750B1A86B32
:101AC000214B224E9847224B00932249224B7F22E2
:101AD0000120B047214BAC6320469847204B064677
:101AE00098470746F0B91C4B1A49009385220320FA
:101AF000164CA0471B481C4932463B468847FEE728
:101B00000368AB420AD1194B00931249124B0F4C98
:101B100075220120A04702B0BDE8F08101462046B1
:101B2000B047C5E7002EF6D035602046C047864254
:101B3000F1D1054B204602B0BDE8F041184700BF87
:101B4000B5E60000F9410000711A0000E9E8000064
:101B500008EE01008DED01004AEE010061E6000093
:101B6000E1170000BEED0100E9170000CCED010017
:101B7000A9E60000F8B5846B0646002C33D0E36874
:101B8000002B30D01B681C4D83421BD1237DDA070C
:101B900044BF6FF3000323752046A847E3688342E0
:101BA00022D1164B20469847E36898421CD1006822
:101BB0000022C36917219847E3681B68B34204BF3A
:101BC0000023E3602046A8470D4F05465DB12B6812
:101BD000B342294620460BD10A4B98470A4B284668
:101BE00098470023B363F8BD084B20469847E3E7C6
:101BF000B8470546EAE700BFA9E60000AFE60000E7
:101C0000B5E600006DE70000E5EA0000711A00008B
:101C100010B1C06800B10068704710B1007DC0F31A
:101C200040007047F8B50C4D0C4E04460020A84704
:101C3000002700B9F8BD90F8503043F0020380F857
:101C400050307368984208BF376014B1C36B9C4230
:101C500000D1C763A847ECE719DA0000EC80002048
:101C6000014B0020184700BF251C0000014B58689D
:101C7000704700BFEC800020034690B190F85020E0
:101C800042F0020280F85020084A5068984204BF8F
:101C90000020106011B1DA6B8A4205D10022DA63AC
:101CA0007047034B08461847704700BFEC80002080
:101CB000251C0000014B1868704700BFEC80002015
:101CC0002DE9F047051D124BDFF8489028460E46D7
:101CD000174698471FFA86F804461FFA87FA0CB988
:101CE000BDE8F087238A43442382638A5344638296
:101CF000A38A4344A382E38A5344E38220463A46BC
:101D00003146FFF7DDFF21462846C8470446E6E78F
:101D1000A9E60000B5E60000013900F1080311F85A
:101D2000012F00F8012B9842F9D17047F0B5204EF1
:101D3000204D337885B043B11F4B00931F49204B92
:101D400078220220A84705B0F0BD1E4B1E4C1F4F45
:101D500098471F4B98471F4B98471F4B98471F4B5F
:101D600098471F481021A0471E4B009302224FF0B6
:101D70001F01CDE901334FF60000B8471A4B9847D1
:101D80001A4B98471A484FF4B871A0476021194878
:101D9000A047194B9847194B9847194B0120984772
:101DA000184B00930120064B04493070A222C9E76A
:101DB000F4800020E9E800008AEE01005BEE0100FB
:101DC00062F0010015EA000005E6000009250100A7
:101DD00031F80000D9E3000031DC0000391A0000BE
:101DE0006086002010000020CD020100094F000095
:101DF0000C86002018860020611C0000D5D0000051
:101E0000A9C60000A2EE010073B50E4B04460E46B3
:101E10009847054668B90C4B0C49009340F2945220
:101E200003200B4EB0470B480B4922462B468847F0
:101E3000FEE794F8343066F3C71384F8343002B008
:101E400070BD00BFE1170000B7F001005BEE0100BC
:101E5000E9E80000BFEE0100E917000073B50E4B82
:101E600004460E469847054668B90C4B0C4900934A
:101E70004FF4B46203200B4EB0470B480B49224687
:101E80002B468847FEE794F8343066F3000384F865
:101E9000343002B070BD00BFE1170000CEF0010089
:101EA0005BEE0100E9E80000BFEE0100E917000069
:101EB0002DE9F043804687B016461F460C4691B187
:101EC000244B08469847054668B9234B234900939D
:101ED0004FF4DB620320224EB047224822492246BB
:101EE0002B468847FEE7214D039400238DF81030E0
:101EF0006B68059303AB6B601D4BD5F80890AF6022
:101F0000984718B183680BB131469847B8F1000F74
:101F100002D031462046C0476B68C5F808909B68E0
:101F20006B609DF8103083B98CB194F834305A0648
:101F30000DD5206858B10F4B3A4631469847431E9D
:101F40005842584107B0BDE8F0830020FAE701206D
:101F5000F8E700BFE117000093F101005BEE01001C
:101F6000E9E80000BFEE0100E9170000F48000205E
:101F70006D1C0000791F00007FB50E4603920446D9
:101F8000D8B10F4A9047039B054668B90D4B0E49DF
:101F9000009340F2C46203200C4EB0470C480D4938
:101FA00022462B468847FEE7A06921460A4C324666
:101FB000A44604B0BDE870406047012004B070BD85
:101FC000E1170000A6F101005BEE0100E9E8000066
:101FD000BFEE0100E9170000B11E000073B50B4B06
:101FE00004460E469847054668B9094B09490093CF
:101FF00040F21B720320084EB047084808492246A9
:102000002B468847FEE7E66102B070BDE11700008D
:10201000B4F101005BEE0100E9E80000BFEE010051
:10202000E917000010B1C36903B1184701207047D8
:1020300073B50B4B04460E469847054668B9094BE5
:102040000949009340F237720320084EB047084810
:10205000084922462B468847FEE7266202B070BD3B
:10206000E1170000C9F101005BEE0100E9E80000A2
:10207000BFEE0100E91700007FB50E4B0391044647
:1020800098470399054668B90B4B0C49009340F2F9
:10209000497203200A4EB0470A480B4922462B4694
:1020A0008847FEE7606A094B984700B1606204B058
:1020B00070BD00BFE1170000DEF101005BEE010022
:1020C000E9E80000BFEE0100E917000015EE00008E
:1020D00073B50E4B04469847054668B90C4B0D493D
:1020E000009340F2597203200B4EB0470B480C4945
:1020F00022462B468847FEE7E36900220621204658
:10210000628602B0BDE87040184700BFE1170000CA
:10211000F7F101005BEE0100E9E80000BFEE01000D
:10212000E917000073B50B4B04469847054668B99C
:10213000094B0A49009340F29F720320084EB047B2
:102140000848094922462B468847FEE7206802B026
:1021500070BD00BFE117000013F201005BEE01004B
:10216000E9E80000BFEE0100E917000073B50E4B6F
:1021700004469847054648B10C4E2046B0472546D0
:1021800004460028F9D1284602B070BD084B094921
:10219000009340F26B720320074EB047074808498E
:1021A00022462B468847FEE7E11700002521000064
:1021B00025F201005BEE0100E9E80000BFEE01003E
:1021C000E91700002DE9F7431E4B054698470446E2
:1021D00068B91D4B1D49009340F27F7203201C4ECD
:1021E000B0471C481C492A4623468847FEE72B680F
:1021F0001BB12846194B984705461948194E1A4FE6
:10220000DFF85C80B047044664B9184B00930F496F
:102210000D4B0F4D4FF4F2620220A847204603B049
:10222000BDE8F08304F130094846B04720B92146A3
:102230004046B8470446E7E78542EFD001464846A6
:10224000B847F3E7E117000037F201005BEE010049
:10225000E9E80000BFEE0100E91700006D21000071
:102260000C860020A9E60000B5E60000CCEE0100D7
:1022700073B5104B04460D469847064668B90E4B99
:102280000E49009340F2AD7203200D4DA8470D4852
:102290000D49224633468847FEE7201D25B90B4BE2
:1022A00002B0BDE870401847094B294602B0BDE8AE
:1022B00070401847E117000047F201005BEE010093
:1022C000E9E80000BFEE0100E9170000A9E6000000
:1022D000B5E6000073B50E4B04460E46984705461A
:1022E00068B90C4B0C49009340F6010203200B4ED9
:1022F000B0470B480B4922462B468847FEE70A4B5E
:1023000004F11001304602B0BDE87040184700BF2C
:10231000E1170000B8F201005BEE0100E9E80000FF
:10232000BFEE0100E9170000191D000073B5104B46
:1023300004469847054668B90E4B0F49009340F68E
:10234000220203200D4EB0470D480E4922462B466F
:102350008847FEE70C4B2046984728B1238A028A1B
:10236000981A00B202B070BDB4F91000FAE700BFCD
:10237000E1170000CAF201005BEE0100E9E800008D
:10238000BFEE0100E91700002521000073B5104BD6
:1023900004469847054668B90E4B0F49009340F62E
:1023A000360203200D4EB0470D480E4922462B46FB
:1023B0008847FEE70C4B2046984728B1638A428A3B
:1023C000981A00B202B070BDB4F91200FAE700BF6B
:1023D000E1170000D7F201005BEE0100E9E8000020
:1023E000BFEE0100E91700002521000073B50D4B79
:1023F00004469847054668B90B4B0C49009340F6D4
:102400004A0203200A4EB0470A480B4922462B468F
:102410008847FEE7A38A228A0133981A00B202B0E5
:1024200070BD00BFE1170000E4F201005BEE0100A7
:10243000E9E80000BFEE0100E917000073B50D4B9D
:1024400004469847054668B90B4B0C49009340F683
:10245000560203200A4EB0470A480B4922462B4633
:102460008847FEE7E38A628A0133981A00B202B015
:1024700070BD00BFE1170000F5F201005BEE010046
:10248000E9E80000BFEE0100E917000013B511B93B
:10249000283002B010BD8DF800100024044B0194C8
:1024A0006A460821984701280CBF01982046F0E7AA
:1024B000252000002DE9F84F0746984619481A4B89
:1024C000DFF86090DFF87CB00D461646984704466A
:1024D0000CB9BDE8F88F4445FBD0144B2146484663
:1024E000984782462068B8421AD1A179A94201D002
:1024F000FF2D15D1A288B24201D0FF2E10D1D847AE
:102500000B4A9047A1880B4A90470B4A002120466E
:1025100090470A4A484621469047094A2046904734
:102520005446D5E760860020AFE60000D5E60000FF
:10253000B95C000011580000B1DC00006DE700003C
:10254000E5EA00008D24000037B50E4B04460D4629
:10255000984750B90C4B00930C490D4B0D4C40F271
:1025600092420220A04703B030BD0B4B9847204653
:102570000A4C0023FF222946A44603B0BDE83040A0
:10258000604700BF8D24000014EF01005BEE0100E6
:10259000B1F30100E9E80000C95C0000B5240000C7
:1025A0002DE9F041154B04681548154E154F984715
:1025B000002590B945B9A179134B20689847134B72
:1025C0009847A188124B98470D48124B21469847CF
:1025D0002046114BBDE8F0411847A0420AD00268DE
:1025E00023689A4206D143686268534033F07F43C0
:1025F00008BF012501463046B847DAE7A9E60000E2
:1026000060860020B5E600008D240000B95C000063
:10261000115800006DE70000E5EA000073B50C4BAF
:1026200004469847054668B90A4B0B49009340F6A3
:1026300041220320094EB04709480A4922462B4649
:102640008847FEE794F83400C0F3001002B070BD74
:10265000E1170000FFF301005BEE0100E9E8000074
:10266000BFEE0100E91700002DE9F041354B86B0BF
:10267000044688469847054668B9334B334900936A
:102680004FF4F0720320324EB047324832492246AE
:102690002B468847FEE7314F2046B847002841D1F6
:1026A0002F4B204698472F4B054698472E4B064602
:1026B000984785422CD1B4F932502C4B04F11001CB
:1026C00002A89847BDF80820ABB2D21AADF808208E
:1026D000BDF80A20264DD21AADF80A20BDF80C200C
:1026E0001A44ADF80C20BDF80E204146134404A84E
:1026F00002AAADF80E30A847A0B1DFF884802046CA
:10270000C047044688B91B4B04A93046984709E0E6
:10271000194B304698478542CDD0184B30469847E4
:102720008542C8D006B0BDE8F08104A904F11002CA
:102730000846A8470028F5D02046B8470028F1D120
:102740002046DDE7E117000011F401005BEE010017
:10275000E9E80000BFEE0100E91700001D260000B7
:102760006D210000C521000071180000191D000036
:102770008DDE00000D4F0000AD180000E9180000CC
:10278000252100007FB51A4B05469847044668B9D5
:10279000184B1949009340F20D220320174EB04701
:1027A000174818492A4623468847FEE7B5F93240BC
:1027B000154B05F1100102A89847BDF80820A3B2F7
:1027C000D21AADF80820BDF80A20D21AADF80A20B6
:1027D000BDF80C201A44ADF80C20BDF80E201344AF
:1027E000ADF80E3002A9094B2846984704B070BDD9
:1027F000E117000028F401005BEE0100E9E80000A9
:10280000BFEE0100E9170000191D00006926000055
:10281000F7B5194B05469847044668B9174B184950
:10282000009340F262220320164EB0471648174923
:102830002A4623468847FEE7154B28469847071D3A
:10284000144B044638469847854213D0124E204612
:10285000B0472A46394638460123104FB847E36946
:102860002A460121204698472046334603B0BDE85A
:10287000F040184703B0F0BDE11700003AF4010042
:102880005BEE0100E9E80000BFEE0100E91700007F
:1028900025210000A9E6000085270000EDE70000E3
:1028A0002DE9F0432E4B87B00446884617469847DB
:1028B000054668B92B4B2C49009340F29622032021
:1028C0002A4EB0472A482B4922462B468847FEE726
:1028D00026685EB9284B00932349224B234C4FF4C2
:1028E00027720220A04707B0BDE8F083228A338A0E
:1028F0009B1A03EB0801628A738A9B1ADA1997B252
:102900001FFA81F812B258EA07030DB20392EAD017
:102910002046DFF87090C84704A92046174B984717
:10292000238A039A43442382638A3B446382A38AB3
:102930009844E38AA4F814801F4429462046104B8B
:10294000E7829847E36904AA022120469847F36981
:1029500022460121304698472046C847C3E700BFBA
:10296000E117000068F401005BEE0100E9E80000F7
:10297000BFEE0100E91700004AEF0100D522000078
:10298000C11C00008527000073B50F4B04460E469E
:102990009847054668B90D4B0D4900934FF43372C3
:1029A00003200C4EB0470C480C4922462B46884762
:1029B000FEE70B4B204698470A4B0246314620461D
:1029C00002B0BDE870401847E117000077F401003D
:1029D0005BEE0100E9E80000BFEE0100E91700002E
:1029E0008D230000A128000073B50F4B04460E464E
:1029F0009847054668B90D4B0D4900934FF4367260
:102A000003200C4EB0470C480C4922462B46884701
:102A1000FEE70B4B204698470A4B014632462046BC
:102A200002B0BDE870401847E117000084F40100CF
:102A30005BEE0100E9E80000BFEE0100E9170000CD
:102A40002D230000A12800002DE9FF47DFF8D8A0C2
:102A5000BDF9308004460D4617461E46D0478146D4
:102A600068B92A4B2A49009340F26D320320294D60
:102A7000A8472948294922464B468847FEE71DB901
:102A8000274B2046984705462846D047814668B9D7
:102A90001E4B1F49009340F2713203201D4CA0478A
:102AA0001D481E492A464B468847FEE73A4604F130
:102AB000100103AB05F11000DFF87090C847184B08
:102AC00020469847BDF80E20BDF80C10B0F9123022
:102AD000008A42443144091AD21A09B212B2114B87
:102AE000ADF80C102046ADF80E20984794F8493008
:102AF00084F848706FF34103A4F84460A4F846805A
:102B0000256484F8493004B0BDE8F08791F40100F1
:102B10005BEE0100E9E80000BFEE0100E9170000EC
:102B200025210000A1280000E117000031E100008C
:102B30002DE9F04F87B0CDE90323DFF8A4B1BDF94B
:102B40004030059380460E46D847044668B95A4B34
:102B50005A49009340F295320320594DA8475948ED
:102B60005949424623468847FEE7584BDFF874919F
:102B700040469847564B044640469847554A824639
:102B80004046904705464046C84707461EB9524949
:102B90004046884706463046D8474E4A834668B97D
:102BA000454B4649009340F2A1320320444CA047D4
:102BB0004448454932465B468847FEE7039B05EBA0
:102BC000D57507EBD77745F34F0547F34F07142B20
:102BD00024D8DFE803F00B5819615E4B6B5B665835
:102BE00019615E4B6B585B5E61666B0030469047C7
:102BF00000EBD070C5EB600424B23046C84700EB50
:102C0000D070C7EB600307E03046904700EBD07010
:102C1000C5EB600424B27B420FFA83FA2E4A404689
:102C20009047049B318A028A19442144059B891AE2
:102C3000728A1A44438A5244D21A12B2274B09B2FA
:102C400040469847039B88F84830049BA8F84430D6
:102C5000059BA8F8463098F84930C8F8406043F022
:102C6000020388F8493007B0BDE8F08F304690473E
:102C700000EBD070C5EB600424B23046C847C01BDF
:102C80000FFA80FACAE76D422CB2C4E76D422CB24B
:102C9000B3E76D422CB2F0E730469047401B04B2D8
:102CA000B9E730469047401B04B2A6E7304690474C
:102CB000401B04B2E1E700BF9EF401005BEE01009F
:102CC000E9E80000BFEE0100E91700002D23000035
:102CD0008D230000ED23000025210000A128000025
:102CE000E11700003D24000073B5124B04469847DD
:102CF000054668B9104B1149009340F22A4203205F
:102D00000F4EB0470F48104922462B468847FEE732
:102D100094F84950B4F94600216C94F84820B4F96D
:102D2000443000902046AC074CBF084C084CA047EC
:102D300002B070BDE1170000B1F401005BEE0100CC
:102D4000E9E80000BFEE0100E9170000312B0000A8
:102D5000492A0000F8B500210B4E0C4F0546B0473C
:102D6000044604B9F8BD2046B847E36900220421AF
:102D7000204698472046B8472046FFF7EBFF2146FC
:102D80002846B0470446ECE7712200008527000082
:102D900073B5364B05460C469847064668B9344B22
:102DA0003449009340F21D520320334CA04733486E
:102DB00033492A4633468847FEE7902C314E38D8AF
:102DC000722C19D8532C2ED83F2C22D8072C25D85A
:102DD000012C18D92846B047EB6900220421284667
:102DE0009847182C34D8142C34D9286890B3C36968
:102DF0000022012198472DE0A4F17302224B92B2E8
:102E0000D340DA07E6D42846334602B0BDE8704026
:102E10001847A4F140021D4B92B2F1E7A4F1100350
:102E2000082BF0D8D6E75C2CD4D0A4F17003012B8A
:102E3000F7E748F281039C4206D848F27F039C42A0
:102E4000C8D8FF2CDFD1C5E748F28E039C42F9E7D2
:102E5000FF2CCAD02846B047FF2C01D0230402D54E
:102E60000B4B2846D1E702B070BD00BFE117000050
:102E7000C0F401005BEE0100E9E80000BFEE0100D4
:102E8000E917000085270000071A002003100F0033
:102E9000552D000010B5044B044698472046034BBF
:102EA000BDE81040FF21184749250000912D000082
:102EB000F8B51E4C06460D460027F9B22846A04735
:102EC0000246F8B101794FF0000C5FFA8CF3994299
:102ED00015D9507900F00600062823D10133DBB262
:102EE000994216D9106850F823309E4203D00CF155
:102EF000010C002EE9D10E4BFF21284698470137DF
:102F0000402FDAD10B4F00212846B847044610B9AC
:102F1000F8BD0023E9E721463046FFF7C9FF214607
:102F20002846F2E70029DDD10B46DEE78D240000BC
:102F3000912D0000712200002DE9F84F0F4FDFF8AE
:102F40004090DFF840A006460020B84704460CB980
:102F5000BDE8F88F04F130084046C847DFF828B0D4
:102F600005461DB92046B8470446F0E729463046D5
:102F7000D04729464046D8470546F2E7C5D9000064
:102F8000A9E60000B12E0000B5E600002DE9F041F1
:102F90003B4B04460D46817900689847394B98476A
:102FA000A18801F00F03082B16D84DB9B4F90820F9
:102FB000354B9847A1882068344BBDE8F04118474D
:102FC000FF2DB4F90C20F3D0B4F90830D21A6A43BB
:102FD00003EB22231AB2EBE70B2B38D8002D03DCCE
:102FE00022892B4B9847E5E7FE2D01DDA289F8E702
:102FF0002389A28994F808C0C5F1FF07C3F34513DC
:103000007B43C2F3451215FB0232237B0CF01F0CED
:1030100007FB0CFC03F01F0348F2810615FB03C3FA
:1030200072437343C3F3C45394F809C0C2F3C55247
:1030300043EA4212637B4FEADC0CDB0807FB0CF728
:1030400015FB03737343DB0D42EAC322C9E70D2B63
:103050000FD8002D03DC227A0E4B9847AAE7FE2DED
:10306000227BF9DC237AD21A6A4303EB2223DAB2F9
:10307000F2E77F2DD4BFA268E268074B984799E733
:103080008D240000B95C000079580000912D0000EB
:1030900049590000195A0000ED5A000073B50B4B56
:1030A00005469847044668B9094B0A49009340F61B
:1030B000B1220320084EB047084809492A46234652
:1030C0008847FEE7002002B070BD00BFE117000096
:1030D00081F501005BEE0100E9E80000BFEE0100B0
:1030E000E91700002DE9FF470D460646002877D175
:1030F000894B9847044640B9884B00938849894BCF
:10310000CF220220884DA84716E0884B30309847E0
:10311000874B04469847074660B9824B8049009325
:10312000D4220320804DA8478248834922463B464B
:103130008847FEE724B90024204604B0BDE8F087A4
:103140004C217E4B2046984794F83530A66166F3B3
:10315000051384F835307A4BE3617A4B236226619C
:10316000794B304698470138A082784B30469847D3
:103170000138E082764B4C21201D9847B4F8483046
:1031800023F4FF7323F00103A4F84830A38E23F443
:103190007F6323F00F0343F4E063002243F0010355
:1031A00004F12800A386C4E910226A4B2263A263BB
:1031B000A2876262039098470398002D40F0D88060
:1031C000654B002E00F09D80022120469847F36950
:1031D0002246012130469847604B2046984793E0AD
:1031E000534FB847044660B94E4B4D490093ED220A
:1031F00003204D4DA8475A484F4932462346884739
:10320000FEE74A4B301D98470446B847074660B969
:10321000444B43490093F0220320434DA8474548BF
:10322000454922463B468847FEE7002C83D0434B66
:10323000DFF838914C212046984794F835302660C5
:103240006FF3051384F835303D4BE3613D4B23624A
:103250004FF00008B6F912306382C4F81880404677
:10326000778AC8474FF0320A00FB0AF0EF282CDDBE
:103270004046C847502300FB0A30A02390FBF3F0E0
:1032800080B20744E782374B20469847012807461B
:103290001DD1B6F91480A4F814800020C8474FF05F
:1032A000640A00FB0AF0EF281FFA88F808DD002006
:1032B000C847502700FB0A77A02397FBF3F7BFB25C
:1032C000A8EB0708A4F8108054E70120D9E7B6F965
:1032D000107027820020C8474FF0640800FB08F0F8
:1032E000EF28BFB20BDD0020C847502300FB083099
:1032F000A02390FBF3F080B20744A7823AE70120B5
:10330000FAE7012120469847174B00930449054BE3
:1033100040F287120120F5E6FDD80000B0EF010071
:103320005BEE010095F50100E9E8000019E60000F8
:10333000E1170000BEED0100E917000019F00000E0
:103340002D4B00009D45000009D900002DD900003B
:1033500005E600003D550000E5020100852700005C
:10336000BFEE01009D30000000F0010051D90000C7
:10337000544B05F128019847534B04F1100005F117
:1033800010019847B5F93230638695F8303084F8EB
:10339000303095F8313084F8313095F8483084F881
:1033A0004830B5F94430A4F84430B5F94630A4F8B3
:1033B00046302B6C95F84920236494F8493062F329
:1033C000000384F84930AB69A36195F8343094F870
:1033D0003420DB0963F3C71284F8342095F83420D5
:1033E00094F8343062F3000384F8343095F83430C4
:1033F00094F83420C3F3400363F3410284F834208B
:1034000095F8353094F83520C3F3420363F3430253
:1034100084F8352095F8343094F83420C3F38003D1
:1034200063F3820284F8342095F83430D2B2C3F3C7
:10343000C00363F3C30284F8342095F83430D2B269
:10344000C3F3001363F3041284F8342095F8343086
:10345000D2B2C3F3401363F3451284F8342095F8D5
:103460003430D2B2C3F3801363F3861284F834206D
:1034700095F83C3084F83C3095F8352094F8353098
:1034800062F3000384F83530A86B10B10F4B21466E
:1034900098470F4B2846984778B1002E3FF434AF39
:1034A0000C4B284698470C4B0390284698470399A5
:1034B0000A4B02462046984789E6002E7FF487AEE5
:1034C00022E700BF2D5D0000191D00009D1A0000BD
:1034D000252100002D2300008D230000A1280000DD
:1034E0002DE9FF41334B04460D46174698470646E3
:1034F00068B9314B3149009340F2E5220320304D49
:10350000A84730483049224633468847FEE72F4BCC
:1035100020469847854204D12D4B20469847874244
:103520003AD020462B4EB04702A92B4B2046984755
:10353000638A013F1F44E782284B204698470128B1
:10354000ADB20BBFA38A238AC5F1010505F1FF3592
:103550000ABFED18ED182582E36918BFA58202AAFB
:103560000221204698471E4B2046984718B1C36950
:10357000224601219847271D1A4BDFF870803846F4
:10358000984705465DB92046B04794F84930DB07B7
:1035900002D5154B2046984704B0BDE8F081EB6991
:1035A00002AA03212846984729463846C0470546BF
:1035B000E8E700BFE1170000B5F501005BEE010090
:1035C000E9E80000BFEE0100E9170000ED2300006C
:1035D0003D24000085270000D52200009D3000001A
:1035E00025210000A9E60000E92C0000B5E6000056
:1035F00073B50F4B04460E469847054668B90D4B08
:103600000D49009340F2273203200C4EB0470C487E
:103610000C4922462B468847FEE70B4B204698472D
:103620000A4B01463246204602B0BDE870401847BA
:10363000E1170000D6F501005BEE0100E9E80000AB
:10364000BFEE0100E9170000ED230000E1340000A7
:1036500073B50E4B04460E469847054668B90C4BA9
:103660000C49009340F6D72203200B4EB0470B487D
:103670000B4922462B468847FEE794F83C301E4211
:1036800014BF0120002002B070BD00BFE117000090
:10369000FBF501005BEE0100E9E80000BFEE010070
:1036A000E91700007FB5134B04460D4698470646C0
:1036B00068B9114B1149009340F6DE220320104DEA
:1036C000A84710481049224633468847FEE73F2D59
:1036D00003D894F83D0004B070BD00238DF80D3080
:1036E00003AA0A4B8DF80C500921204698479DF8F3
:1036F0000D00F0E7E11700000FF601005BEE01009E
:10370000E9E80000BFEE0100E917000025200000F5
:103710002DE9F74FDFF894A0DFF894B005460E4688
:1037200017464FEA1228144665B924F4FE44222CA9
:10373000A0B230D027D803282FD0C21F504250410A
:10374000000213E0174B3146284698473146814620
:103750002846D04707EB002084B20DF1060221462F
:103760004846D847012804D1BDF9060003B0BDE89A
:10377000F08F18F0800FD8D01EB928460A4B984712
:1037800005460026D0E7312809D0A0F1C0035842F1
:1037900058410001EAE7FF20E8E70620E6E70F20AE
:1037A000E4E700BF8D24000025210000A5360000BD
:1037B0008D5E00002DE9F74FDFF874A0DFF874B0DC
:1037C00005460E4617464FEA122814464DB924F412
:1037D000FE44293C012C96BF124B0020B3F8020690
:1037E00012E0114B3146284698473146814628461B
:1037F000D04707EB002084B201AA21464846D847AB
:10380000012804D1BDF8040003B0BDE8F08F18F022
:10381000800FDCD01EB92846044B98470546002689
:10382000D4E700BF62F001008D24000025210000D4
:10383000A5360000155F00002DE9F74FDFF880A0E6
:10384000DFF880B005460E4617464FEA12281446A8
:1038500075B924F4FE446D2CA0B22AD048F2AD0311
:10386000984226D02C3818BF4FF0FF30C0B213E07A
:10387000114B314628469847314681462846D04765
:1038800007EB002084B20DF1070221464846D847D5
:10389000012804D19DF8070003B0BDE8F08F18F0AF
:1038A000800FD6D01EB92846044B984705460026FF
:1038B000CEE70020F0E700BF8D24000025210000A6
:1038C000A53600009D5F00002DE9F74FDFF884A0CA
:1038D000DFF884B005460E4617464FEA1228144614
:1038E0006DB924F4FE44BE2CA3B227D048F28E0258
:1038F000934201D07E2B23D1124B984711E0124BFB
:10390000314628469847314681462846D04707EB3E
:10391000002084B201AA21464846D847012803D195
:10392000019803B0BDE8F08F18F0800FD9D01EB910
:103930002846064B984705460026D1E70448F0E79D
:103940000020EEE7D90201008D24000025210000AF
:10395000243F0200A53600002560000070B5046811
:10396000A5882068A17905F00F03082B2A460CD8FA
:103970000D4B984720810023A380A17920680B4E2E
:1039800023462A46B047A58070BD0B2B02D8084BB2
:103990009847EFE70D2B03D8064B98472072EAE7CC
:1039A000054B9847A060E6E711370000B5240000FA
:1039B000B537000039380000C93800002DE9F04F54
:1039C00090F83D308B429FB00446884600F042821A
:1039D000954B9847054668B9944B9549009340F23A
:1039E00037620320934EB0479348944922462B46B2
:1039F0008847FEE794F83D300293002384F83D8029
:103A000003939DF80C608E4B3146204698470590F5
:103A100040B1477917F008070BD0039B0133402BC7
:103A20000393EED1874BFF2120461FB0BDE8F04F36
:103A30001847854DB02231462046A847B12209904B
:103A400031462046A847814B0890BE223146204689
:103A50009847B222069031462046A847B322ADF8D7
:103A60002C0031462046A847B422ADF82E0031463E
:103A70002046A847B522ADF8300031462046A84779
:103A8000B622ADF8320031462046A847B722ADF83D
:103A9000340031462046A8470497ADF83600049A12
:103AA0000BAB33F81270002F00F0B680684B05980E
:103AB0009847634B314620469847664B05469847E2
:103AC00007F00F03082B824600F2DC806B79DFF8E9
:103AD00078B143F004036B71029B84F83D303A46A1
:103AE00031462046D8473A46079084F83D80314613
:103AF0002046D8476A79079B6FF38202834281464A
:103B00006A7100F08980029B84F83D303A46314664
:103B10002046D847504B84F83D80024683463946BC
:103B200050469847012F22D147F6FF739B4501D09D
:103B300099451CD1DFF848A12046D04700EBD07052
:103B400040F34F052046D04747F6FF7300EBD07097
:103B50009B4540F34F002AD185421EDA05F1010B47
:103B600099450FFA8BFB02D101350FFA85F93B4BD2
:103B70003B4898472C4B054698478246E0B9394B5D
:103B80002B49009340F6B26203202A4CA0473648E6
:103B90002A492A4653468847FEE700F1010B99451A
:103BA0000FFA8BFBE3D101300FFA80F9DFE799457B
:103BB000DDD18542F7DAD7E7002D2DD0A5F808B082
:103BC000A5F80C90294B2C60AF80AE710EA89847D9
:103BD000274B0F93274B1093274B11930022FF2362
:103BE000CDE91423099B1693089B069A0E955B4218
:103BF0001793069BD11D013B12AA13F8010F02F87F
:103C0000010B9942F9D19DF86E306FF300038DF8E6
:103C10006E300EA8194B9847049B0133062B049372
:103C20007FF43DAFF9E600BFE117000066F6010042
:103C30005BEE0100E9E80000BFEE0100E9170000BB
:103C40008D240000912D000011370000C9380000BC
:103C5000E15D0000B95C00007958000019E6000041
:103C60006086002077F60100BEED010079DC0000DF
:103C70008D2F00005D390000A125000021DD00002E
:103C8000ED2300000B2B4BD86B79DFF800B243F02B
:103C900004036B71029B84F83D303A46314620465E
:103CA000D8473A46814684F83D8031462046D84779
:103CB0006A79ADF81C006FF382026A711FFA89F904
:103CC00082B29145A8D0029B84F83D303A463146F5
:103CD0002046D84739460246604B84F83D808146ED
:103CE000504698475E4B5F4898475F4B054698475C
:103CF000824668B95D4B5E49009340F6C662032078
:103D00005C4CA0475C485D492A4653468847FEE71D
:103D1000002D81D0BDF81C30A5F80890AB8151E78B
:103D20000D2B49D86B79DFF868B143F004036B7150
:103D3000029B84F83D303A4631462046D8473A4601
:103D4000079084F83D8031462046D8476A79079B22
:103D50006FF38202834281466A713FF45DAF029B3A
:103D600084F83D303A4631462046D8473946024627
:103D7000434B84F83D80834650469847384B39483A
:103D80009847394B05469847824668B9374B3849BA
:103D9000009340F6DB620320364CA0473648374993
:103DA0002A4653468847FEE7002D3FF435AF85F895
:103DB00008B085F80C9005E7029B84F83D306B79DC
:103DC000DFF8D0B043F004036B713A463146204629
:103DD000D8473A460A90314684F83D802046D84775
:103DE0000E906B796FF3820381466B710422254B31
:103DF0000EA90AA8984700283FF40EAF029B84F84A
:103E00003D303A4631462046D847394602461E4B99
:103E10000A90834684F83D8050469847104B1148DD
:103E20009847114B05469847824668B90F4B104991
:103E3000009340F6EF6203200E4CA0470E480F4956
:103E40002A4653468847FEE7002D3FF4E5AEC5E914
:103E500002B9B7E61FB0BDE8F08F00BF49590000B6
:103E600019E6000060860020E117000077F60100E7
:103E70005BEE0100E9E80000BEED0100E91700007B
:103E8000195A000095620100ED5A0000B537000094
:103E900039380000C938000073B5114B04460D468F
:103EA0009847064668B90F4B0F49009340F27E626F
:103EB00003200E4DA8470E480E4922463346884738
:103EC000FEE794F83D3043EA05019D4305D00A4BD7
:103ED000204602B0BDE87040184702B070BD00BF78
:103EE000E117000084F601005BEE0100E9E8000044
:103EF000BFEE0100E9170000BD39000073B5114B9A
:103F000004460D469847064668B90F4B0F49009383
:103F100040F28F6203200E4DA8470E480E492246FC
:103F200033468847FEE794F83D301D4223EA0501F9
:103F300005D00A4B204602B0BDE87040184702B0D9
:103F400070BD00BFE117000095F601005BEE0100B7
:103F5000E9E80000BFEE0100E9170000BD390000EC
:103F600073B50B4B04469847054668B9094B0A4997
:103F7000009340F6F5220320084EB047084809494F
:103F800022462B468847FEE7E06902B070BD00BFBD
:103F9000E1170000A8F601005BEE0100E9E800006F
:103FA000BFEE0100E917000073B50B4B04469847BC
:103FB000054668B9094B0A49009340F61E320320B2
:103FC000084EB0470848094922462B468847FEE775
:103FD000606A02B070BD00BFE1170000E6F60100A4
:103FE0005BEE0100E9E80000BFEE0100E917000008
:103FF00073B50B4B04469847054668B9094B0A4907
:10400000009340F66F320320084EB0470848094934
:1040100022462B468847FEE7A06B02B070BD00BF6A
:10402000E11700000AF701005BEE0100E9E800007B
:10403000BFEE0100E91700002DE9F047394B0446B7
:10404000002215219847384B20469847074610B163
:10405000364B20469847364B364DDFF8F49000211A
:1040600020469847FF2200231146204604F1040809
:10407000A847314B4046984705463DBB2F4B5E68ED
:10408000012366BBDFF8CC80DFF8CC90DFF8CCA052
:104090003046C047054645BB2A462946E369284DB8
:1040A00020469847274B20469847002837D1264B73
:1040B0002046984721463030A847606A234D00B11A
:1040C000A84720462B46BDE8F047184729464046FA
:1040D000C84706462846FFF7AFFF3546CDE73268AA
:1040E000944208BF3371B668CBE76B6BA34202D032
:1040F000AB6BA34202D121462846C847EB6BA342D3
:10410000AB6D08BFEE63BB4205D1D047844202D1FC
:1041100021462846C8472846C0470546BBE72146F2
:104120000430C9E7791F0000F13F0000751B000053
:10413000B1DC0000B5240000A9E60000F4800020F6
:104140006DE7000025210000C5210000E5EA000020
:10415000B5E6000019DA0000791C0000B51C00006B
:10416000F7B51B4B04469847054668B9194B1A49E1
:10417000009340F293120320184EB0471848194993
:1041800022462B468847FEE7174B20469847174B99
:10419000204698470646B8B9154B2046984705462D
:1041A00078B1C76B3B1B5F425F41124B204698477B
:1041B00026B1F36900220121304698470FB1002350
:1041C000EB63002003B0F0BD00273D46EDE700BFE4
:1041D000E11700001BF701005BEE0100E9E80000B9
:1041E000BFEE0100E917000085270000252100002F
:1041F000C52100003940000073B50E4B04469847B6
:10420000054668B90C4B0D4900934FF43862032002
:104210000B4EB0470B480C4922462B468847FEE719
:10422000A06B20B1094B9847231A5842584102B05D
:1042300070BD00BFE117000047F701005BEE010011
:10424000E9E80000BFEE0100E9170000111C0000C2
:1042500007B5028A90F83030D21AADF80020828A71
:104260001344ADF80430428A90F83130D21AADF8D8
:104270000220C28A1344ADF806300022024B684681
:10428000984703B05DF804FB25DF000010B500235C
:1042900050F82340DAB21CB10133072BF8D11A468B
:1042A00040F82210012010BD2DE9F0471446B64F0A
:1042B000DFF8E082012205460E46B84748F20C02BC
:1042C000208031462846C047052881460AD8002369
:1042D0002373237584F8283084F8363084F844300A
:1042E000BDE8F087237B43B32C2231462846C047E4
:1042F0000528207321D929223146DFF890A22846CB
:10430000D0472322608031462846B847C0B2A0710A
:1043100070B12A2231462846D0472122A08031465A
:104320002846B8472222208131462846B847608176
:10433000202231462846B8476073237DEBB13022F6
:1043400031462846B8472082B8B13C22314628463B
:10435000C047052820750BD9312231462846B84779
:10436000C0B26082894B3922314628469847E081A5
:10437000322231462846B8476075237FE3B1402298
:1043800031462846B8472083B0B14C2231462846F2
:10439000C047052820770AD9412231462846B84728
:1043A0007A4B60834922314628469847E082422270
:1043B00031462846B847607794F83630002B3BD01A
:1043C000DFF8D4A16E2231462846D047E0620028AB
:1043D00032D06C2231462846C047052884F8360082
:1043E0002AD96D2231462846C047612284F8370019
:1043F00031462846B84794F83830003818BF0120B5
:1044000060F3000384F83830E06A614B9847022873
:1044100040F0AD805D4B692231462846984748F20E
:104420008E02A08631462846D0472063602231465E
:104430002846B84784F8390094F82830052B28D945
:10444000502231462846B847208410B35C223146BA
:104450002846C047052884F828001AD95122314639
:104460002846B8475222608431462846B84753222E
:10447000A08431462846B847444BE084592231464F
:10448000284698475422E08331462846B84784F8A6
:10449000290094F84430052B40D9DFF8FCA07F2296
:1044A00031462846D047E063002837D07C22314689
:1044B0002846C047052884F844002FD97322314686
:1044C0002846B8477422A4F8480031462846B84721
:1044D0002E4BA4F84A0079223146284698477E227E
:1044E000A4F8460031462846D04770222064314661
:1044F0002846B8477122A4F84C0031462846B847F0
:104500007522A4F84E0031462846B847722284F836
:10451000500031462846B84784F85100B9F1F90FE8
:104520003FF6DEAE237B1FFA89F013FB00F3C3F3E3
:1045300007232373237D13FB00F3C3F307232375A2
:1045400094F8283013FB00F3C3F3072384F82830D2
:1045500094F8363013FB00F3C3F3072384F83630A6
:1045600094F8443013FB00F3C3F30723B6E694F842
:104570003730052B7FF65AAF044B69223146284667
:104580009847A08652E700BF11370000B5370000FA
:104590000578000039380000C93800002DE9F04FD7
:1045A000022A99B004460F46154659D1DFF83092D9
:1045B0000021C8470646002850D101460122204666
:1045C000C8470422824631462046C8470522834612
:1045D00031462046C847774B804604F1100103A8B6
:1045E0009847BDF80C30BDF80E201FFA8BF01B1A4F
:1045F000ADF80C30BDF8103018441FFA88F3D21A09
:10460000ADF80E20BDF81220ADF810001344ADF83F
:1046100012305246684B03A938469847D0B1674FCD
:104620002C2231462046B847F92813D9314620229A
:104630002046C84710F0FF010CD132222046C8475F
:1046400010F0FF0106D148F20C022046B847F928C5
:1046500088BF0125284619B0BDE8F08F0325F9E78A
:10466000002A56D103A8564BDFF8748198473322AD
:1046700029462046C04708B18DF82050514B03AA67
:10468000002120469847042200212046C0470522E9
:10469000064600212046C04704F11009454B8246DA
:1046A000494601A89847BDF80420B3B2D21AADF824
:1046B0000420BDF808201344ADF80830BDF80630DA
:1046C0001FFA8AF01B1AADF80630BDF80A301844FC
:1046D000ADF80A0003AA394601A83B4B98470222CD
:1046E00000212046C0470028B4D0384B384F1C204A
:1046F00098470122064600212046C0474946024607
:1047000000233046B847334B04F5187130469847BC
:10471000A0E7012A01D000259CE7DFF8C48002222F
:104720000021C04728B12C4B04F5187098472B4B3B
:104730009847332200212046C0470028EBD00025AF
:1047400003A81F4B98471F4B8DF8185003AA294602
:1047500020468DF842508DF834509847294604225F
:104760002046C0470522064629462046C04704F198
:10477000100180460F4B01A89847BDF80420B3B242
:10478000D21AADF80420BDF808201344ADF8083063
:10479000BDF806301FFA88F01B1AADF80630BDF8D8
:1047A0000A301844ADF80A00074B03AA394601A89D
:1047B00098474FE7191D000091E0000039380000CC
:1047C000A19B0000A9420000ED9B0000B5EE000097
:1047D0001599000011970000C997000069EB0000CF
:1047E000113700002DE9F0411446284F48F28C02A1
:1047F00005460E46B8470528207245D948F20C02F6
:1048000031462846B847F9289FBF237A13FB00F0AA
:10481000C0F307202072237A052B35D948F289028C
:104820003146DFF874801A4F2846C04748F28002AC
:10483000208031462846B84748F28102A08131469F
:104840002846B84748F28202608131462846B84778
:1048500048F28302207631462846B8470D4B6076F1
:1048600048F28E02314628469847E28960604FF64A
:10487000FF739A4208D0228A9A4205D048F28A02EF
:1048800031462846C0472080BDE8F0813938000015
:1048900011370000C9380000B5370000F8B51446DC
:1048A000234F48F2AC0205460E46B8470528207053
:1048B0003CD948F20C0231462846B847F9289FBF38
:1048C000237813FB00F0C0F3072020702378052B1A
:1048D0002CD9002363804FF480732381AB8A2A8A0A
:1048E00001339B1AC3F3C03202FA83F35B10A38037
:1048F000EB8A6A8A01339B1AC3F3C03202FA83F34C
:104900005B10E38048F2AD0231462846B847094BB8
:10491000A07248F2A902314628469847064BA0816A
:1049200048F2A002314628469847A073F8BD00BF60
:1049300039380000B5370000113700002DE9F04785
:104940005022754F8AB004460E46B84705460028E7
:1049500040F0B4800025DFF8C8A17F223146204610
:10496000D047804600287ED06C4B7C2231462046C2
:104970009847052877D9702231462046B8477022DB
:10498000059031462046B8477E2281463146204672
:10499000D0474FF0000A47F61841CDE9011A024608
:1049A0004146059BDFF87C81CDF8009006A8C04702
:1049B000BDF81830CDF820A0013BADF82430BDF88B
:1049C0001A307522013B31462046ADF82630B847F3
:1049D0007322824631462046B847742281463146CA
:1049E0002046B8475FFA8AF2804607AB08A904F16F
:1049F0001000DFF834A1D047BDF81E20BDF81C30F0
:104A0000B4F9101008EB0200BDF820204B4412FA54
:104A100083F212B2891AA942B8BF2946BDF82250C2
:104A2000B4F9122015FA80F52DB2521B09B28A4250
:104A3000B8BF0A46BDF8241011FA83F3B4F9141074
:104A40001BB25B1A12B29342B8BF1346BDF82620C0
:104A500012FA80F0B4F9162000B2801A1BB2984204
:104A6000B8BF184605B2402231462046B8478046B6
:104A700078B12A4B4C22314620469847052808D960
:104A8000412231462046B8474044A842B8BF284694
:104A900005B2314604222046B847052280463146F9
:104AA0002046B8474045B8BF404600B20028C4BFC2
:104AB000401905B228460AB0BDE8F087174B5C22C2
:104AC00031462046984705287FF644AF53223146A9
:104AD0002046B84705EBD57500EB650551223146F8
:104AE0002046B8475222804631462046B847002823
:104AF000B8BF4042B8F1000FB8BFC8F10008013597
:104B0000ADB280B21FFA88F840452CBF2D1845443D
:104B10002DB225EAE5751EE711370000393800008F
:104B2000C93800009D01010031E1000070B5054663
:104B30001046172911D8DFE801F0551A102E37104A
:104B400023150C10103B10404010101010101010C6
:104B5000445313781BB92835556001240EE0002317
:104B60005360FAE7BDE870402049214B1847214BBC
:104B700001212846984780F00100C4B2204670BD4C
:104B80001D4B002128469847B5F932309842B8BFEE
:104B900018466886E1E795F8494014F00104DCD036
:104BA000164B28469847E9E7154B28469847D4E71F
:104BB000144B102128469847CFE71021124B284666
:104BC000F9E7124B28469847114B98470D4B10B107
:104BD00006212846EFE70221284698470421EDE701
:104BE0000621EBE70B4B00212846E4E75BF00100D0
:104BF0008D420000513600003D490000E92C0000C4
:104C0000D1200000993E0000FD3E0000F13F000071
:104C10001B1C00004925000038B5174D174B2868AC
:104C20009847174B04462868984758B928680123C5
:104C30004268A361116AC90709D400230AE0C36965
:104C40000BB198472868A369002BF8D1EEE7126AE8
:104C50009207F2D5E361C3681BB1A26804F11001A9
:104C60009847226832B1636823B1A1688A4218BFAD
:104C70001346A36038BD00BF00810020E1D90000C9
:104C8000E5D900002DE9F84300220C46174B1031FE
:104C90000746984710B90020BDE8F88394F83430EF
:104CA000DB06F8D4236A9BB1022239462046984796
:104CB00003280646EFD004F104080D4BDFF83490CA
:104CC0004046984705462DB9012EE4D12046E3E73A
:104CD0000226F0E729463846FFF7D4FF0028DBD14B
:104CE00029464046C8470546EDE700BF91E0000071
:104CF000A9E60000B5E600002DE9F04390F8348005
:104D000018F010088BB004460F463CD1B0F9325071
:104D1000314EDFF8CC9004A9B047BDF81020ABB2FB
:104D2000D21AADF81020BDF81220D21AADF8122018
:104D3000BDF814201A44ADF81420BDF816203946E9
:104D4000134402A804AAADF81630C847D8B1236AA4
:104D50001BB1424602A92046984704A92046B04705
:104D600004AA39466846C84738B1271D1B4BDFF8EF
:104D7000748038469847054645B9236A1BB101221D
:104D800002A9204698470BB0BDE8F08308A9284641
:104D9000B0476B8EBDF82020D21AADF82020BDF8A8
:104DA0002220D21AADF82220BDF824201A44ADF8F2
:104DB0002420BDF826206946134406A808AAADF8A9
:104DC0002630C84718B106A92846FFF795FF29469F
:104DD0003846C0470546CFE7D5220000AFE60000C1
:104DE0008DDE0000D5E600002DE9F0470E460446B2
:104DF00028B9154B1868154B9847044658B13146E9
:104E00002046134FDFF84C80DFF84C90B84720461F
:104E1000C04705460DB9BDE8F08705F1040A2146F3
:104E20005046C847044650B92B6A1BB1012231468F
:104E3000284698472846C0472C460546EAE73146AB
:104E40002046B847EBE700BF008100207118000042
:104E5000F94C000025210000D5E6000073B51A4C7E
:104E60001A4B064620689847194B05462068984714
:104E700020B305F110023146164B174D684698478E
:104E8000164B20689847164B014668469847694676
:104E9000A847144B206898476946A847124B2068DA
:104EA00098476946A8472068104B984708B9104BA7
:104EB000984702B070BDC3690BB198472068AB69D1
:104EC000002BF8D1D5E700BF00810020E1D9000018
:104ED000E5D900008DDE0000E94D000071180000EA
:104EE000854C0000AD180000E9180000F5D900005D
:104EF000194C0000013900F1080311F8012F00F8E6
:104F0000012B9842F9D17047704700002DE9FF410D
:104F10000D46044618B92D4B9847044630B145B9A3
:104F2000B4F8683165F30903A4F8683104B0BDE84A
:104F3000F081002300932046254B98470138254BEC
:104F4000ADF80400204698470138ADF80600224B22
:104F50006A46294602A898470028E7D0236913B17A
:104F600002A92046984704F14805DFF8788000261A
:104F70002F46B4F86831B2B2C3F3090090421CD88E
:104F80001F289BBF0930C0F309006FF3090302A972
:104F900091BF04EBC000A4F86831694638460F4A57
:104FA0009047B4F86831E06A5A1C62F30903A4F828
:104FB000683103210A4B9847B8E72946002202A826
:104FC000C047013608350028D3D0AFE7FDD8000030
:104FD00009D900002DD900008DDE0000F54E00003B
:104FE0006DFB000091E00000014B1868704700BFA6
:104FF000008100202DE9F04F2DED028B824B834C78
:105000008BB005469847EB6823600021804B08EE83
:10501000900A284698472368D96B002940F08B8076
:10502000B3F8682161F30902A3F868210BB0BDEC65
:10503000028BBDE8F08F334493F84851002D3CD0EB
:1050400001362368B3F86821C2F309018E42F2D316
:1050500000206060002971D16C4F3868B0F8683169
:10506000C3F3090303B36B4B9847002840F0A181B9
:105070002068694D4FF480714830A847206820218E
:1050800000F5A470A8472368B3F868216FF30902FC
:10509000A3F8682118EE900A604B984701462068F3
:1050A0008369002B40F0DD815D4B98475D4B0BB071
:1050B000BDEC028BBDE8F04F18474FEAC609DFF898
:1050C00084A109F148092068B0F86831C3F30903E5
:1050D0009D42B5D2431993F8483153BBAE4228D014
:1050E0004FEAC50B0BF1480B00EB0B014844B847E6
:1050F000F8B121684C4B01EB0B0208A849449847D2
:1051000008A8D047804620684844D04703902068CC
:105110005844D047039B184480450AD2D4F800B0C5
:10512000424B0BEB090008A9AB44984701238BF8CD
:1051300048310135C7E73E4F002682E74F1E03F591
:10514000A472791C5BD100275B68DFF8C08093F8FC
:1051500020206FF3000283F8202093F820206FF3C3
:10516000410283F820204FF0000BD8F80050B5F82A
:105170006831C3F309039B45BFF66EAF05EB0B0324
:1051800093F84831002B40F0C6806B68BB4502BFE6
:1051900093F8202042F0010283F8202093F8202089
:1051A0004FEACB096FF3410283F8202009F148034D
:1051B0000493EB1808EE103A2846164B98471D4BFF
:1051C000002841D020689847002605461A4B0682E1
:1051D000206898470138194BA8826E82206898474A
:1051E000236801385A68E88292F8203043F00203BD
:1051F00082F8203018EE100A114B98477EE0D15DFE
:105200000029A1D0013F9CE749DA0000008100207D
:105210006DFB0000F5D9000019F000005DDA000018
:10522000DDEB000041D70000E1DE0000F54E00009C
:1052300055E00000E1D9000009D900002DD9000097
:105240005D4E000071DE00004D4420689847B5F8BF
:105250004C90B5F84830B5F94E20039209F1010998
:10526000A9EB0309B5F84A3002F1010AAAEB030AD7
:1052700006467D4B20689847039A7B4B82420FFA83
:1052800089F90FFA8AFA49DB20689847013803B296
:10529000F268B2FBF9F25245A8BF52460392D8F821
:1052A00000201269002A40D00022BDF90C9008921B
:1052B000ADF82420D8F800000593CA4609F1FF395B
:1052C0000FFA89F90269ADF8269008A99047BDF94F
:1052D0002610BDF82220039B01318A1A12B2934294
:1052E000059B1EDAB9F1000FE4DC604B00936049C6
:1052F000604B614D4FF4CF720220A847D8F80000F0
:10530000836943B1049B18445C4B9847D8F8043038
:105310001844C8F804000BF1010B26E7B5F94E302C
:10532000B6E7BAF1000FE0DD0391BDF80C10B5F956
:105330004A20481E4FF000090590039810180138C4
:1053400098420CDD4B45D9D0B5F948002168308230
:10535000B5F94C00B0827282F3824A6844E7B5F92D
:1053600048003082B5F94C00B082059872821FFA6D
:1053700082FA10FA82F212B293429946A8BF91467D
:105380009342A6F8169008DCD8F80020506890F8F0
:10539000202042F0020280F82020394A18EE100A3C
:1053A000CDE9063190470799069B8A440FFA8AF2A5
:1053B000C3E738684369002B7FF45AAE314B9847F6
:1053C000314B05469847AB69002BFCD1D5F80090CE
:1053D000D5F808B02D4B3868D94508BFD5F80490EA
:1053E00098470025804643003A68B2F86811A8B291
:1053F000C1F3090181427FF63BAE511991F8481182
:1054000009B10135F0E702EBC502B2F94800B2F983
:105410004A60B2F84C20013208FB0601121A05F16D
:10542000090012B2C0000BEB410A4FEA420C09EB33
:10543000410103903868039A1044B0F90600B04265
:10544000DFDB06936246124B5046CDE9041C9847B9
:10545000069B0499DDF814C0013636B29A4419440B
:10546000E8E7626898471FE62DD9000089F7010038
:1054700059F70100D9F70100E9E8000071DE0000EA
:105480005D4E0000E1D90000194C000009D9000070
:1054900031EC0000437903F00603062B08BF01310D
:1054A000037908BFC9B28B4286BF036853F8210055
:1054B00000207047F0B578B34FF0FF35CFB24FEA18
:1054C000112C00232E46C1F30621C25CFF2A01D114
:1054D000284609E0974211D1C41864788CEA040E7A
:1054E0001EF07F0F01D11846F0BD04F07F0434EAAE
:1054F000010E03D1B442C4BF26B21DB202F00F02A6
:10550000082A02D802330233DFE70B2AFAD90D2A20
:1055100094BF01330433F6E74FF0FF30E4E701397D
:10552000024411F8013F00F8013B9042F9D1704765
:10553000014B0421184700BF19F00000014B08215E
:10554000184700BF19F00000F7B5037904460E466E
:105550004BB10068002250F82210B1423CD0013219
:10556000D1B28B42F7D803B0F0BD013B9900214B7B
:105570009847214B05469847074668B91F4B204975
:1055800000934FF4827203201E4CA0471E481F490F
:105590002A463B468847FEE74DB1002321791A464B
:1055A000D8B288420DD3013921712560DBE7184B51
:1055B00000931349114B134C4FF483720220A04700
:1055C000D1E7206850F82300B0421EBF45F8220002
:1055D0000132D2B20133E3E7012BC6D10D4B98471C
:1055E00000232360A38823F4FF7323F00103A38027
:1055F000B9E700BF15EE0000E1170000EFF8010069
:10560000E6F70100E9E80000BEED0100E91700003F
:1056100017F80100E5EA00002DE9F3410F460546C1
:1056200038B3294B98472979A1B9284B04209847CA
:10563000274B04469847064690B9264B26490093C7
:10564000D0220320254DA847254826492246334627
:105650008847FEE701312868234B89009847E7E730
:1056600054B9224B00931C491A4B1C4CD2220220E5
:10567000A04702B0BDE8F0816B792E79C3F34008F2
:10568000DB0748BF08F10108A6EB0802D2B2464585
:10569000C2F1010006F180414FEA800001F1FF31C3
:1056A00038BF042000EB810100EB86004FEA820244
:1056B0000F4B38BF0022214420440136984744F85C
:1056C00028702E712C60D4E7495500002DEA0000A7
:1056D000E11700000BF90100E6F70100E9E800001E
:1056E000BEED0100E917000015EE000052F80100C0
:1056F000D16201004379DB0773B5054605D51A4B26
:10570000002102B0BDE870401847184B04209847AC
:10571000174B04469847064668B9164B164900933E
:1057200040F235420320154DA84715481549224639
:1057300033468847FEE75CB9134B00930E490D4B87
:105740000E4D40F237420220A847204602B070BDFD
:105750000E4B204698470E4B2146284698476B79BA
:1057600043F001036B71F0E7955400002DEA00004F
:10577000E117000024F90100E6F70100E9E8000064
:10578000BEED0100E917000082F80100315500006C
:105790001956000010B5034B0446006898470023D3
:1057A000236010BDE5EA0000006828B10023C25C58
:1057B000FF2A02D1023398B2704702F00F02082A82
:1057C00002D802330233F2E70B2AFAD90D2A94BF2A
:1057D00001330433F6E7000037B505460C4679B1CE
:1057E0000B686BB10846074B9847074B01909847E9
:1057F0002860019A2168054B03B0BDE83040184786
:1058000003B030BDA95700002DEA000031EC0000C4
:10581000F8B50F46044630B30668144B3046984737
:10582000051E20DB2E44737883EA17235B061AD10A
:105830000F4B204607F00F0198470B290CD90E2972
:1058400034BF03230623C11AA942206806D8094B96
:10585000984720600120F8BD0423F4E74219D25C88
:1058600042550135F0E70020F5E700BFB5540000D0
:10587000A957000015EE000070B50668284B86B0E9
:1058800005463046ADF80E10ADF80C200C46984792
:1058900000280DDB33185B7883EA14235B0607D1FD
:1058A0000230204B022203A93044984706B070BD55
:1058B000FF23ADF8163028461B4B9847041E08BF3F
:1058C00002240434A4B2194B214630469847184BA1
:1058D00028609847064668B9164B174900934FF45D
:1058E000C3720320154CA0472A6815481549334652
:1058F0008847FEE728680B4EA31F0DF10E011844E0
:105900000222B0472868231F03A918440222B04787
:105910002868023C02220DF116012044B047C5E779
:10592000B55400001F550000A957000015EE0000F7
:10593000E11700003AF90100E6F70100E9E800008C
:10594000BEED0100E917000070B50668284B86B06F
:1059500005463046ADF80C20ADF80E100C469847C1
:1059600000280DDB33185B7883EA14235B0607D12C
:105970000230204B022203A93044984706B070BD84
:10598000FF23ADF8163028461B4B9847041E08BF6E
:1059900002240434A4B2194B214630469847184BD0
:1059A00028609847064668B9164B1749009340F29D
:1059B000B5120320154CA0472A68154815493346EF
:1059C0008847FEE728680B4EA31F0DF10E0118440F
:1059D0000222B0472868231F03A918440222B047B7
:1059E0002868023C02220DF116012044B047C5E7A9
:1059F000B55400001F550000A957000015EE000027
:105A0000E11700004CF90100E6F70100E9E80000A9
:105A1000BEED0100E917000070B50668294B86B09D
:105A200005463046ADF80E108DF80D200C4698470F
:105A300000280EDB33185B7883EA14235B0608D159
:105A40000230214B01220DF10D013044984706B080
:105A500070BDFF23ADF8163028461C4B9847041E36
:105A600008BF02240334A4B2194B2146304698479C
:105A7000184B28609847064668B9174B174900939A
:105A80004FF4F2720320164CA0472A6815481649B5
:105A900033468847FEE728680B4E631F0DF10E0161
:105AA00018440222B0472868E31E0DF10D01184486
:105AB0000122B0472868023C02220DF11601204461
:105AC000B047C4E7B55400001F550000A9570000B7
:105AD00015EE0000E117000060F90100E6F7010093
:105AE000E9E80000BEED0100E917000070B50668A6
:105AF000284B86B0054630460292ADF80E100C4693
:105B0000984700280DDB33185B7883EA14235B0683
:105B100007D10230204B042202A93044984706B036
:105B200070BDFF23ADF8163028461C4B9847041E65
:105B300008BF02240634A4B2194B214630469847C8
:105B4000184B28609847064668B9174B17490093C9
:105B500040F213220320164CA0472A681548164924
:105B600033468847FEE728680B4EA4F108030DF181
:105B70000E0118440222B0472868A31F02A9184446
:105B80000422B0472868023C02220DF1160120448D
:105B9000B047C4E7B55400001F550000A9570000E6
:105BA00015EE0000E117000072F90100E6F70100B0
:105BB000E9E80000BEED0100E91700002DE9F04121
:105BC0000E4617460546C0B1D0F80080B8F1000F68
:105BD00013D00B4B40469847041E0EDBA11C094B0B
:105BE00038460222414498472B6823445878C0F332
:105BF000060000EA1620BDE8F0814FF0FF30FAE71A
:105C0000B55400001F5500002DE9F0410E4617461F
:105C10000546C0B1D0F80080B8F1000F13D00B4B8F
:105C200040469847041E0EDBA11C094B3846012252
:105C3000414498472B6823445878C0F3060000EA93
:105C40001620BDE8F0814FF0FF30FAE7B5540000B0
:105C50001F5500002DE9F0410E4617460546C0B11C
:105C6000D0F80080B8F1000F13D00B4B4046984796
:105C7000041E0EDBA11C094B384604224144984700
:105C80002B6823445878C0F3060000EA1620BDE8CC
:105C9000F0814FF0FF30FAE7B55400001F550000C7
:105CA000427912F0010305D0036892074CBF58688F
:105CB0001868704718467047437913F002031ABFFB
:105CC000036818681846704738B5044628B3437906
:105CD000DA0708D5114B9847054620B1104B984775
:105CE000104B2846984763799B0709D50E4B2046F1
:105CF0009847054620B10A4B98470A4B28469847D3
:105D0000237913B12068074B984700232360A388A9
:105D100023F4FF6323F00703A38038BDA15C0000D8
:105D200095570000E5EA0000B95C000070B50C462C
:105D3000264B054698472368B3B163792079244EF2
:105D400013F0010F03F00202224B17D16AB10138A0
:105D500080009847286022792168013A9200043136
:105D6000B0472379013B2B7170BD800098472860B4
:105D7000227921689200B0472379F4E7CAB102384A
:105D800080009847286022792168023A9200083101
:105D9000B0472379023BDBB22B710F4E2846B04748
:105DA00005462046B0470D4B01462846BDE87040E9
:105DB0001847013880009847286022792168013A05
:105DC00092000431B0472379013BE4E7C95C00004D
:105DD00031EC00002DEA0000F5560000D957000014
:105DE00043799A0773B5054604D51D4B02B0BDE84B
:105DF000704018471B4B042098471B4B044698479C
:105E0000064668B9194B1A49009340F2CD22032087
:105E1000184DA84718481949224633468847FEE7D7
:105E20005CB9174B00931249104B124D40F2CF2230
:105E30000220A847204602B070BD124B204698476A
:105E40002146114B284698476B7943F002036B714A
:105E5000DB0742BF2B68D3E90021C3E90012E9E761
:105E6000B95C00002DEA0000E117000084F9010090
:105E7000E6F70100E9E80000BEED0100E9170000C7
:105E8000AFF8010031550000195600002DE9F74F19
:105E90000F469046054618B3006808B300261B4B12
:105EA000DFF86CB0ADF806604FEA112A4FF0FF340E
:105EB0002A790FFA86F9914503DBE043C0F3C0303D
:105EC0000EE0F1B2284698470DF106023946D84750
:105ED00082450E4B07D1BDF80630A8F800300120EE
:105EE00003B0BDE8F08F6A79910706D5002804DB7E
:105EF000B9F1000F01D15207EDD58442BEBFBDF804
:105F00000620A8F8002004460136D1E79554000089
:105F1000BD5B00002DE9F74F0F469046054610B3D4
:105F2000006800B300261B4BDFF86CB0ADF80460CE
:105F30004FEA112A4FF0FF342A790FFA86F991457A
:105F400003DBE043C0F3C0300DE0F1B228469847D0
:105F500001AA3946D84782450E4B07D1BDF8043017
:105F6000A8F80030012003B0BDE8F08F6A799107EE
:105F700006D5002804DBB9F1000F01D15207EDD599
:105F80008442BEBFBDF80420A8F8002004460136B4
:105F9000D2E700BF95540000BD5B00002DE9F74F2C
:105FA0000F469046054618B3006808B300261B4B01
:105FB000DFF86CB08DF807604FEA112A4FF0FF341C
:105FC0002A790FFA86F9914503DBE043C0F3C0302C
:105FD0000EE0F1B2284698470DF107023946D8473E
:105FE00082450E4B07D19DF8073088F8003001201C
:105FF00003B0BDE8F08F6A79910706D5002804DB6D
:10600000B9F1000F01D15207EDD58442BEBF9DF812
:10601000072088F8002004460136D1E79554000097
:10602000095C00002DE9F74F0F4690460546F8B190
:106030000068E8B1194BDFF868B04FEA112A002672
:106040004FF0FF342A790FFA86F9914503DBE043DC
:10605000C0F3C0300CE0F1B22846984701AA394697
:10606000D84782450D4B06D1019BC8F8003001206E
:1060700003B0BDE8F08F6A79910706D5002804DBEC
:10608000B9F1000F01D15207EED58442BEBF019A8B
:10609000C8F8002004460136D4E700BF955400003C
:1060A000555C0000F0B5C1F34513C2F1FF06C0F323
:1060B0004514734304FB023301F01F0400F01F0773
:1060C000744348F2810507FB02446B436C43C3F3FE
:1060D000C553C4F3C45444EA4314C1F3C423734303
:1060E000C0F3C42000FB023205FB02F3DB0D44EADF
:1060F000C320F0BD0B46052A2DE9F04100F01F0C2E
:10610000C0F3451EC0F3C42803F01F06C3F34515B2
:10611000C3F3C42402D80846BDE8F08104EB0803A9
:106120001F2B05EB0E0428BF1F2306EB0C053F2C8D
:1061300028BF3F241F2D28BF1F25FF2A03F01F0360
:1061400004F03F0405F01F0508D14FF0000065F38F
:10615000040064F34A1063F3CF20DDE765F3040025
:1061600064F34A1063F3CF20BDE8F041004B1847B9
:10617000A56000000B46052A2DE9F04100F01F0C38
:10618000C0F3451EC0F3C42803F01F06C3F3451532
:10619000C3F3C42402D80846BDE8F081A4EB080389
:1061A000A5EB0E04A6EB0C0523EAE37324EAE474E2
:1061B00025EAE575FF2A03F01F0304F03F0405F00C
:1061C0001F0508D14FF0000065F3040064F34A1086
:1061D00063F3CF20E0E765F3040064F34A1063F350
:1061E000CF20BDE8F041014B184700BFA56000007B
:1061F0002DE9F04F8DB0054605939DF85C309DF874
:1062000058709DF860B00493042B0E46144640F27B
:10621000A380002F00F0A080A44B9847A44B824697
:106220009847A44BD0F808908046324629460AA8E1
:106230009847002800F09080BDF82820B8F810009A
:10624000BDF82C30B8F81260BDF82A50111A181A8F
:10625000ADF82C00BDF82E00801BAD1BADF82E0054
:10626000059809B22DB2ADF82810ADF82A500028D3
:1062700045D1DAF81400A6B200285AD1BBF1000FBC
:1062800040F02782894B9847B8F81430B8F81020AE
:10629000BDF92A100133A3EB0208BDF82C30BDF97B
:1062A000282001339B1A1BB20693BDF92E300893A8
:1062B00001330FFA88F85B1A1BB208FB0122012F89
:1062C000079382460B4609EB420540F03281049B5E
:1062D000FA2B40F29E80436A002B00F09580764BAB
:1062E0000AA89847F02840F28F80DAF82450ADF8D9
:1062F00000400AAB424649465046A8472CE09AF86F
:106300000800C007B5D4581C801A059E0FFA80FEFD
:106310000598C6F1010C01380CEB0006B645A8DD66
:1063200010F8016F802E4FF0FF3698BF00260670E0
:10633000F2E75E4B9847B8F81420B8F81030BDF972
:106340002A500132D21A012F064612B221D1AA4692
:10635000BDF92E309A4502DD0DB0BDE8F08FBDF9D4
:1063600028700FFA8AF8BDF92C309F4202DD0AF13D
:10637000010AEDE7049B0293ADF80440CDF80080DC
:106380003BB27569059249463046A8470137059AE0
:10639000E9E7BDF82C70BDF9283005990137FF1ADF
:1063A000A1EB030A3BB20593BDF92E309D42D3DC2D
:1063B000BDF928800FFA85FBBDF92C30984503DD27
:1063C000059B01359A44EFE71AF808300499ADF8B7
:1063D000044013FB01F31B0A0293CDF800B00FFA3F
:1063E00088F37769069249463046B84708F10108B4
:1063F000069AE1E72846069A3146B84745440134F3
:10640000079BA342F6DCA7E72C4F4FEA480800247D
:10641000F6E7036A13B3284B0AA89847F0281DD95A
:10642000274B069A5A4514DCBDF92A60244F4FEADF
:106430004808BDF92E309E428EDC049B009329460D
:10644000DAF82040069B3A465046A04745440136BC
:10645000EFE723F8026B0BF1010BE2E7049A194B0B
:1064600020464FF000019847049EC4F3C4227243B3
:106470000592C4F3451204F01F0402FB06FB04FB63
:1064800006FA4FEA4802F64300F01F03C0F3451C2A
:106490000492C0F3C4204FF00008F6B2079A4245B8
:1064A0007FF75AAF2F464FF0000E3AE0E94F000059
:1064B000E1D900008DDE000071DE000009E300007C
:1064C00008810020A56000003A461FFA81F914886F
:1064D000A14507F1020715D05078059B37F8021C3B
:1064E000C00800FB06301378C4F3451403F01F0303
:1064F00004FB06B403FB06A3C0F30420C4F3052C7D
:10650000C3F30423147863F30404147014886CF345
:106510004A141480C4F3072460F3C70454700EF1C6
:10652000010E069A7245CFDC049A08F10108154461
:10653000B4E739F812104FEA48020992049AFA2A8D
:1065400040F2C480069BDFF89882043B0493079BCB
:106550005B457FF701AFDDF814A0A946002413E0E6
:10656000B9F800103046C047A9F8000009E01AF059
:10657000030F0DD01AF8012B1AB1FF2AF0D1A9F898
:106580000060013409F10209069BA3425746EEDC84
:1065900005EB4409049BA3420EDA013F05EB4409D5
:1065A000069BA3424CDC099B1D44DDE905321344E4
:1065B00005930BF1010BCAE73B684BB101330CD1DA
:1065C000A9F80060A9F80260A9F80460A9F80660BB
:1065D0000437043409F10809DCE73A781AB1FF2AD4
:1065E00019D1A9F800607A781AB1FF2A1AD1A9F84E
:1065F0000260BA781AB1FF2A1BD1A9F80460FA78B0
:10660000002AE5D0FF2AE1D0B9F806103046C0478D
:10661000A9F80600DCE7B9F800103046C047A9F831
:106620000000E0E7B9F802103046C047A9F80200C0
:10663000DFE7B9F804103046C047A9F80400DEE7E8
:1066400017F8012F1AB1FF2A05D1A9F8006001340B
:1066500009F10209A4E7B9F800103046C047A9F8CB
:106660000000F4E7059A12F80840D4B15C45B7F889
:10667000009012D0FF2C17BF049ADDF810A014FB75
:1066800002F24FEA122A07933988554B5246304698
:106690009847A346079B80B201E04945F3D1388073
:1066A000494608F101080237069A4245DADC099AA0
:1066B0001544DDE90524224405920133089A9342EA
:1066C0003FF74AAE2F464FF00008EDE70846DA469E
:1066D000F4E7BBF1010FB8F91000B8F914600CD061
:1066E000BBF1020F2DD03F4B00933F493F4B404C35
:1066F0004FF404720220A0472EE6DFF8F8B001360E
:10670000361A36B206FB05F0012F09EB400A4FEAB4
:10671000460627D14FF00008049A314B41462046E7
:106720009847BDF92E309D423FF716AEBDF928704F
:106730000AEB4709BDF92C309F4205DDB244013513
:10674000EFE7DFF8B4B0DAE7B9F800101FFA88F322
:106750008B4203D0049A20468846D84729F8020B7A
:106760000137E7E7C2F1010203EB0208059B5F1A5C
:1067700039F810100FFA88F808464FF0000CBDF9F0
:106780002E309D423FF7E8ADBDF928900AEB490352
:10679000BDF92C20914503DDB24447440135EEE7B5
:1067A00017F80920BAB1624503D1B3F800E08E456D
:1067B00010D0F92A94BF0499049A05939CBF12FB48
:1067C00001F2120A19882046D847059B17F809C01C
:1067D000198880B2188009F101090233D8E700BF97
:1067E000A5600000D9F90100A3F90100FEF901003C
:1067F000E9E80000F5600000756100002DE9F04F48
:106800008FB0894606939DF860300A939DF86430F6
:106810009DF868A00B92042B059340F2D7800A9B49
:10682000002B00F0D3800A46B64B01460CA89847CF
:10683000002800F0CB80B44B9847B44B05469847EE
:1068400083468368BDF832E00893BBF81230BDF888
:1068500036C0BDF83040008AAEEB03020FFA82F872
:10686000ACEB0303BDF83420ADF83630211A069B9B
:10687000ADF8328009B2101AADF83010ADF834001E
:10688000002B5ED16B69002B72D1C4F1010422444C
:10689000B9F80470BBF81460BBF91030BBF91200F2
:1068A00012B20792B9F90020B9F902900136013706
:1068B000F61ABF1AA9EB000936B23FB2A8EB0909D4
:1068C00006FB08F407FB09F9BAF1000F40F0EA8172
:1068D000CEF10100D51A84440B9B0FFA8CF04D1BAE
:1068E00009904D4408980C4403EB4505864B00EB9A
:1068F000440498477B0008930A9B012B80464FEA8B
:10690000460B40F0E080036A002B00F0AF80804B24
:106910000CA89847F02840F2A980BDF93270BDF963
:1069200036309F4252DC059B00932A46079BD8F8DD
:10693000206021464046B047089B5C441D44013717
:10694000EDE72B7AD8079DD40698069E531C1B1B97
:106950001BB20138C6F101073E18B34292DD10F8B0
:10696000016F802E4FF0FF3698BF00260670F3E7C8
:10697000654B9847B9F80450B9F90010BBF81420DA
:10698000BBF912C0B9F90270BBF91040BDF9326011
:10699000BDF93030BDF9348001356D1A0132A7EBF5
:1069A0000C07121B2DB2641AF71B0B9905FB074449
:1069B00001EB44040A99012912B2C3F1000A4FEA1B
:1069C000450B23D1BDF936309E4202DD0FB0BDE844
:1069D000F08FBDF9308037B2BDF93430984502DD13
:1069E0005C440136EEE7059B029334F81830ADF8AD
:1069F000043000974569089907920FFA88F30690CA
:106A000008F10108A847DDE90602E5E708F10108F9
:106A1000A8EB0308069B53440FFA88F89A46BDF981
:106A200036309E42D2DCBDF9309037B2BDF93430F9
:106A3000994503DDC2445C440136F0E71AF8093099
:106A40000599079213FB01F31B0A029334F81930DE
:106A5000ADF8043000974569089906900FFA89F35C
:106A6000A84709F10109DDE90602DFE7059BFA2BDA
:106A700025D9079BDFF89C805F000026099BB34265
:106A8000A4DD294620463A46C047089B5C441D4485
:106A90000136F3E734F8161035F81600059AC047AA
:106AA00024F816000136079BB342F3DC089B5C44D4
:106AB0001D440137099BBB4288DD0026F3E7DFF860
:106AC00058800027F6E7059BFA2B40F2E980079BE8
:106AD000DFF84480CDF814A0043B0A93099B059A83
:106AE00093427FF773AF069BAA46A146002625E096
:106AF000B9F80010BAF800000B93C0470B9BA9F837
:106B0000000016E08DDE0000E94F0000E1D9000032
:106B100071DE000031EC0000A56000009A0711D082
:106B200013F8012B2AB1FF2AE2D1BAF80020A9F804
:106B3000002001360AF1020A09F10209079AB2425D
:106B40001F46EBDC05EB460A04EB46090A9BB34201
:106B500012DC013F05EB460A04EB4609079BB342F2
:106B600062DCDDE9063213440693089B1D44059B55
:106B700001335C440593B1E73B688BB1013316D117
:106B8000BAF80030A9F80030BAF80230A9F802309B
:106B9000BAF80430A9F80430BAF80630A9F806307B
:106BA000043704360AF1080A09F10809CEE73A78F1
:106BB0002AB1FF2A20D1BAF80030A9F800307A783B
:106BC0002AB1FF2A20D1BAF80230A9F80230BA78E7
:106BD0002AB1FF2A20D1BAF80430A9F80430FA7893
:106BE000002ADDD0FF2AD7D0B9F80610BAF806007F
:106BF000C047A9F80600D3E7B9F80010BAF80000BA
:106C0000C047A9F80000DAE7B9F80210BAF80200A4
:106C1000C047A9F80200DAE7B9F80410BAF804008E
:106C2000C047A9F80400DAE717F8012F2AB1FF2AB4
:106C300009D1BAF80030A9F8003001360AF1020A89
:106C400009F102098AE7B9F80010BAF80000C04754
:106C5000A9F80000F1E7069B9A5D72B1F92A98BF86
:106C6000059B34F8161035F816008EBF059A13FBF5
:106C700002F2120AB84724F816000136079BB34205
:106C8000E9DCDDE9063213440693089B5C441D44AD
:106C90000AF1010A099B53457FF798AE0026EDE7FC
:106CA000364FF7E7BAF1010F0CD0BAF1020F2BD033
:106CB000334B00933349344B344C40F2533202206F
:106CC000A04783E6DFF8C8B0089800EB44040B98AF
:106CD00000EB49090A9801284FEA46064FEA4707A0
:106CE00020D19B1A09EB4305BDF9363098453FF793
:106CF0006DAEBDF93090BDF93430994507DD3444AF
:106D00003D4408F10108EFE7DFF888B0DCE734F82C
:106D1000191035F81900059AD84724F8190009F117
:106D20000109E8E7069BA9EB41095D1ABDF9363078
:106D300098453FF74BAEBDF930A0BDF934309A45C8
:106D400006DD079B34441D44B94408F10108EDE712
:106D500015F80A2072B1F92A94BF059B059A34F8F8
:106D60001A1039F81A009CBF13FB02F2120AD84716
:106D700024F81A000AF1010ADFE700BFA56000004D
:106D8000D9F90100A3F901000BFA0100E9E80000BC
:106D9000F56000007561000030B5A1B004460392B3
:106DA0000BA80C4A029190470B4A02991288ADF841
:106DB0002E2020460BAA094DA84704A8084A904750
:106DC000002200922046039B0299064C04AAA04789
:106DD00021B030BDA19B00009CFA0100ED9B00009A
:106DE0004578000075780000013900F1080311F8BA
:106DF000012F00F8012B9842F9D170472DE9F04F8F
:106E00002DED028BB9B01C469DF810310C939DF806
:106E10001431079382469C4B22A889461546984711
:106E20009A4B98479A4B9847BDF88830018A428A16
:106E300004905B1AADF88830BDF88A309B1AADF823
:106E40008A30BDF88C305B1AADF88C30BDF88E30CE
:106E50009B1AADF88E308F4B98470B90F8B963882A
:106E6000EBB92389B3F5807F19D10C9BBBB9079B84
:106E7000002B40F09980A37A002B40F09780A27BF2
:106E800002922278019201220092834C2A465146B6
:106E90004846A04739B0BDEC028BBDE8F08F079B98
:106EA0000233DBB20593049BBAF80480B3F91210E5
:106EB000BAF90020B3F91030BAF90270BDF9886050
:106EC000BDF98A0008F10108A8EB02087F1AD21A5E
:106ED000C71BB21A0FFA88F808FB0722059F02FBAE
:106EE00007520892BDF88C200132921B13FA86F3E8
:106EF00096B212B29BB21192721EADF8903013444A
:106F0000ADF89430BDF88E3001331B1A1BB211FA64
:106F100080F11793638809B2ADF89210ADF896101E
:106F2000002B40F064822389B3F5807218BF0122E0
:106F300015920B9A002A40F05C82B3F5807F40F0F6
:106F400058820C9B002B40F05482A37A002B40F017
:106F50005082079B002B00F04C82504D22A8A8477E
:106F6000B0F5F07F24D822A8A84707464C4E7800F9
:106F7000B04708EE100A3846B047059B119A13FB3C
:106F800008FA22EAE2724FF00008064643460492ED
:106F9000179A42454DDD18EE102A06EB030C02EB62
:106FA000430E0021089A14E003237BE7022379E7CC
:106FB0004FF4F077DAE790780CF8010B30B192F8E3
:106FC00001B0107800EB0B202EF81100059801316C
:106FD000024411988842EEDC049ABDF888101344EC
:106FE000089A52440892BDF88C200132521A03FAD2
:106FF00082F2BA4208D2BDF89620013212B2ADF840
:10700000962008F10108C3E7A37B0293237801933C
:10701000022318EE102A00931F4D334624A9484638
:10702000A847BDF89620013212B2ADF89220002395
:10703000E5E7BDF99630BDF992209A420FD0013BA9
:10704000ADF89630A37B029323780193022300933B
:1070500018EE102A104C334624A94846A047304663
:10706000104CA04718EE100AA04713E74FF4F07336
:107070000A93C8E10522DEE110931693199313E2F7
:107080004FF0020B24E200BFE96D0000E94F000061
:10709000E1D90000F1970000FD67000071DE0000FB
:1070A000B5EE000069EB0000049BBDF98820B3F940
:1070B00010301344BAF900209B1A1B9307EB080306
:1070C00008EE903A069318EE103A03EB48031D932E
:1070D000089B0D930023099A0E931A9B13441BB22D
:1070E0001E93119B0E9A934243DC1F9B98440B9B6B
:1070F00033B30498BDF88A20408ABDF88C30BDF8BF
:1071000088109D4D0244099802440498008A013376
:107110005B1A01441BB218EE900A12B209B2A847DA
:10712000002840F02381BDF88C10BDF88830013173
:10713000C91A18EE900A914B09B298474FF0020B0A
:10714000089B1C9A13440893BDF88C30BDF8882026
:1071500001339B1A0A9A08FA83F3934280F016814E
:10716000BDF896300133ADF89630099B0133099391
:10717000C9E1159B002B00F0D7800E9A1B9B1E992E
:1071800026981344BDF9A0201BB29B1ABDF9A2207A
:107190008A1ABDF8A610B1F5807FDDE92F6519D1F7
:1071A000DDE931E101FB03FC51430EFB12CC0EFB88
:1071B000031106EBEC1605EBE113BDF99C200F93D0
:1071C000B2EB262F4FEA262318931BDC069A0023E6
:1071D0001370B0E0BDF8CE104B434A43BDF9A41084
:1071E00011B91E44AB18E8E7DDE931E103FB01FC0E
:1071F000514302FB1ECC03FB0E1106EBEC3605EBF4
:10720000E133DAE73312002BE0DB0F9B0F991B12FF
:107210001293BDF99E30B3EB212FD7DD129B002BCB
:10722000D4DB9DF8CC5015F00401139166D03112D7
:1072300002FB031215F0020F4FEA420351D110F87E
:1072400012208DF8AC20C1184A788DF8AD200222AA
:1072500013929DF8CC20D20704D5BDF8AC20B2F52E
:10726000FC6FB3D09DF8AB209AB10F9AADF8D22045
:107270003693189A139BADF8D4208DF8DC30129A0F
:107280003F4BADF8D06026A8ADF8D620984700282F
:107290009CD0069A9DF8AE301370BDF8AC30A27A3F
:1072A000D2B116991498149DC3F3451202FB001233
:1072B000109803F01F01D20801FB0501C1F304215E
:1072C00002F4FC620A431999DB0A03FB0513C3F3BA
:1072D000072342EAC3239BB21D9A0E9922F811306C
:1072E00029E01344C218C15C8DF8AC1051788DF8B8
:1072F000AD1092788DF8AE200322A9E7BDF9601099
:10730000BDF94820BDF8A8301E4D2CA8CDE92012AB
:10731000A8471D4BADF8AC00DDE920122CA898471A
:10732000139B8DF8AE0094E7079B7BB10D9B069AEB
:107330009B7813706BB90E9B059A01330E930D9BCE
:1073400013440D93069B01330693CAE6069AFF2366
:1073500013700D9B5A781B7803EB02230C9A9BB297
:10736000002A9CD0B3F5FC6F99D12FE7022808BF03
:107370004FF0020BE4E600BF6197000019F0000037
:10738000E5C1000089BD000079BE0000A37B029327
:1073900023786B4DCDE900B318EE102A3B4624A9A3
:1073A0004846A847BDF8963001331BB2ADF892307D
:1073B000ADF89630079BA3B90C9B93B9638883B94A
:1073C0002389B3F5807F14BF4FF0020B4FF0010B00
:1073D0000B9B4BB10A995B4B384698474FF000081E
:1073E000C3E64FF0020BF3E7DDF82C80BDE6012386
:1073F0001593554E22A8B047B0F5F07F3FF636AE54
:1074000022A8B0470A900A9B504E5800B04708EE99
:10741000100A0A98B0474E4B0746482126A89847BD
:10742000159B63B3079B002B7FF424AE0C9B002BB2
:107430000CBF042206226388ADF8A4302389ADF87E
:10744000A630BAF80630BAF80210269501335B1A56
:10745000ADF89E30A388ADF8A030E388ADF8A23037
:10746000A389ADF8A830E37BADF89C80C3F300039B
:107470008DF8AB3026A8374B8DF8AA209847A37A11
:10748000DA43D2B21492002B3FF4F6AD627BD208FD
:107490005A431992A289C2F345125A431692227B8B
:1074A00002F01F0253431093079B002B7FF4E8ADBB
:1074B0000C9B002B7FF4E4AD6388002B7FF4E0ADE0
:1074C0002389B3F5807F14BF4FF0020B4FF0010BFF
:1074D0000B9B1BB10A991B4B38469847049BBDF97F
:1074E0008A20B3F912301344BAF902209B1A1A9376
:1074F000059B13FB08F31C93002309939846119BEB
:1075000023EAE3731F93179B099A93423FF7CCAD8D
:10751000BDF99630BDF992209A420ED0013BADF8EC
:107520009630A37B02932378054CCDE900B318EE87
:10753000102A3B4624A94846A047384690E500BF9C
:10754000FD67000075F0000071DE0000B5EE000080
:1075500019F0000065BF000010B5084B044610216B
:1075600098470023A381FF2323704FF48073238166
:10757000E37B43F00103E37310BD00BF19F000008B
:107580000438C0B20A289DBF024B1B18987800200F
:10759000704700BF9CFA0100032805D00638042874
:1075A0008CBF002001207047012070470E289DBF2E
:1075B00047F6A47323FA00F000F0010000207047A2
:1075C0002DE9F04F2DED028B04468DB088461F4605
:1075D00010464AB9764B0093764B4D227649774D4B
:1075E0000220A847764A17E01B78052B69D9B9898C
:1075F000744B98470546002800F0BC80037B8269E5
:1076000003F01F038AB1704B0093F7226F4B6A4956
:107610006A4E0220B047AA696D4B414620460DB024
:10762000BDEC028BBDE8F04F18471846694A9047F9
:1076300003901846684B98472B690490002B45D05F
:10764000664B08A8214698477B88388913B9B0F55E
:10765000807F26D0E288618826880132521AA1886C
:107660000131891B3E1DCDE900061BB212B209B2E1
:107670005B4E08A8B0472288BDF82030BDF8221024
:107680001344ADF8203063881944ADF82210BDF8DA
:1076900024100A44ADF82420BDF826201344ADF888
:1076A0002630504B08AA41460AA8984748B1049B87
:1076B0000193039B009320462A694B4C3B460AA941
:1076C000A0470DB0BDEC028BBDE8F08F454B2246C4
:1076D000414606A898470028F3D0BDF81C60BDF8C5
:1076E00018300136F61A33B2059303EB43003F4BD3
:1076F00098473A4B06A9814608A898473C4B012178
:1077000008A89847BDF91830B4F90020BDF91AA0AF
:10771000B4F902109B1A1BB208EE103AAAEB010B47
:10772000BDF91E309A4503DD324B48469847C8E7FD
:107730002C4B08AA41460AA89847002835D0059B3B
:107740002D4ECDF8009018EE101A0FFA8BF2284645
:10775000B047012813D02846284B184D9847284B8E
:1077600000930220194B14494FF49A72A847214BF9
:1077700048469847144B009358220E4B2EE7049B23
:107780000193039B0093184E3B464A460AA908A85A
:10779000B047BDF822300133ADF82230BDF82630B5
:1077A0000133ADF826300BF1010B0AF1010AB7E7FE
:1077B0004BFA0100A9FA010017FA0100E9E80000FC
:1077C00063FA0100A5C400006BFA0100B5FA0100DC
:1077D000996D000099750000AD750000E96D00001D
:1077E00061C000008DDE0000FD6D0000B5EE000000
:1077F00067DE000069EB00002DD000004DD00000D6
:107800007CFA010038B10078A0F120035F2B04D985
:10781000C009400070470320704701207047A0F165
:107820003003DBB2092B0AD9602884BF2038C0B2EC
:10783000A0F14103052B9ABF3738C3B20023184685
:107840007047000010B5094B04461C219847FF23E0
:107850002372074B63604FF6FF73E38123824FF47B
:10786000F81323600023A37510BD00BF19F00000BA
:10787000100000202DE9F04F2DED048BD1B08A4689
:107880000A9300232193137A5E9C0590052B93465F
:1078900040F2DB80536808EE103A0A9B1B78002BFD
:1078A00000F0D3800A469C4B014631A89847002837
:1078B00000F0CB809BF817309F0700F1CB80059B31
:1078C000059A9B88128801339B1A1BB218EE102A66
:1078D000B2F90860059ABBF90A50B2F900200B9280
:1078E000059AB2F90200BBF912202492BBF91420C8
:1078F0008718B9B23FB235440697002C00F0BC801F
:10790000002A40F0BB80002880F2B980A268121AD9
:10791000002AB8BF5242C5F50070B2EB400FC4BF99
:107920004FF0FF3222602268002AC0F2A780049242
:1079300062680A4412B206921BB2049F0A98BBF90D
:107940000C2009EE103A9BF817300093384419EEDA
:10795000103A18EE101A714FB847049BC3180793DA
:10796000069ABAF902109BF8173032448A420A9AF2
:10797000C0F2878004995E0702EB010040F1AB8002
:10798000079A0093511ABBF90C30654C18EE102A77
:1079900089B2A047059B059A9B88128801339B1AE0
:1079A0001BB2181A0B9B00EBD07003EB600003B204
:1079B0000B939BF808302093BBF80E301093BBF864
:1079C00010301193DDE91032934288BFCDE91023C6
:1079D0009BF8183099071CD0524B35A89847BBF834
:1079E0000030ADF8D430DBF80430B3F908300A22A7
:1079F000053393FBF2F3ADF8D6309BF808309BF8D3
:107A000019208DF8DC309DF8DD3062F301038DF82C
:107A1000DD30454B3BA89847BBF80230ADF8EE305F
:107A2000209B0B9CFA2B88BFFF230993ABB22293B8
:107A3000BDF818301E9300231D93049A0A9B13442B
:107A40001C930A9B9B5C002B5ED151B0BDEC048B58
:107A5000BDE8F08F029347F618430193BBF90A3053
:107A60000093DBF80420BBF90C300A992F4D3BA89A
:107A7000A847BDF9EC3029E704945DE700220492A1
:107A80005AE70799009302EB010819EE103ABBF987
:107A90000C2018EE101A4046B847079B1844069B66
:107AA0002B441BB2069374B113F5806F0BDB236874
:107AB000002B08DA079B2360059B069AB3F9023076
:107AC000D21AC4E90123079B049398F80030002BD5
:107AD000BBD0079044E71C077FF56BAF079A04996A
:107AE0000093511ABBF90C300D4C18EE102A89B2D4
:107AF000A047059B059A9B88128801339B1A1BB2ED
:107B0000181A0B9B184452E7249B1C4423B20C9375
:107B1000002330930893C2E08DDE0000C5FF000013
:107B20001DFF0000E1850000A19B00009D010100F8
:107B3000109A4FF6FF739A4224D0119A9A4221D09C
:107B4000049AA34B0A981B681144984786B2A14C2B
:107B50001C98236830A998471C9A236805463098DA
:107B60000021104498479BF8173013F00103024698
:107B700000F02581232D0FD1089929B9BDF8C02027
:107B80001D92C7E70026E2E7089B012B45D0022B98
:107B900040F018810023BDE7089B012B40F00F81C6
:107BA000202D7CD1309B1D9A9B1A072B32D11C9B18
:107BB0001D999A1858589388ADF8E430864A389041
:107BC000C0F30745C0F30764C0F30726C0B290476F
:107BD0000146F0B2904700EB0111E8B2904705462C
:107BE000E0B2904700EB05149DF8E400904705468D
:107BF0009DF8E500904700EB0510C0F3C400C4F306
:107C0000850440EA4410C1F3C40140EAC123219332
:107C100002237FE7BBF80030F9E70023BBF8004000
:107C200008936E4B18EE100A29469847109A1F9039
:107C30004FF6FF739A4220D0119A9A421DD0109BA2
:107C4000B3421AD8B24218D90C9BADF8E030069B6B
:107C5000ADF8E230BBF80C300C9A013B13440344FE
:107C6000ADF8E430229B069A013B1344ADF8E630B0
:107C70003BAA5B4B514638A898479BF819301B9399
:107C8000209B042B00F285841F9B43B1BBF80C3072
:107C90000C9A1A4413461F9A1A4413B20C93079B6A
:107CA000049A30999B1A8B423FF642AF9BF81830EA
:107CB0009D071FD50B9BADF8CC30DBF80430494C49
:107CC000B3F9083003EBD372BDF9D63003EBD373AD
:107CD0005B1003EB62031E9A13441BB20C9AADF8BF
:107CE000CE30ADF8E020ADF8E230524635AB38A9E1
:107CF00033A8A0479BF81830DC071ED50B9BADF8C6
:107D0000CC30BDF9D630DBF80420364C11895289CD
:107D100003EBD3735B1001330B449B1A1E9A13447D
:107D20001BB20C9AADF8CE30ADF8E020ADF8E230E1
:107D3000524635AB38A933A8A0470A9B079A2A4C6C
:107D40009E189BF81730009318EE101A19EE103A8F
:107D5000BBF90C203046A047079BC518059BB3F91B
:107D600000409BF817300146580740F1FD8318EE9C
:107D7000102A00933046BBF90C301C4EB047059BCF
:107D8000059A9B88128801339B1A1BB2181A00EBC4
:107D9000D07004EB600004B2229A069B13441BB21D
:107DA00006931E9B13449BB21E93079B069A049353
:107DB000BAF906309342FFF648AE07953DE6089BB8
:107DC000022B02D0BBF800402BE7219C29E700BF23
:107DD00064000020580000201F78000075D10000CA
:107DE000ED9B0000FD850000C5FF00001DFF0000A9
:107DF000BDF8E420BDF8E21052EA01033FF444AFBD
:107E00000C98BDF9E63003440D930D9F3944BAF93F
:107E1000007018EE100A18EE103AB942B0F90A6074
:107E2000B3F90830BDF9E800FFF62EAFBAF9041037
:107E30000D9F8F423FF728AF06999B1B0B449B1A5F
:107E40001B1A1A441693BAF902309A42FFF61CAF75
:107E5000BAF90630169A9A423FF716AF18EE100A92
:107E6000A94B29469847074628B9A84B009340F2EA
:107E7000B712A74B9FE318EE103A1A7BBDF9346096
:107E8000BDF958809DF8EA30920700F0FA8104F0BD
:107E90001F022A92C4F345122692032BC4F3C42274
:107EA000259200F0E680013B072B00F2D780DFE847
:107EB00013F0DB000800D500E000D500D500D500A8
:107EC000D000C0231393934B02241493BDF8E230E7
:107ED000179304FB03F1BAF90030179DBDF8E420B5
:107EE000B342C6BF9B1B03EB430300231293BAF9B3
:107EF00004300320B5FBF0F030449842C5BF9B1B13
:107F00000133179B03EB43031993BAF9023043453E
:107F1000CCBFA3EB080300230E93BAF9063002EBA3
:107F200008009842C2BFA3EB080301332393129BBE
:107F30000E98D8BF2392634300FB013307EBE301A4
:107F400003F007030F93179B734F1A915343B3F535
:107F5000F07FA8BF4FF4F07318461893B847189BEA
:107F600005465800B8476D4B08EE900A98476C4B91
:107F70009847B0F81490B0F910C0129BD0F808E000
:107F8000032209F1010993FBF2F1B0F912300E98C6
:107F9000A9EB0C090FFA89F9A8EB030309FB0363AA
:107FA00009FB0010A3EB0C0303440EEB43030D98F5
:107FB0001593BDF8343011FA80F1013BADF8CC10C7
:107FC000199991FBF2F21A44ADF8D020169B0E9A43
:107FD00013441BB2ADF8CE30ADF8D230514B9847B8
:107FE000129A199B27909B1A1693179B1344199A60
:107FF0009B1A6343169A28936FF0020392FBF3F3E4
:108000004B445B00299300231F46C4F108032D93C2
:108010000E9B239A934231DBBDF9D230BDF9CE20BD
:108020009A420FD0013BADF8D2301B9B0293099BC3
:1080300001930223009318EE902A3B4C2B4633A960
:108040005046A0472846394CA04718EE900AA04752
:108050001AE6FF2313930824354B36E7354B00937C
:1080600040F27A22344BA6E2802313930124334B4F
:108070002BE7F02313930424314B26E70F9A139B2D
:10808000DDF848E023FA02FC3E460022199B7345C6
:108090005CDC279BCBB13B462B449846BDF8D030E7
:1080A000BDF9CC10BDF9D220264F01335B1A1BB2AB
:1080B0004046B84748B9BDF8D010BDF8CC300131C2
:1080C000C91A09B2204B40469847169B189AF318D4
:1080D0009A4240F3C180BDF8D23001331BB2289AD6
:1080E000ADF8D2300F9B13441A9A02EBE30203F06F
:1080F00007031A920F93299A159B134415930E9B0D
:1081000001330E93374683E765D1000021FB010060
:10811000A6FC010092FB0100B5EE0000E94F000053
:10812000E1D90000F1970000FD67000069EB000055
:10813000A6FB01004EFB0100B5FC010090FB010015
:1081400096FB01006197000019F000000F9BE318F7
:108150000D931A9B0D991B78C1F1080103EA0C03DA
:10816000CB4007D00999FF2960D1082C1ABF149978
:10817000CB5CDBB202F5A07169440132032A01F83D
:10818000843C48D1159A9DF8BC305178259A9DF8C9
:10819000BE90C3F1FF00C90813FB02F200FB0122ED
:1081A000120A1792159A10782A9A00F01F00C9F146
:1081B000FF0819FB02F108FB00122B92159A9DF89B
:1081C000BD8032F8020B1592C0F345121146C8F17A
:1081D000FF0243EA09032C92269A58EA030318FB8C
:1081E00002F018BF4FF0FF330A4608BF00232C9956
:1081F000AB552B9B01FB0200C0F30520C3F3042108
:10820000179B41EA401141EAC32118EE903A00223F
:1082100023F8161001360F9B2D998B4214DA0D9B13
:108220000F932CFA04FC0EF1010E2FE7082C17BF58
:1082300014990999CB5C09990BBF4B4313FB01F3CC
:10824000C3F307231B0A95E71A9BDDF84CC00133E3
:108250001A9300230F93E6E71B9B0293099B01935C
:108260000223A74E009318EE902A2B4633A95046BE
:10827000B047BDF8D23001331BB2ADF8CE30002686
:108280002DE7032B09EE904A00F0C080013B072B3D
:1082900000F2B080DFE803F0B404AEBAAEAEAEA731
:1082A000C0221392974A022504230E92099AF92AB2
:1082B00012D8954A099892F80011814240F0AC809A
:1082C000D2F80421AA4240F0A7808F4B099A83F884
:1082D0000021C3F804510E93BAF90030BDF8E290C2
:1082E000BDF8E420B342CCBF9B1B00230F93BAF927
:1082F000043009EB06009842C4BF9B1B0133BAF956
:108300000260C8BF1293BAF90630D8BFCDF84890C2
:1083100002EB08004645CCBFA6EB080600269842B3
:10832000C2BFA3EB0803013317930F9BD8BF17926B
:1083300005FB09F103FB05F406FB014407EBD4033D
:10834000149302FB09F3B3F5F07FA8BF4FF4F07369
:10835000159318466D4B98470D9A0F99BDF8343018
:1083600011FA82F2ADF8CC20129A013B1344ADF819
:10837000D030169B33441BB2ADF8CE30ADF8D230BE
:10838000634B08EE900A9847C5F108030D930F9BC5
:1083900019909944129BA9EB030905FB09F304F01A
:1083A00007041A934FF00009179B9E4245DBBDF965
:1083B000D230BDF9CE209A4210D0013BADF8D23078
:1083C0001B9B0293FF260223CDE9003619EE902A6B
:1083D00018EE903A4F4C33A95046A04718EE900A39
:1083E0004D4B984750E4FF22139208254B4A4FF417
:1083F00080735AE74A4B009340F2E512494BDAE0AA
:10840000802213920125484A02234EE7F02213925C
:108410000425464A102348E70E993B480B4411F8BF
:10842000012BFF2A17BF099C099A12FB04F2120ABA
:10843000994200F8012BF2D147E7139B0F99CDF831
:108440008C9023FA04F218EE903A03EB09084746A1
:10845000129B8B423ADC0F9A12999B1A16938A420E
:10846000C8BF002318939944199BB3B1BDF8D0300D
:10847000BDF9CC10BDF9D2202D4F01335B1A1BB2D0
:108480004046B84748B9BDF8D010BDF8CC300131EE
:10849000C91A09B2274B40469847189B169A1344AD
:1084A0009846239B9844159B434545D9BDF8D23047
:1084B00001331BB2ADF8D2301A9B1C44149B03EB62
:1084C000D403149304F0070401366DE7149B0D9850
:1084D0001B78A0EB040C134033FA0CF31CBF0E986E
:1084E000C35C07F8013B0D9BA3429DBF149B139AED
:1084F000013364198EBFEA40149300240131A7E7C9
:10850000FD67000092FB0100C8840020B5EE00006A
:10851000F1970000F161000069EB0000A6FB01008B
:1085200074FB0100C7FC010090FB010096FB0100F9
:108530006197000019F000001B9B0293FF270223A4
:10854000CDE9003719EE902A18EE903ADFF88C80CA
:1085500033A95046C047BDF8D23001331BB2ADF845
:10856000CE304FF00009A5E71A077FF515AC18EEDD
:10857000102A00933046BBF90C30124EB047059BD1
:10858000059A9B88128801339B1A1BB2181A204443
:1085900001E418EE100A0C4E00232A4638A9B04711
:1085A00000287FF425AC1F2D7FF66EAB074B0093A0
:1085B000074B40F2A1120749074C0220A047FFF7E2
:1085C00063BB00BF1DFF000069D10000FCFA010081
:1085D000A6FC0100C6FA0100E9E80000F161000014
:1085E00010B5054B04460A219847FF232372002348
:1085F00023800123638010BD19F000002DE9F04FA6
:108600002DED048B9B46B3F90230C7B0CDE90501CF
:1086100008EE902A002B00F0E4809BF80820052A41
:1086200040F2DF80059AB0F90040B1F90000B2F9DC
:108630000210069A8442B2F9022002D1914200F05F
:10864000D08003EBD373C3F34F038442D4BFC3EB97
:108650000405C3EB0005ADF828508442ACBF1D19DA
:108660001D189142D4BFC3EB0100C3EB020091423D
:10867000ACBF5B189B180AA9ADF82A0018EE902A27
:10868000AA4CADF82C500846ADF82E30A047002873
:1086900000F0A780059BB3F90290069BB3F9028016
:1086A000C14540F05981A24B9BF808409847A14B27
:1086B0009847BBF90230BBF90650013B03F00106B5
:1086C00080465F1006EB630625B1BBF90450003D00
:1086D00018BF0125984B9847002840F0878085F007
:1086E0000102069B0599B3F90030B1F900108B42E5
:1086F0001846A8BF08468B42B8BF0B46013BADF8F1
:108700009C30059BADF898005B889E1B3B44ADF800
:108710009A60ADF89E30002A6AD09BF8093003F0C9
:108720000303CDE9014301230093BBF80020834CF0
:10873000002326A90AA8A0479BF8093013F00C0FC4
:108740004FD07F4B31A89847BBF80030ADF8C6300A
:1087500047F6FF73ADF8C4309BF80830BBF9025000
:108760008DF8D0309BF809306C105A076FEA050578
:1087700005F0010518D5059B1A88A3B2D11AADF8EA
:108780009810059949881A44C81A0B44521B5B1B60
:10879000ADF89A00ADF89C20ADF89E3018EE901A16
:1087A000684B31AA26A898479BF809301B0718D5B3
:1087B000069B1A88A3B2D11AADF898100699498879
:1087C0001A44C81A0B44521B5B1BADF89A00ADF853
:1087D0009C20ADF89E3018EE901A5A4B31AA26A86C
:1087E000984747B0BDEC048BBDE8F08F002278E7D6
:1087F00026AA4E4B0AA91046984700289CD0B8F8E4
:1088000012E0BDF99A10B8F81020B8F91060BDF860
:108810009800BDF99C70BDF998C0ADF8C4C0A1EB3B
:108820000E04ADF89A40BDF89C40ADF8C870831AAC
:10883000A21AADF89C20BDF89E20ADF8C6100134F8
:108840001BB2A2EB0E02241AADF89830ADF89E20B0
:1088500024B2ADF8CA10DDB11E44BBF90420BBF947
:108860000630134496FBF3F203FB126633B2079310
:10887000354BDFF8C8A020469847BDF99A900746C7
:10888000BDF99E30994505DD3846304B984753E792
:108890000795EDE72E4B2F4E214638469847BDF8F9
:1088A0009830B8F81220B8F810104A44194412B29F
:1088B000234609B23846B047024695B188B1002335
:1088C000079918460AE0BBF904208A4225DB1344C5
:1088D0005B1A1BB2013301321BB211B29C42F2DCB3
:1088E00002229BF8093003F0030302939BF808303F
:1088F00031A9CDE900230AA83B46BBF80020D047A8
:10890000BDF8C6300133ADF8C630BDF8CA3001330A
:10891000ADF8CA3009F10109B2E7BBF906C06244FB
:108920009142BABFF8540A460022D3E78DDE000018
:10893000E94F0000E1D90000F1970000F16100006B
:10894000A19B0000ED9B0000B5EE000069EB00006C
:1089500075F0000061970000059BB3F90070069B5D
:10896000B3F90060B74240F0DB80664B9BF80860CB
:108970009847654B9847BBF90230BBF90650013B5D
:1089800003F0010807464FEA630908EB630825B1C5
:10899000BBF90450003D18BF01255C4B984720BB34
:1089A00085F00102059B05991B88B1F90210A3EB24
:1089B00008084B44ADF89C30069BADF89880B3F99D
:1089C00002308B421846A8BF08468B42B8BF0B4600
:1089D000013BADF89A00ADF89E3042B19BF80930EA
:1089E00003F00303CDE901639DE60022DAE726AA3E
:1089F0000AA91046A04700283FF49EAE3B8ABDF866
:108A00009840B7F812C0BDF99800BDF89C60ADF869
:108A1000C400E21AADF89820BDF99A20ADF8C6203E
:108A2000A2EB0C01F31AADF89A10BDF99C10ADF849
:108A30009C30BDF89E30ADF8C8100136A3EB0C0396
:108A4000361BADF89E3033B2184608EE103AADF83A
:108A5000CA202F4B98478046C5B1BDF99830B7F969
:108A60001040BBF904201C44BBF90630134494FBAE
:108A7000F3F203FB124424B2BDF99A90DFF89CA0F4
:108A8000BDF99E30994503DD4046FEE62C46F3E7EE
:108A900018EE101A1F4B204E40469847BDF89830EC
:108AA0007A8A398A4A44194412B218EE103A09B245
:108AB0004046B0476DB150B1BBF90420BBF9063058
:108AC0001344A242B8BF00209C42A8BF0024013436
:108AD00024B2002302939BF80830BBF80020CDE9B4
:108AE000000331A943460AA8D047BDF8C630013378
:108AF000ADF8C630BDF8CA300133ADF8CA3009F15F
:108B00000109BDE7E94F0000E1D90000F19700003D
:108B1000B5EE000075F0000061970000F161000003
:108B2000C14505DB4B46C14698463B4637461E4687
:108B3000F31B0993A8EB09030893F31B83EAE37281
:108B4000A2EBE372089B079283EAE37AAAEBE37A4B
:108B500052451346D8BF079BBBF90250CABF4FEA24
:108B60004A135B01B3FBF2F3B34AD8BFB3FBFAF38A
:108B7000D25C3F2315FB0235C5F3CF13BE42D4BFF1
:108B8000C3EB0602C3EB0702ADF83020BE42ACBF18
:108B90009A19DA19ADF834200CA9C845D4BFC3EB33
:108BA0000802C3EB0902C845ACBF43444B44ADF8CF
:108BB0003220ADF836300AAAA04B0846EC1198478F
:108BC00000283FF4B9AD079B04F0010404EB252411
:108BD0005345A4B2C5F30F2540F3ED8014FA89F391
:108BE0001BB208EE103AF31BA9EB050A14FA88F43D
:108BF000A8EB0505002B4FF0000324B20FFA8AFA08
:108C00002DB2019340F3C680009533465246394653
:108C100010A88B4DA8470123CDE9004318EE102A78
:108C2000334639461BA8A847DFF840A2002110A808
:108C3000D047002109EE100A1BA8D0479BF8095025
:108C400015F0100509EE900A40F0CF800322BDF820
:108C500020400192F21BBDF82430079319FA82F2EA
:108C60003B1B12B239460092754F1BB24A4626A8EA
:108C7000B84702220192079A424412B2331B1BB238
:108C800000923146424631A8B847294626A8D04727
:108C90002946099031A8D04782466A4B6A4E9847C8
:108CA0006A4B9847BDF83020038ABDF83440D11A8A
:108CB000E31AADF83010ADF83430418ABDF83630E3
:108CC0000546BDF832000134401A5B1AA41AADF80B
:108CD0003200ADF836300CA823B20793B047B0F598
:108CE000F07F80F087800CA8B0470746584B384685
:108CF00098472B8ABDF830201A4412B20892ADF87A
:108D00003820BDF834201344ADF83C306A8ABDF8F1
:108D1000323013441BB2ADF83A30ADF83E3039462C
:108D20004C4B06469847BDF93280B5F912304FF0EA
:108D300000099844BDF93630B5F91220134498451E
:108D40005BDDBDF93E30BDF93A209A4213D0013BBC
:108D5000ADF83E309BF80930BBF800203E4C03F0E4
:108D6000030302939BF808300193022300930AA99E
:108D700033460EA8A047394B394C3046984719EE78
:108D8000100AA04719EE900AA0470998A04750463C
:108D9000A047D1E418EE102A009433463946284CF7
:108DA00010A8A0470123CDE9005352463346394667
:108DB0001BA8A04738E714FA86F3002214FA87F4B8
:108DC00021B2CDE900821BB24A461D4C10A8A04733
:108DD0001FFA86FABAB2511BAAEB05030122CDE9AC
:108DE00000821BB24A4609B2E2E74FF0FF3ACDF8E3
:108DF00024A052E74FF4F07778E706EB090308EE7A
:108E0000103A0899079B174C18EE100A0FFA88F2CF
:108E1000A04720B90799144B18EE100A9847079BF2
:108E200099444B449F4223D9BDF83E300133ADF8FD
:108E30003E3008F101087DE7E2FC01008DDE000014
:108E40000D980000E94F000071DE0000E1D900003C
:108E5000B5EE000075F00000F161000069EB000064
:108E6000A19700006197000019F000001197000021
:108E70009BF80930BBF800200D4C03F0030302936C
:108E80009BF808300193022300930AA933460EA8E9
:108E9000A047BDF83E3001331BB2ADF83A30ADF813
:108EA0003E303946034B304698474FF00009C0E743
:108EB000F161000075F00000F9290AD8052907D9E9
:108EC00010FB01F048F281035843C0F3C7507047CC
:108ED000002070472DE9F047089E1C46B38AD21A3D
:108EE000738AC91A0FB296F82830316A054612B251
:108EF00003F0010099BB337C03F0020680B13EB160
:108F000003F00303022B05D10132ACBF0020012086
:108F1000BDE8F087032B01D1002AF9DC0020F7E738
:108F2000002E40F0878103F0030001280AD1002FB2
:108F3000EEDCE742F2D4002F00F37E8179428C42CE
:108F4000ECDD9BE00028F4D1391900F17381002F8A
:108F5000E4DC7842A042C0F29C800220D8E703F013
:108F6000020C002800F09780F16907FB01F300294B
:108F70004FEAA3235FFA8CF005DD9A4205DA003848
:108F800018BF0120C4E79A42F9DC3B194B43002982
:108F90004FEAA32305DD9A4206DDB0FA80F04009CE
:108FA000B6E79A42F9DB0132B36912025A439212D0
:108FB000111212F0FF021FBF736AC2F1FF0803FB18
:108FC00008F84FEA282814BFC8F1FF084FF0FF083F
:108FD000CF1B002A54D0002F0FDBBC420DDDC2F1A5
:108FE000FF01C8F1FF035943C1F3472108B9C94341
:108FF000C9B2E85DA34B9847E8557A1CDFF8849224
:10900000716A96F82830884503F0020318DC944210
:1090100029DD002A27DBB169F06901FB08F189121B
:1090200008FB01F1C1F347210028BCBFC943C9B205
:109030000BB1C943C9B2A85C924B9847A85412E03F
:10904000002A0ADB944208DDA8EB6101C9B20BB12A
:10905000C943C9B2A85CC847A854736A0132944294
:10906000A8EB0308CCDC96F8283099070AD5BC4257
:10907000FFF654AF002FFFF670AF3946284683E065
:109080003A46BBE7501C3FF549AF8442FFF665AF57
:10909000211A284478E0B16901FB02F300294FEA64
:1090A000A323CCBF03F1010E9E4677455FFA8CF0F7
:1090B0003FF765AF07EB040C63453FF76EAF4FEA30
:1090C000022C013212024A4301FB0CFC4FEAA24976
:1090D000B9EBAC4FCCF38723C7EBAC4A00F0AE80C2
:1090E00000295ADA0AF1FF38002B00F0C980F26932
:1090F00052425A43BAF1000F4FEAA2220DDB544507
:109100000BDD5343C3F3472108B1C943C9B215F876
:109110000A005C4B984705F80A00B8F1000F17DB0E
:10912000444515DDB36915F80800C2F1FF02594244
:10913000514396F82830891251439F07C1F34721C4
:1091400058BFC9434F4B58BFC9B2984705F80800EC
:1091500096F828309E071AD54445FFF6FEAEB8F1C2
:10916000000F7FF7FAAE414688E708F10108A045F5
:10917000A8BFA046B8F1000F3FF4D0AE7FF7EDAE28
:10918000A4EB080105EB08003F4B9847E5E60AF120
:10919000010084424EDB002878E7F769C3F1FF0342
:1091A0005F43BAF1000F4FEAA7270DDB54450BDDF3
:1091B0007B43C3F3472108B9C943C9B215F80A0074
:1091C000304B984705F80A001AF1010215D4944271
:1091D00013DDB369C7F1FF0703FB07F1891296F8A6
:1091E000283079439807C1F3472148BFC943A85C99
:1091F000244B48BFC9B29847A85496F828309B071B
:1092000008D55445FFF68AAEBAF1000FFFF6A5AEB9
:10921000514633E70AF1020AA245A8BFA246BAF1B5
:10922000000F3FF47BAE7FF798AEA4EB0A0105EB8D
:109230000A00A9E701206BE6002C81E6D046B8F1D0
:10924000000F0FDB44450DDDC2F387211944C1F344
:10925000470108B1C943C9B215F80800094B98473E
:1092600005F8080096F828309B077FF57EAFA9EB3C
:1092700007018C427FF752AE0029FFF66EAEFDE685
:10928000FF23DCE7B98E000019F00000013900F17E
:10929000080311F8012F00F8012B9842F9D170470B
:1092A0002DE9F04F8DB01D46DDF8588098F81290EA
:1092B000B8F910A00023CDE9023306468B4B8B464C
:1092C0000AA808F1080109F0010917469847BDF9F5
:1092D0002A30B9F1000F3AD1BB4201DD002039E05C
:1092E000BDF92E20BA42F9DBBDF9281001EB0A02C4
:1092F0009345A1EB0B0407DBBDF92C2005EB0B001C
:10930000A2EB0A02904209DD03EB0A029742BDF983
:109310002E003DDBA0EB0A02974239DCB9F1000FC9
:1093200025D1A542DADB002C03DB714B2146304608
:109330009847BDF92C00A0EB0B0001300028CDDDD3
:10934000A8420FDA291A3044694B98470DE0BB4216
:1093500003DD01200DB0BDE8F08FBDF92E20BA422B
:10936000C2DAF6E70CB9A842F3D00220F2E724EA09
:10937000E470A842F9DCBDF92C10A1EB0B01091A2D
:1093800001314318AB4200DD291A0029EDDBDAE791
:10939000BDF82C209BB20130C01AFF1A0132B8F977
:1093A0001030521A3FB212B25B43BA45049200B277
:1093B000019300F39081A0EB0A039F42D5DBC01B11
:1093C000D8F81430BAF5807FAAEB0000D4BF4FF470
:1093D00000624FF40042984200F1010767D0019B00
:1093E000059200FB103007A9424B9847059A61E0AF
:1093F000D8F818300693019B059207F1FF3B0BFB51
:109400001B3007A93B4B9847BDF81E30A8F81A300F
:10941000BDF81C30C8F814B0BDF81C10A8F81830FE
:10942000BDF81830059A01398B4207D1BDF81E10DE
:1094300021B9FF21ADF81C30ADF81E10BDF81C108D
:1094400099425BD1BDF81A10BDF81E201144C1F33A
:109450004701B9F1000F01D0C943C9B2AAEB030318
:109460005A1EA71805D4AF4203DAF05D224B984785
:10947000F055049B9A1A501E041905D4AC4203DA25
:10948000305D1D4B98473055B9F1000F22D1AF42E6
:109490003FF724AF002F03DB154B39463046984782
:1094A000601C3FF51BAFA8423FF75FAF4AE7D8F813
:1094B00018300793019B059207FB173006A90D4B47
:1094C0009847BDF81A30A8F81A30C8F81470BDF8DB
:1094D0001830A1E7781C20EAE070AC42D4BF211A12
:1094E000291AA842BFF641AF4FE700BF8D92000096
:1094F00019F0000095E90000B98E000004990133CD
:10950000AAEB030304EB0308CB1A013B1C44B9F19B
:10951000000F10D008F1010020EAE070A542ACBFB6
:10952000211A291AA84206DA002904DB754B049295
:1095300030449847049ABDF818B0019B049208A9DA
:109540000BFB1B30704B9847BDF822106E4B049AF2
:109550000BF1010A39B9BDF820100139ADF820101E
:10956000FF21ADF82210BDF82010B9422EDB019882
:1095700009A90AFB1A009847BDF82620BDF81A1061
:10958000C2F1FF03C1F1FF015943C1F34721B9F112
:10959000000F01D1C943C9B2B8F1000F07DB45453F
:1095A00005DD16F80800594B984706F80800002C0E
:1095B00005DBA54203DD305D544B9847305508F17B
:1095C000FF380134ADF822200BF1020ABDF820204B
:1095D000BDF81CB0BDF822104C4F12010023D3453A
:1095E00042D23BB1029BADF82630039BADF824304C
:1095F000ADF82210BDF82230FBB1BDF81E10594362
:10960000C1F34721B9F1000F01D0C943C9B2B8F184
:10961000000F07DB454505DD16F808003B4B984772
:1096200006F80800002C05DBA54203DD305D374B52
:109630009847305508F1FF380134B9F1000F7FF435
:1096400094AE08F101018D42FFF648AE002902DB1D
:109650002C4B30469847002CFFF640AEA5427FF7D2
:1096600084AE291B30196FE6019BC1F30F10104423
:109670000AFB1A3C00FB00F3C3EB0C234FEA400C3F
:1096800093FBFCF30344C3F30F101B0103F0F0033F
:10969000194403900293C1F34701B9F1000F01D0BF
:1096A000C943C9B2B8F1000F06DB454504DD16F821
:1096B0000800B84706F80800002C04DBA54202DDCC
:1096C000305DB8473055029908F1FF3801340AF18E
:1096D000010A012383E7D8F81430BAF5807FAAEB9A
:1096E0000707D4BF4FF400624FF40042BB423FF47F
:1096F0007FAE019B059207FB173006A9024B9847E6
:10970000059A78E619F0000095E90000B98E00008E
:1097100073B50E4C002354F83360DAB204EBC30582
:1097200076B10133102BF6D1094B00930220094B7F
:1097300009490A4C5722A0474FF0FF3002B070BDD4
:1097400044F83300696010B2F8E700BFF4860020E7
:1097500038FD01005EFD010003FD0100E9E80000A5
:109760002DE9F3470D4E0746884691469A46002458
:10977000356825B90134E0B202B0BDE8F087009544
:109780002D6853464A4641463846A8470028F3D03C
:10979000022808BF01240836EAE700BFF48600204B
:1097A000431C18BF074B4FF000021DBF53F8301089
:1097B00043F8302003EBC003114618BF5A60084637
:1097C000704700BFF48600200022084B30B51146D8
:1097D00014465D680132854204BF1968C3E900443C
:1097E000102A03F10803F4D1084630BDF4860020A6
:1097F0000023054A184652F8331009B10130C0B2AF
:109800000133102BF7D17047F48600202DE9F04189
:10981000BDF9188015460E461F462C213B4B0446C9
:109820009847454505DD2B464546984633463E4616
:109830001F46237C9DF81C20658162F3010323747D
:10984000A8EB0502BB1B83EAE37082EAE271A0EB9E
:10985000E370A1EBE271884294F82810A582D4BF8E
:109860000020012060F30001294D84F82810002019
:10987000C907C4E906002681A781A4F80E80668284
:10988000256020712BD533B14FF4801191FBF3F19A
:1098900051438912E16132B14FF4801191FBF2F230
:1098A00053439B12A361E269237C226213F00303FA
:1098B00007D0012B05D0022B23D1002AD4BF0023CF
:1098C000012394F82810002A63F341014FEAA20310
:1098D000B8BF5B4284F828106362BDE8F08132B102
:1098E0004FF4801191FBF2F159438912A16133B118
:1098F0004FF4801191FBF3F353439B12E361A26990
:10990000D2E7002ACCBF00230123DAE719F00000D8
:10991000D58E0000F8B50446C8888D881F464B8850
:109920000130C01A0B880135ED1A00B22DB2A842E1
:10993000A8BF2846B2EB600F4FEA6003164604F159
:109940000800C8BF1EB2084B9847A37C268267F365
:109950000003A374054B2360022323714FF00042E0
:109960000023C4E90523F8BD8D920000A1920000F8
:1099700070B5B0F9084004FB01F3B2EB232F4FEAB6
:10998000232501DC408870BDB0F90A3001FB03F6E5
:10999000B2EB262F01DB8088F5E71B1B5943521BD6
:1099A0000B1212B241880679C2EB022292FBF3F34A
:1099B0008288DBB2C3F1FF05C1F34511C2F3451242
:1099C000694303FB0211827802F01F0206F01F06B2
:1099D0006A4348F2810403FB062261436243C1F3F8
:1099E000C551C2F3C45242EA4112C1784679C9084E
:1099F000F608694303FB06136343DB0D42EAC32009
:109A0000C1E700002DE9F04F45004FEA610987B03A
:109A1000CB0704465A4B28460E461746CA4658BF3F
:109A200009F1FF3A9847AB1E00934FEA49030193AF
:109A30006FF001030AFB03330146B8464FF0000BF9
:109A400002935C4522DC3B8893FBF6F304FB04F8AD
:109A50003B803A463B464FF0010CC44541D36B4234
:109A600009FB03F30393631E05FB037302930AF1DF
:109A7000010301930AFB055A4FF0000C64453EDCDC
:109A8000404B084607B0BDE8F04F1847009B0198CF
:109A900038F8032000EB080C02987243631E404420
:109AA00021F8132003EB090E7445CCBF3CF813E0FA
:109AB0004FF0000EA2EB0E0EA3EB0A02002AD4BF59
:109AC000B8F8002030F81320013B7244E8D2404639
:109AD0002D4B03912A469847A84403990BF1010B9B
:109AE000AFE7588833F802EB70451CBF90FBF6F0E7
:109AF0001FFA80FEA3F800E00CF1010CADE703981B
:109B0000138810187343059000270AEB0200049095
:109B10009646009390463846009B002BACBFC3F39B
:109B20008F1B4FF0000B21F810B0A0EB090BBBF11D
:109B3000000FCABF059BB8F800B033F807B0009B10
:109B4000A3EB0B0B019B03449C42CBBF049B029BEA
:109B5000DB5B33F81C3001305B4484420093A84443
:109B60002F44D9DC002331F81300AEF80000013394
:109B70009C42AE44F7DC0CF1010C02327EE700BFE0
:109B8000B5EE000069EB000031EC0000013900F196
:109B9000080311F8012F00F8012B9842F9D1704702
:109BA00010B50F4B5421044698470E4B1B88638019
:109BB0000022FF23A280E281A4F84620E283638191
:109BC000237323772375A28684F83630064A84F8F7
:109BD000443084F828300F2322632264638210BD4E
:109BE00019F00000F0FD0100100000202DE9F04FF9
:109BF0009246C2884588531C2DED048B5B1B1BB21B
:109C0000002BADB08346884641F36E818188008881
:109C10004B1C1B1A1BB2002B41F36681BAF9204082
:109C2000002C00F042859AF828300893052B40F26A
:109C30003C85DAF82070BAF92460BAF92630012F91
:109C400003D116B9002B40F33085BAF822709BB2CD
:109C5000A7EB030CB6B21F443944F71A33441A4435
:109C600004EBD4735B105B4292B25E1E89B2C3F107
:109C70000103ADF8441011FA83F112FA83F3ADF841
:109C80004E30089BADF8462060443D44FB2BADB2FE
:109C900080B228BFFF23ADF8400010FA86F015FA15
:109CA00086F6ADF84C10ADF842500893ADF8480078
:109CB000AC4BADF84A609847AB4B9847AB4B054669
:109CC000424612A914A89847002800F0EE84298A79
:109CD000BDF850306A8A5B1AADF85030BDF852308A
:109CE0009B1AADF85230BDF854305B1AADF85430C1
:109CF000BDF856309B1AADF8563059469C4B16A805
:109D00009847BDF85850BDF85A00BDF85C20BDF822
:109D10005E10BDF8447001350130ADB280B2531E03
:109D2000ADF85C30521B4B1E091A12B209B28A42BE
:109D3000A8BF0A46ADF85E30BAF90030BDF842104F
:109D4000ADF85A0052109A42A8BF1A4608EE902A5F
:109D5000BDF84020ADF858500137BF1ABDF8462075
:109D6000844D0132521A12B23FB29742A8BF174631
:109D70007F109F42A8BF1F4604EB070909FB09F0AB
:109D80004000A847BAF92040794B069010A91EA8B8
:109D9000984704F0010204EBD473BDF840100A9216
:109DA000C3F34F0364F00102BDF844001A443A447F
:109DB0000139091A92B2ADF87C200A44ADF8782036
:109DC000BDF84620BDF8421001330132521A9BB251
:109DD000ADF87A3013443E193A46ADF87E30664FFE
:109DE00000231EA925A8B847012C304618BF6410CF
:109DF000A84773000993069B05930023079333B28A
:109E000008EE103A0746079B9E4208DC5B4B38463B
:109E10009847012C06FB06F574D100233EE0584B11
:109E200031463846984725AB0093BDF91C20259D47
:109E300018EE103A00213846A84758B909990598F4
:109E4000504B9847099B059A1A44079B059201338A
:109E50000793D8E73B78059A05989B0193FBF4F3A9
:109E600022F8023B099B394618188242EAD08C46F8
:109E700011F8013F9CF800C09C4517BF9B0132F8C8
:109E8000023C93FBF4F39BB222F8023BEDE7069A07
:109E9000069932F813209209CA540133AB42F6D125
:109EA000BDF84E30BDF84A2001339B1AC3F3C031D0
:109EB00001FA83F302EB63039AB21BB20993BDF874
:109EC0004C300B92BDF8482001339B1AC3F3C031CC
:109ED00001FA83F302EB63039AB21BB20A932A4B93
:109EE0000C92984700283BD1BAF92230002B4FD171
:109EF000BAF9242022B9BAF92630B3FA83F35B0900
:109F0000079346E030B22146069A204F0590B847A5
:109F10000A99214401290CDD069B069A1B880598A5
:109F20009B010124B3FBF1F31380AC4203D3069AE7
:109F3000B847002311E0538832F8026BB3421EBFCA
:109F40009B01B3FBF1F39EB216800134EDE7069A54
:109F5000069932F81320CA540133AB42F7D19FE778
:109F60000023CDE7E94F0000E1D900008DDE0000BD
:109F70008D9B0000B5EE00001599000069EB000014
:109F800075F0000019F00000F1970000059A00003C
:109F90000790BDF84C00BDF84830B24D0130C01AF2
:109FA00000B2B14B984718EE902A012316A908EE8B
:109FB000100A25A8A847AD4B002125A89847BDF950
:109FC0004C30ADF864301FFA89F201339B1AADF8BA
:109FD0006030BDF94A30ADF86230013B134408EE01
:109FE000900A0592ADF866304246A14B18A91AA80E
:109FF0009847002839D0BDF96E30099ABDF86C60D9
:10A000009342C4BF1346ADF86E300A9ABDF968306A
:10A010009342D8BF0C9BBDF96A20DCBF0133ADF879
:10A020006830BDF96850BDF96E300136761B36B226
:10A03000002E1ADD01339B1A1BB20D93BDF962305D
:10A04000D21ABDF96030ED1A069B09FB02551D447A
:10A050001AA9884B1EA89847BDF97A300027ADF899
:10A060007E300D9B9F42C0F2A380BDF94C30059A13
:10A07000ADF8643001339B1ABDF94E200599ADF857
:10A080006030531C5B1AADF86230ADF86620784B37
:10A09000424618A91AA8984700283AD0BDF96A3054
:10A0A000099ABDF86C609342D8BF0B9B0A9ADCBF3B
:10A0B0000133ADF86A30BDF96830BDF96A109342DA
:10A0C000D8BF0C9BBDF96E20DCBF0133ADF8683002
:10A0D000BDF968500136761B36B2002E19DD531CCF
:10A0E0005B1A1BB20C93BDF966309B1ABDF9602058
:10A0F000AD1A09FB0355069B1AA91D441EA85D4B0A
:10A100009847BDF87E30ADF87A3000270C9B9F420F
:10A110007ADBBDF94C30059AADF8643001339B1AF7
:10A12000ADF86030BDF84A301344ADF86230BDF888
:10A130004E309B1AADF8663042464D4B18A91AA80E
:10A14000984780B3079B43B1BBF90430BDF9682041
:10A150009342B8BF1346ADF86830BDF86C50BDF9F6
:10A1600068600135AD1B2DB2002D1CDDBDF86E30D1
:10A17000BDF86A2001339B1ABDF960201BB20C9315
:10A18000B61A09F1FF3309FB0366069B1AA91E44A0
:10A190001EA8384B9847BDF97A300027ADF87E30BD
:10A1A0000C9B9F426EDB069A4FEA69060020A3E0F3
:10A1B0002946314B314C324618EE100A9847BDF90A
:10A1C0007A20BDF97810334618EE100AA0479AF8A5
:10A1D000293002930128089B294C08BF0220CDE9B1
:10A1E00000031EA918EE103ABAF81E204046A047F8
:10A1F000BDF87A300133ADF87A30BDF87E300133E6
:10A200001BB24D4401372AE729461B4B1B4C3246F3
:10A2100018EE100A9847BDF97A20BDF97810334638
:10A2200018EE100AA0479AF8293002930128089BDB
:10A23000134C08BF0220CDE900031EA918EE103A06
:10A24000BAF81E204046A047BDF87A30013BADF871
:10A250007A30BDF87E30013BADF87E304D44013799
:10A2600054E700BF15990000B5EE000011970000FB
:10A270008DDE00008D9B000031EC00006197000036
:10A28000F1610000204B18EE100A2A46314698472B
:10A29000079B53B9BDF97A20BDF978101B4C18EE15
:10A2A000100A2B46A047012800D102209AF8293035
:10A2B00002939AF82830164CCDE900031EA918EE37
:10A2C000103ABAF81E204046A047BDF87A30013354
:10A2D000ADF87A30BDF87E3001331BB201375DE74F
:10A2E00011F8017F13F801CD81F800C01F70EF1A3B
:10A2F000BE42F5DC4A44013081450BDD09EB020525
:10A30000511E2B46F3E700BF31EC000061970000BF
:10A31000F1610000BDF94830059AADF86030013BAD
:10A320001344ADF86430BDF94A30ADF86230013BFA
:10A330001344ADF866304246B84B18A91AA898479E
:10A34000002837D0BDF96E30099ABDF968509342A4
:10A35000C4BF1346ADF86E300A9ABDF96C30934213
:10A36000C4BF1346ADF86C30BDF86C60BDF96E30FB
:10A37000BDF96A200136761B36B2002E1ADD013394
:10A380009B1A1BB20C93BDF96230D21ABDF9603032
:10A39000ED1A069B09FB02551D441AA9A04B1EA8E5
:10A3A0009847BDF97A300027ADF87E300C9B9F426C
:10A3B000C0F29F85BDF94830059AADF86030013B89
:10A3C0001344BDF94E200599ADF86430531C5B1A57
:10A3D000ADF86230ADF86620904B424618A91AA835
:10A3E0009847002839D0BDF96A30099ABDF96850FC
:10A3F0009342D8BF0B9B0A9ADCBF0133ADF86A3099
:10A40000BDF96C30BDF96A109342C4BF1346ADF874
:10A410006C30BDF86C60BDF96E200136761B36B22B
:10A42000002E1ADD531C5B1A1BB20993BDF966306E
:10A430009B1ABDF96020AD1A09FB0355069B1AA9AA
:10A440001D441EA8764B9847BDF87E30ADF87A3093
:10A450000027099B9F42C0F27985BDF94830059AD3
:10A46000ADF86030013B1344ADF86430BDF84A30BC
:10A470001344ADF86230BDF84E309B1AADF866302B
:10A480004246664B18A91AA8984788B3079B43B160
:10A49000BBF90030BDF96C209342A8BF1346ADF85C
:10A4A0006C30BDF86C50BDF968600135AD1B2DB244
:10A4B000002D1DDDBDF86E30BDF86A2001339B1AFA
:10A4C000BDF960201BB20993B61A09F1FF3309FBED
:10A4D0000366069B1AA91E441EA8514B9847BDF956
:10A4E0007A300027ADF87E30099B9F42C0F25C8530
:10A4F000059ABDF848301344ADF86030BDF84C30D3
:10A500009B1AADF86430BDF94A30ADF86230013BBA
:10A510001344ADF866304246404B18A91AA8984734
:10A5200078B3079B43B1BBF90230BDF96E2093426B
:10A53000A8BF1346ADF86E30BDF86C50BDF868305A
:10A54000BDF96A200135ED1ABDF86E3001339B1A52
:10A550001BB20993BDF9623009F1FF36D21A069B8E
:10A5600009FB02661E441AA92D4B1EA89847BDF987
:10A570007A302DB20027ADF87E30099B9F42C0F2A1
:10A580004285059ABDF8483005991344ADF860300E
:10A59000BDF84C309B1ABDF94E20ADF86430531C09
:10A5A0005B1AADF86230ADF866201C4B424618A924
:10A5B0001AA89847002835D0079B43B1BBF906304D
:10A5C000BDF96A209342B8BF1346ADF86A30BDF8B2
:10A5D0006C50BDF86830BDF96E20BDF86A100135C9
:10A5E000ED1A531C5B1A1BB20993BDF9663009F1D1
:10A5F000FF369B1A09FB0366069B1AA91E441EA878
:10A60000074B9847BDF87E30ADF87A302DB2002761
:10A61000099B9F42C0F2428504E000BF8DDE00002E
:10A620008D9B0000059ABDF848301344ADF86030AA
:10A63000BDF84C309B1AADF86430BDF84A30134475
:10A64000ADF86230BDF84E309B1AADF86630424628
:10A65000B94B18A91AA89847E8B1079BDBB9BDF810
:10A660006C60BDF86830BDF86E70DFF8109301368D
:10A67000F61ABDF86A300137FF1A1AA9AF4B1EA8A7
:10A680009847BDF97A30079D36B23FB2BD42ADF86A
:10A690007E30C0F23C85AA4BAA4C18EE900A98472F
:10A6A00018EE100AA0470698A0479AF80C30052B20
:10A6B00040F2A880A14B594616A89847BAF9103025
:10A6C000012B24DD9AF81430F92B20D9BAF9003087
:10A6D000EBB1BAF81230BDF85810C3F380020A4447
:10A6E000BDF85A10ADF85820C3F340020A44ADF843
:10A6F0005A20BDF85C20C3F3C001521AADF85C20AB
:10A70000BDF85E2003F00103D31AADF85E309AF86D
:10A710000C908D4BB9F1FB0F28BF4FF0FF09984704
:10A720008A4B9847844B0590424616A918A898472B
:10A73000002867D0059BBDF860101A8A8B1AADF807
:10A740006030059B588ABDF862301B1AADF8623044
:10A75000BDF864309A1AADF864200133BDF8662064
:10A760005B1A121A1BB2ADF86620184608EE903A32
:10A77000774B9847774B054698470C90BDF830309B
:10A780000D93002B40F0EF849AF80630023B18BF7F
:10A790000123BDF85C600893BDF85830BDF85E40F9
:10A7A0000136F61ABDF85A300134E41A24B236B232
:10A7B000B442BAF90030A8BF344664109C42A8BF26
:10A7C0001C46089B002B00F0D184002C40F0CE8466
:10A7D0009AF80630002B40F07C859AF80D205E4CEC
:10A7E000CDE9019201220092BAF8022016A9404652
:10A7F000A0474FF0FF330B93514B0B989847514BA9
:10A8000028469847DAF82C00D0B19AF83630052B54
:10A8100016D9524B98470128064600F2BC86DAF852
:10A820002C004F4B25A99847012800F056864D4B28
:10A8300000934D494D4B4E4C40F294520220A0479C
:10A840009AF814300593052B40F27481BAF9103050
:10A85000002B00F06F81BAF91230002B00F06A81F2
:10A86000059BFB2B28BFFF230593374B9847374B9E
:10A870009847314B06904246594614A898470028FD
:10A8800000F05881069BBDF850101A8A8B1AADF85B
:10A890005030069B588ABDF852301B1AADF8523022
:10A8A000BDF854309A1AADF854200133BDF8562043
:10A8B0005B1A121A0FFA83F9ADF85620244B48465A
:10A8C0009847244B04469847002840F04987BAF936
:10A8D0001230A3F10F056B426B411F46BBF80430E9
:10A8E000BBF80020BBF8021001339B1ABBF806200E
:10A8F0000132521A1BB212B29342A8BF1346BAF9E0
:10A9000000205B109342A8BF1346002B099340F32D
:10A910002A87099A174D002359461EA8A847164BA7
:10A9200000211EA898470C9016A8044B594698473A
:10A93000BAF8121024E000BF8DDE00008D9B0000ED
:10A94000A197000069EB0000E94F0000E1D9000089
:10A95000B5EE0000F1970000F161000005780000FD
:10A9600029CF0000A4FD01006FFD0100F2FD0100F0
:10A97000E9E800001599000011970000B9EF000008
:10A98000BDF82450BAF81030BDF8582048075EBF13
:10A990005B195B429BB21344BAF81020ADF85830F3
:10A9A0000B0758BF5319BDF85C0056BF5B421346F6
:10A9B0009BB2C31A8E07ADF85C3058BF5319BDF86F
:10A9C0005A00C34E56BF5B4213469BB20344ADF8D8
:10A9D0005A30CB075CBF53195B42BDF85E004CBFD9
:10A9E00013469BB2C31AAA1A12B2ADF85E3016A96A
:10A9F000012325A8B047B74B002125A89847BAF9ED
:10AA00001030099ABDF95260BDF956C0BBF900106B
:10AA10009A42A8BF099BBBF90420B8BF03F1FF33DA
:10AA20000893BAF80E3008EE103A9AF815300793EA
:10AA3000069BB3F912E00EEB060308EE900A1BB278
:10AA4000002F00F09D87BBF90200089FADF8601051
:10AA5000A0EB0E0038448445A8BF8446CDF828C03A
:10AA6000ADF86420ADF86230ADF866300A9BB342B1
:10AA700080F27E86069BBBF90620B3F91230089956
:10AA8000BDF95260D21A521A9642B8BF16460A9AB7
:10AA9000B242A4BF1646013633441BB2ADF8623051
:10AAA000ADF86630BDF956309E4240F3DD86BBF806
:10AAB0000230089A884D013313FA82F3ADF8623000
:10AAC000BBF80630013B9B1ABAF81020ADF866308F
:10AAD000BBF90030ADF86030013A1344ADF8643092
:10AAE000079B02930126059B019318EE102A002371
:10AAF00018A940460096A847BAF81030BBF90420C0
:10AB0000ADF86420F31A1344ADF86030079B02934C
:10AB1000059B18EE102ACDE9006318A900234046D2
:10AB2000A8476E4D18EE900AA8470C98A8476C4BA2
:10AB300020469847DAF83C10002964D09AF844304F
:10AB4000052B60D9002447F61843CDE90134BAF942
:10AB50004E300093BAF94C30DAF84020614D18A815
:10AB6000A847BDF860309AF850201E94013BADF81C
:10AB70007C30BDF862305C4D013BADF87E301EA9E3
:10AB80001AAB5846A847BAF84830BDF86820BAF85A
:10AB90004A101A44BDF8783013FA82F3ADF87830D1
:10ABA000BDF86A300B44BDF87A1011FA83F1ADF8A4
:10ABB0007A10BDF87C1011FA82F2ADF87C20BDF855
:10ABC0007E2012FA83F3ADF87E3025A8474B9847D4
:10ABD000DAF840302693BAF84C30ADF8A030BAF825
:10ABE0004E30ADF89E30BAF84630ADF894309AF851
:10ABF000443000948DF89C303D4CDAF83C3025AA66
:10AC000041461EA8A0479AF81C300593052B40F238
:10AC10006B81BAF91830002B00F06681059B354D29
:10AC2000FB2B28BFFF230593334B984759460B90C6
:10AC300012A8A847BAF81A70BDF84890BDF84C4061
:10AC4000A9EB0703ADF84830BDF84A300793DB1B8A
:10AC5000ADF84A30BDF84E303B449BB23C440893BB
:10AC6000ADF84E30A4B2BAF900300C9312A9BAF97B
:10AC70001830ADF84C4014A80D93A847BAF81860E6
:10AC8000BDF8503009939B1BADF85030BDF85430DF
:10AC9000BDF8565033441FFA83FBBDF852300A9377
:10ACA00035449B1BADB2ADF85230ADF854B0134BE8
:10ACB000ADF856509847124B9847124B06904246B3
:10ACC00014A916A89847002800F00E811CE000BFC8
:10ACD0001599000011970000F1610000A197000094
:10ACE00069EB00009D01010031E1000045780000A2
:10ACF000757800008D9B0000F1970000E94F00007F
:10AD0000E1D900008DDE0000079BBDF85810C3F1AB
:10AD10000103C9F10109B9441F44089B04EB09026E
:10AD20003B4412B21BB29A42A8BF1A460C9B521067
:10AD30009A42A8BF1A46099BC3F1010333449B44BE
:10AD40000A9BC3F101031E4435440FFA8BFB2DB25D
:10AD5000AB450D9BC84EA8BFAB4613444FEA6B0BE7
:10AD60009B45D946A8BF9946069BBDF85C501B8AF7
:10AD7000C81AADF858000698EB1A448AADF85C3052
:10AD8000BDF85E30BDF85A0001351B1B6D1A001B63
:10AD9000ADF85E302BB208EE103AADF85A00012340
:10ADA00012A91EA8B047B54C00211EA8A0470FFA53
:10ADB00089F2002314A908EE900A25A8B0470021C3
:10ADC00025A8A047AE4B09EE100A18EE100A9847C6
:10ADD000BAF91830BDF95A600B9ABAF816709AF899
:10ADE0001DB0BDF954109945BCBF03F1FF33079363
:10ADF000069BA8BFCDF81C90B3F912C00CEB06035C
:10AE000004461BB2BDF95000002A40F03F87BDF94F
:10AE10005220079DADF86000A2EB0C022A44089274
:10AE2000ADF86410ADF86230ADF86630089BB342FF
:10AE300080F22486069BBDF95660B3F91230079A5A
:10AE4000F61AB61A089AB242A4BF1646013633441F
:10AE50001BB2ADF86230ADF86630BDF95E309E428F
:10AE600040F38D86BDF85230079A864D013313FAB0
:10AE700082F3ADF86230BDF85630013B9B1AADF855
:10AE80006630BDF95030BAF81820ADF86030013B9B
:10AE900013440126ADF86430059B01933A46002324
:10AEA00018A94046CDF808B00096A847BDF954202F
:10AEB000BAF81810ADF8642093195B1AADF8603039
:10AEC000059BCDF808B0CDE900633A46002318A9E8
:10AED0004046A8476C4D18EE900AA84719EE100A94
:10AEE000A8476A4B204698472DB0BDEC048BBDE8BF
:10AEF000F08F2946664B674C324618EE100A984789
:10AF0000BDF97A20BDF97810334618EE100AA04733
:10AF10009AF8293002930128089B5A4C08BF022056
:10AF2000CDE900031EA918EE103ABAF81E204046DB
:10AF3000A047BDF87A300133ADF87A30BDF87E30E5
:10AF400001331BB24D440137FFF72EBA2946504B4F
:10AF5000504C324618EE100A9847BDF97A20BDF9D8
:10AF60007810334618EE100AA0479AF82930029359
:10AF70000128089B434C08BF0220CDE900031EA90D
:10AF800018EE103ABAF81E204046A047BDF87A30B5
:10AF9000013BADF87A30BDF87E30013BADF87E3034
:10AFA0004D440137FFF755BA394B18EE100A2A46BF
:10AFB00031469847079B53B9BDF97A20BDF97810FF
:10AFC000344C18EE100A2B46A047012800D102206D
:10AFD0009AF8293002939AF828302A4CCDE90003D8
:10AFE0001EA918EE103ABAF81E204046A047BDF838
:10AFF0007A300133ADF87A30BDF87E3001331BB2C0
:10B000000137FFF76FBA3378089A02EA0301FF2984
:10B010001CBF12FB03F3C3F3072118EE100A1E4BEB
:10B020002A469847079B53B9BDF97A20BDF9781095
:10B03000184C18EE100A2B46A047012800D1022018
:10B040009AF829300293FF23CDE900030D4CBAF89A
:10B050001E2018EE103A1EA94046A047BDF87A30CF
:10B060000133ADF87A30BDF87E3001331BB24E4467
:10B070000137FFF780BA00BF159900001197000053
:10B08000B5EE0000F1610000A197000069EB00003F
:10B0900031EC000061970000B9EF00003378089AA6
:10B0A00002EA0301FF291CBF12FB03F3C3F30721CC
:10B0B00018EE100AB54B2A469847079B53B9BDF9BD
:10B0C0007A20BDF97810B24C18EE100A2B46A04732
:10B0D000012800D102209AF829300293FF23CDE9FC
:10B0E0000003AC4CBAF81E2018EE103A1EA94046D8
:10B0F000A047BDF87A30013BADF87A30BDF87E301C
:10B10000013BADF87E304E440137FFF781BA9AF823
:10B1100028109F4C18EE100A3246C847BDF97A2015
:10B12000BDF97810334618EE100AA0479AF8293076
:10B130000293012808BF0220FF23CDE90003954CAC
:10B14000BAF81E2018EE103A1EA94046A047BDF8D6
:10B150007A300133ADF87A30BDF87E3001331BB25E
:10B160000135FFF793BA0023FFF713BB002C40F320
:10B17000B0800023224616A925A8874FB847874BE1
:10B18000002125A898470B90BAF8023008EE103A33
:10B190009AF80630022B40F0A980BAF80420BAF8D9
:10B1A00002309A4200F0A2807D4B70009847002741
:10B1B0000690BE427B4B00F39080BDF95C20BDF948
:10B1C0005810ADF86C20531C5B1A1BB2A3EB440360
:10B1D0000A93059BBDF962205B8AADF868101344A1
:10B1E0001BB2ADF86A300792079AADF86E30BDF920
:10B1F00066309A427DDD9AF806300C9A1A4312F0B6
:10B20000FF035DD10A9A322A5ADDBDF8582012FA9E
:10B2100084F2ADF86820BDF85C20A6B2921BADF8B0
:10B220006C20BDF95A20ADF86A203244ADF86E208A
:10B230009AF80D20574CCDE9019201220092BAF8FC
:10B2400002201AA94046A047BDF95E10BDF96E3034
:10B25000504CADF86E108A1B12B29A42D8BF01331F
:10B26000ADF86A20D8BFADF86A309AF80D30CDE954
:10B27000019301270097BAF8022000231AA940463B
:10B28000A047BDF85830ADF86830BDF85C30ADF877
:10B290006C30BDF85A303B443344ADF86A30BDF8E9
:10B2A0005E30013B9B1BADF86E309AF80D30009775
:10B2B000CDE901931AA9BAF8022000234046A0471D
:10B2C000069B002B3FF498AA1846374B9847FFF788
:10B2D00093BA4FF0FF330B9356E73AB231465046DC
:10B2E0009847069B23F81700013762E7002306936F
:10B2F00063E7059BB3F91270079B1F44BDF95A30F1
:10B30000234401339F4208DDBDF95E301B1B013B26
:10B310009F4202DA089B002B36D118EE901A234B7D
:10B320001B4E28469847059B5A8A079B1A44059B43
:10B33000198ABDF86030194412B218EE903A09B279
:10B340002846B04706469AF806300993012B2FD1BC
:10B35000BAF80220BAF804309A420DD0BDF85E1057
:10B36000BDF85A300131FA1AC91A12B20D4B09B29E
:10B370005046984708EE100A089B002B00F0A38067
:10B380000A9B322B1CDC9EE00126DCE7B9EF0000B3
:10B3900061970000F161000015990000119700000D
:10B3A000B5EE00007199000069EB000075F0000037
:10B3B000089B002B00F0A2840A9B322B40F39E8452
:10B3C000BDF95A3023449F4204DDBDF95E301B1B9A
:10B3D0009F425ADBBDF95830ADF87830013B13FA83
:10B3E00084F3ADF87C30BDF86A30ADF87A30BDF842
:10B3F0006E30ADF87E309AF80D309E4F0096A2B2B6
:10B40000CDE9019309922B4618EE102A1EA9404659
:10B41000B8479AF80620012A15D10999BDF8583085
:10B420000B44ADF87830BDF85C305B1AADF87C3079
:10B430009AF80D300092CDE9019318EE102A0023FE
:10B440001EA94046B847BDF95C300999ADF87C307B
:10B450005A1C521AADF87820059ABDF96010B2F95D
:10B4600010201B1B0A4401339B1A9AF80D200096EA
:10B47000CDE9019218EE102A002BACBFEB182B1C63
:10B480001EA97C4E4046B0470DE0099B022B16D109
:10B490009AF80D30069A0096CDE90193764E2B4628
:10B4A0001AA94046B047BDF86A30079A0133ADF893
:10B4B0006A30BDF86E3001331BB2013293E6099B4E
:10B4C000012B40F01F849AF80D300096CDE90193CE
:10B4D00018EE102A2B461AA9D3E7BDF89630259D01
:10B4E000C3F34A171AA8654B98479AF836308DF877
:10B4F00068309AF837308DF87230BAF83430ADF8D9
:10B500007430C5F38A25BBB203F1FF3905939AF86D
:10B510003830BAF90020DB071FFA89F940F1C680FC
:10B52000574C0023594625A8A047564B002125A873
:10B530009847BBF80440BBF80030BBF80620013444
:10B54000E41A24B294FBF5F305FB1344BBF8023074
:10B550000132D21A12B292FBF7F107FB112202EB71
:10B56000D272A3EB62039BB204EBD47408EE100A10
:10B57000ADF8623064104B441BB2BDF96220ADF8E7
:10B580006630BBF906309A423ADD18EE100A3E4B9F
:10B590009847FFF755B9022821D13C4B3C4C1EA8D7
:10B5A0009847BAF83430ADF878309AF836308DF8DC
:10B5B0008030002147F61843DAF830201F92CDE999
:10B5C0000131BDF982300093DAF82C10BDF98430D6
:10B5D00025A8A047BDF99450BDF9967093E72D4B6F
:10B5E00000932D492D4B2E4C40F2AE520220A04725
:10B5F00000232C4C1A4641465846A047FFF720B975
:10B60000BBF800301FFA85F91B1B9BB209F1FF3212
:10B61000ADF8603013441BB2BDF96020ADF8643062
:10B62000BBF904309A4209DDBDF86230059A134433
:10B63000ADF86230BDF8663013449DE7022EDAF8AB
:10B640002C2010D100230093174F134641461EAA09
:10B6500018A8B847BDF860304B44ADF86030BDF86D
:10B6600064304B44D7E70F4F1AAB414618A8B84790
:10B67000F0E700BFF1610000FD67000059750000B0
:10B680001599000011970000A1970000457800006F
:10B690009D010100C3FD01006FFD0100F2FD0100ED
:10B6A000E9E80000C175000075780000BBF80410DF
:10B6B000BBF80040BBF80630BBF802000131091BA3
:10B6C00001331B1A09B2491B1BB201EBD171DB1B01
:10B6D00004EB610403EBD37100EB610080B2A4B210
:10B6E000013D8144ADF860401FFA89F92C44022ED7
:10B6F000ADF86200ADF86440ADF8669007D103F094
:10B70000010318449944ADF86200ADF86690944B7B
:10B71000594618A898470446C8B90346BAF9002004
:10B72000904D594625A8A84721468F4B25A89847F4
:10B730000446022EDAF82C200CD1002300938B4D06
:10B74000134641461EAA18A8A84720461FE74FF0F7
:10B75000FF34EEE7864D1AAB414618A8A847F4E738
:10B760000023FFF7BAB84FF0FF330C93FFF7DCB8B4
:10B77000804B814F494620469847069B5A8A198A32
:10B78000BDF850303244194412B24B4609B220463B
:10B79000B847BDF86230ADF86A30BDF86630ADF834
:10B7A0006E30BBF90030ADF86830013B2B44ADF88A
:10B7B0006C30079B0293059B0B9018EE102A0193A7
:10B7C000009023461AA96D4F4046B847BBF9023096
:10B7D000BAF91010BDF96E200B449A4215DABBF885
:10B7E00000302B44ADF86830BBF804305B1BADF87B
:10B7F0006C30079B0293059B01930123009318EE85
:10B80000102A00231AA94046B847BBF90430ADF806
:10B810006C305A1C521BADF86820099ABDF95010C3
:10B82000564F9B1A069AB2F9102001330A449B1A0C
:10B83000079A0292059A01920B9A0092002BACBFD4
:10B84000E318231C18EE102A1AA94046B847BDF881
:10B8500062300133ADF86230BDF866300133ADF8C7
:10B8600066300136FFF702B9424B434F4946204646
:10B870009847069B5A8A198ABDF8503032441944B9
:10B8800012B24B4609B22046B847BBF90030ADF8BA
:10B890006830013B2B44ADF86C30BDF86230ADF838
:10B8A0006A30BDF86630ADF86E30079B0293059B99
:10B8B0000A9018EE102A0193009023461AA92F4FE0
:10B8C0004046B847BBF90630BAF91010BDF96E20F2
:10B8D0005B1A9A4215DDBBF800302B44ADF8683096
:10B8E000BBF804305B1BADF86C30079B0293059BE3
:10B8F00001930123009318EE102A00231AA9404651
:10B90000B847BBF90430ADF86C305A1C521BADF887
:10B910006820099ABDF95010184F9B1A069AB2F97F
:10B92000102001330A449B1A079A0292059A019249
:10B930000A9A0092002BACBFE318231C18EE102AC1
:10B940001AA94046B847BDF862300133ADF86230FD
:10B95000BDF866300133ADF866300136FFF7A2B8A6
:10B9600091E0000015990000119700007578000023
:10B97000C175000075F0000061970000F1610000E2
:10B98000ADF86230ADF86630BAF91230ADF860103B
:10B99000042BADF864205ED1089A1144ADF8641010
:10B9A0000022022B8DF83E208DF83F205AD1012332
:10B9B0008DF83E309DF83E30002B5DD19DF83F3034
:10B9C00083F0010303F00103AD4D8DF84030BDF964
:10B9D00056309E423FF7A5A89DF840309BB99DF890
:10B9E0003E30BDF962202BB1BBF9023008990B44FF
:10B9F0009A4208DD9DF83F300BB3BBF90630089939
:10BA00005B1A9A421BDB9F4B9F4F49462046984743
:10BA1000069B5A8A198ABDF850303244194412B232
:10BA20004B4609B22046B847079B0293059B18EE88
:10BA3000102ACDE9000318A923464046A847BDF8BF
:10BA400062300133ADF86230BDF866300133ADF8D5
:10BA500066300136BBE7082B02BF0899521AADF8D1
:10BA600060209DE7012B04D0032BA3D101238DF887
:10BA70003E308DF83F309DE70023A3E718EE101A03
:10BA8000804B814D20469847069B5A8A198ABDF8FB
:10BA900058303244194412B218EE103A09B2204616
:10BAA000A847BDF86230ADF86A30BDF86630ADF831
:10BAB0006E30BDF95030ADF86830013B13FA89F3B0
:10BAC0001FFA89F2ADF86C30059B0A900992019338
:10BAD000009023463A461AA9694DCDF808B0404671
:10BAE000A847BDF95230BAF91810BDF96E200B44C1
:10BAF0009A4215DA099ABDF85030CDF808B01344CF
:10BB0000ADF86830BDF854309B1AADF86C30059B29
:10BB10000193012300933A4600231AA94046A847FF
:10BB2000BDF954300999ADF86C305A1C521AADF871
:10BB30006820069ABDF95810B2F91020504DCDF882
:10BB400008B0A3EB09030A4401339B1A059A01923A
:10BB50000A9A0092002BACBFE318231C3A461AA99C
:10BB60004046A847BDF862300133ADF86230BDF8F9
:10BB700066300133ADF866300136FFF757B918EE7D
:10BB8000101A404B404D20469847069B5A8A198A06
:10BB9000BDF858303244194412B218EE103A09B2C6
:10BBA0002046A847BDF95030ADF86830013B13FA84
:10BBB00089F3ADF86C30BDF86230ADF86A30BDF88D
:10BBC0006630ADF86E301FFA89F2059B0990089235
:10BBD0000193009023463A461AA9294DCDF808B0A2
:10BBE0004046A847BDF95630BAF91810BDF96E2085
:10BBF0005B1A9A4215DD089ABDF85030CDF808B0AE
:10BC00001344ADF86830BDF854309B1AADF86C3071
:10BC1000059B0193012300933A4600231AA940464D
:10BC2000A847BDF954300899ADF86C305A1C521A27
:10BC3000ADF86820069ABDF95810B2F91020104DE1
:10BC4000CDF808B0A3EB09030A4401339B1A059A07
:10BC50000192099A0092002BACBFE318231C3A46CC
:10BC60001AA94046A847BDF862300133ADF86230EA
:10BC7000BDF866300133ADF866300136FFF7EDB838
:10BC8000F161000075F0000061970000DFF88C9012
:10BC9000DFF88CA0ADF86000ADF86410ADF862304C
:10BCA000ADF86630BDF95E309E423FF713A918EE3D
:10BCB000101A2046C847069B174D5A8A198ABDF8A4
:10BCC00058303244194412B218EE103A09B22046E4
:10BCD000A847059BCDF808B0CDE900033A462346B6
:10BCE00018A94046D047BDF862300133ADF8623044
:10BCF000BDF8663001331BB20136D1E7099B022B38
:10BD00003FF4C6AB0D9B002B7FF4DDAB0A9B322BBF
:10BD10003FF7C9ABFFF7D7BB6197000075F0000094
:10BD2000F1610000F0B5C1F34513C2F1FF06C0F3A5
:10BD30004514734304FB023301F01F0400F01F0796
:10BD4000744348F2810507FB02446B436C43C3F321
:10BD5000C553C4F3C45444EA4314C1F3C423734326
:10BD6000C0F3C42000FB023205FB02F3DB0D44EA02
:10BD7000C320F0BD01390244904200D1704711F850
:10BD8000013F00F8013BF7E7F7B586680746007802
:10BD900015460022ADF8042000F01F02042A0C46CC
:10BDA00009D0053A092A1AD8DFE802F005051D3244
:10BDB00043582F2F2F2F2E4B00F01F0098473B6822
:10BDC000C0F3C700C3F38A2313FB05F310FB04F190
:10BDD00000FB03110222274B314401A89847BDF80C
:10BDE000040003B0F0BD3B68C3F38A230733DB10C4
:10BDF00005FB036303EBE40304F007021B7AC2F1C3
:10BE00000702012191400B401341ADF80430E6E7F1
:10BE10003B68C3F38A2303339B1005FB036304F0E1
:10BE2000030203EBA40352001B7CC2F106020321B0
:10BE3000E8E73B68C3F38A2301335B1005FB036229
:10BE400002EB640204F00101890092F84030C1F174
:10BE500004010F228A4013400B41D6E73B68C3F32D
:10BE60008A2315FB03452E4496F80034CDE700BF26
:10BE70008175000075BD0000F0B50B46017885683E
:10BE800001F01F01052985B004460AD10168C1F3FC
:10BE90008A2112FB013202EB42022A44907805B05B
:10BEA000F0BD0B39032956D8DFE801F00219324EF4
:10BEB0002168C1F38A210731C91003F0070002FB92
:10BEC0000152DB10C0F10700D35C01228240134015
:10BED00003410CBF4FF0FF300020C0B2DFE71F4925
:10BEE00000912168C1F38A210331891003F0030016
:10BEF00002FB01529B104000D35CC0F106000322FC
:10BF000082401340034110336B4413F8100CC6E712
:10BF1000134EEC4606F1100E30687168674603C791
:10BF200008367645BC46F7D12168C1F38A21013134
:10BF3000491003F0010002FB01525B108000D35C4A
:10BF4000C0F104000F22DBE72168C1F38A2112FB54
:10BF50000132A85CA3E7FF20A1E700BF0055AAFFBC
:10BF6000FFFD01002DE9F84FB0F90830DFF8EC8053
:10BF70001B024362B0F90A301B020A268362B0F941
:10BF80000C3093FBF6F51FFA85F90446C9F1000061
:10BF90004FF6F67700B215FB0737C0470135ADB253
:10BFA0008246684200B2C0478346C9F15A0000B2D7
:10BFB000C047C5F15A05814628B2C047F21B07FBAE
:10BFC0000BF302FB0A3393FBF6F3E36207FB00F388
:10BFD00002FB09301F4B90FBF6F02063A07C9847D2
:10BFE00094F8343060F3000384F83430A07C1A4BAA
:10BFF0009847A37C191F02298CBF00210121420010
:10C0000042EA810294F8341002F0060221F006019F
:10C010000A4384F8342022682262A28803F01F03B6
:10C02000C2F30A0243EA8223B4F9062043EA4253E8
:10C03000A26902F440721343A361E2894FF4803392
:10C04000B3FBF2F3E386FF23A375238AA382BDE843
:10C05000F88F00BF99750000AD7500003DE9000044
:10C060002DE9F04F85B00746DFF874B1BDF8388090
:10C0700002910A264FF6F67A93FBF6F9484619FB29
:10C080000A3A1446D84709F10105039028B2D84767
:10C09000054609F15A0000B2D847019009F15B004A
:10C0A00000B2D847019B0399A6EB0A0C0AFB00F0EB
:10C0B0000CFB03000F9B90FBF6F00AFB05F5B3F9B0
:10C0C00000E00CFB0155B3F902C095FBF6F5CEF18B
:10C0D0000003CCF1000208FB03F308FB02F243F378
:10C0E0000F2342F30F2200FB03F905FB02FA6B4317
:10C0F00042439918C91311FA8CF109B201910299BE
:10C10000A1EB0E0108FB01F141F30F21A4EB0C049C
:10C1100000FB01FB08FB04F4A9EB0A0644F30F241F
:10C12000ABEB0A0A6943F61365434FEAEA3A444324
:10C1300016FA8EF61AFA8EFAA9EB050936B20FFA3C
:10C140008AFA0A44234421444FEAE939564519FA48
:10C150008EF9ABEB050B4FEAE1314FEAE2324FEAE1
:10C16000E3330FFA89F912FA8CF213FA8CF34FEADF
:10C17000EB3B11FA8CFC3146A8BF514649451BFAEE
:10C180008EFE0FFA8EFEA8BF49467145A8BF7146C4
:10C190005645B8BF56464E45B8BF4E463980019900
:10C1A00012B27645B8BF764691421BB2A8BF11467F
:10C1B00099420FFA8CFCA8BF19466145A8BF614699
:10C1C00079800199BE808A42B8BF0A469342B8BFBF
:10C1D00013466345B8BF6346FB8005B0BDE8F08FEA
:10C1E0003DE900002DE9F04F90F83820D0F80080AC
:10C1F000B0F93850B0F93A6090F83A306F2A89B007
:10C20000044600F29280B0F93C90B9F1000FD4BF1F
:10C210004FF000094FF00109C9F10009803DEDB26E
:10C220006F2B00F29780B4F93E70002FD4BF002727
:10C2300001277F42803EF6B2A38AADF80A30A37D83
:10C24000019394F83430580740F1A98094F84430B1
:10C25000216CDFF848A209FB03110222414405A822
:10C26000D047A28894F84430216C13FB02F307FBFB
:10C2700003110222414406A8D04794F84420A38821
:10C28000216C13FB02F309FB021107FB031141446C
:10C29000022207A8D04794F8343099076BD40020C5
:10C2A0000746834694F834309B0740F1C780019AD3
:10C2B000C5F1FF0312FB05F103FB0B114343C1F36F
:10C2C000072115FB0733C3F30723C6F1FF0C06FB59
:10C2D00001F203FB0C2212120529A27500F2AA80BA
:10C2E000052B40F2D4800026019B052B94BF002231
:10C2F0002A46BBF1050F98BFFF22052F98BF0025E6
:10C30000052898BFFF25002A40F09C80BDF81470D6
:10C31000002D40F0A480BDF81C10002E40F0AD8030
:10C32000A182012009B0BDE8F08F902A0ED9B0F9A2
:10C330003C90B0F9042009F101099145ACBF4FF0E0
:10C3400000094FF00109C5F17F0568E7FF254FF0AF
:10C35000000965E7902B0BD9B4F93E70B4F90630AB
:10C3600001379F42ACBF00270127C6F17F0662E775
:10C37000FF26002760E7226C94F84410A388013A56
:10C380000A4409FB012913FB01F37B4308EB03017A
:10C3900018F809B08F5CC84418F8030082E7A38F2F
:10C3A000DFF8FCB0B4F93E2004F1180A13FA89F161
:10C3B00009B2238A5046D847E38FB4F93C10ADF850
:10C3C000140013FA87F212B2238A5046D847E28F3C
:10C3D000A18F238AADF818001FFA89F81FFA87F990
:10C3E0004A44414412B209B25046D84794F8343016
:10C3F000ADF81C009A077FF552AFB4F93C70B4F960
:10C400003E20244B0392B8440FFA88F84146504628
:10C410009847039A1F4B91440FFA89F23946834695
:10C42000504603929847039A1A4B07464146504696
:10C43000984737E7052B98BFFF2655E7FF23A375DD
:10C440002A4660E7FF2A02D1BDF80A7060E7BDF80E
:10C450001410BDF80A00104B9847074658E7FF2D07
:10C4600002D1BDF8181058E7BDF81C10BDF818002F
:10C47000094B2A46984701464FE7FF2E01D1A78274
:10C480004FE7054B324638469847A08249E70020DF
:10C4900048E700BF79BE000025BD000075BD000063
:10C4A00089BD00002DE9F74FDFF89081B8F8004012
:10C4B00005460E465CB9524B00935249524B534DC0
:10C4C00044220220A847204603B0BDE8F08F504B1D
:10C4D00050481F6800233A46116A01338142A8BFC1
:10C4E00001F1FF319BB2A8BF11629C4202F124020C
:10C4F000F2D1DFF84CB14FF0000A4FF02409B8F840
:10C5000000101FFA8AF2914239D807F124023C4602
:10C510000123994256D86368DFF8F080002B5AD087
:10C520003D4B204698473D4B0093374B772235498A
:10C530000120C0473A4B98474FF000092946394B34
:10C54000C4F814900746324620469847054600280E
:10C5500046D1354B2B49009383222B4B334E02207F
:10C56000C0472D4B2046984720462021B047204603
:10C570002421B0474FF0004323622C46A3E71FFA63
:10C580008AF409FB04742A4B6068984780B9626892
:10C59000AA4214D12189B2B2914210D1236A6269B0
:10C5A0001344B3F57A7FA8BF4FF47A7323628AE706
:10C5B000012804D160682946D8470028EED00AF146
:10C5C000010A9CE7176A206A01338742B8BF144604
:10C5D0009BB224329DE7174B00937A220A4BA6E7C1
:10C5E0006369C4F82090002B7FF46DAF124B38467E
:10C5F000984708B1606166E70123636163E700BFA4
:10C600005BFE010026FE01000EFF0100E9E80000CC
:10C610006C860020020000804DD0000082FE0100E8
:10C6200049DA00007DCF0000E4FE010019F00000AF
:10C6300005780000B3FE01005DDA0000D08500201F
:10C6400015630100144B2DE9F7431F68134E144D79
:10C65000DFF8508004464FF0000932881FFA89F352
:10C660009A4202D803B0BDE8F0831FFA89F324226E
:10C6700002FB03704368A34200D04CB913B1019090
:10C68000C047019801902021A84701982421A8477C
:10C6900009F10109E1E700BF6C860020D085002088
:10C6A00019F000004DD000002DE9F7431F4C23681E
:10C6B00005462BB11E4B0020984720681D4B98471C
:10C6C00024271D4B07FB05F098471C4B206098471B
:10C6D000064660B91A4B1B490093A82203201A4D45
:10C6E000A847226819481A4933468847FEE7236855
:10C6F000DFF8608023B9A8F8003003B0BDE8F0830C
:10C70000DFF85490A8F800500025B8F80020ABB22C
:10C710009A42F2D92068AEB27E4320213044C84705
:10C72000206824213044C8470135EEE76C8600209C
:10C7300045C60000E5EA00002DEA0000E117000010
:10C7400021FF010026FE0100E9E80000BEED010026
:10C75000E9170000D085002019F0000070B52C4BBF
:10C7600086B008460E46154698470446D8B9337831
:10C77000C3F30403043BDBB20A2B11D873886A8825
:10C780003168C3F34A1363F34F126A802B68214A5E
:10C7900023F01F1323F47C430A4013432B6001242E
:10C7A000204606B070BD012825D11B4B0222314620
:10C7B00004A89847B8B9194E03AB0422294604A827
:10C7C000B047174B064604A8984716B9039B042B9D
:10C7D00009D0144B0093144B40F221121349144C0E
:10C7E0000220A04705E02B781C3303F01F030A2B1F
:10C7F000D6D90024D4E7022804D12B6803F4787238
:10C800000C4BCAE70C4B00934FF49A72064BE5E7CA
:10C81000057800001FFC1F00A1E4000019E40000DF
:10C82000E9E300006EFF0100DC00020037FF0100B9
:10C83000E9E800000B04200092FF010070B5CC690C
:10C840000D4684B12068084E18B1084B98472068FF
:10C85000B047606800B1B047A06800B1B04720465B
:10C86000B0470023EB6170BDE5EA0000E9E300009A
:10C870002DE9F04F087B8DB0984600F01E03042B85
:10C88000BDF958A0179E0D46144603D000F01F03B3
:10C89000062B3ED195F80A90B9F1010F36D1AF4B76
:10C8A000D5F81CB000F01F009847E968AC4BC1F305
:10C8B0008A2118FB01414143C91007460431DBF8C6
:10C8C0000000984748B1A74B0093A74B40F22E2297
:10C8D000A649A74C0220A04718E0C7F3C70717FBDB
:10C8E0000AF7089008ABDBF80000A24D3A46314643
:10C8F000A847089B9F4200F0DB809F4B00939B4919
:10C90000994B9B4D40F235220220A8474FF0000979
:10C91000CEE0A3F10B02032A00F2CE804FF47F4356
:10C92000ADF81830A3F5AD03A3F528530793934B47
:10C9300008AA03F1100E1746186859689446ACE827
:10C940000300083373456246F6D1298933464FEA1E
:10C95000112C002210B2824503F1030314DC287B62
:10C960007E4B00F01F00984701238340013B9BB2A0
:10C9700004932B7B03F01F030B3B8146032B5FD8F3
:10C98000DFE803F0082E425503F8031C03F802CC3D
:10C990000132DFE7EB68C3F3473213F4E05F4FEA9D
:10C9A000E4010CBF0FFA82FB02F1010BE4430BFB25
:10C9B000081104F0070406AFEB6903935846704B67
:10C9C00005919847AB7A05998046002B3CD16B685E
:10C9D0009A680A44C9F108000021023640B25FE0BB
:10C9E000EB68A110C3F3083213F4406F6FEA04043C
:10C9F0000CBF0FFA82FB02F1010B04F003040BFBE6
:10CA00000811640007AFD7E7EB685905C3F3C922E3
:10CA10004FEA64016FEA040454BF0FFA82FB02F18B
:10CA2000010B04F001040BFB0811A400C4E7EA6841
:10CA3000C2F38A218B4618FB014100242746BBE73D
:10CA400000242146A346F9E7039B04311868444BB0
:10CA5000984703985A460068DFF818B1002341460A
:10CA6000D8474246B6E7049B92F800E003FA04FC7C
:10CA70000EEA0C0395F80CC023410CF01F0CBCF11E
:10CA80000E0FA4EB090401EB410C14BFFB5CDBB2FD
:10CA900064B2002C06F80C30BCBF044601320131F0
:10CAA0000BB29A45DFDC374B404698474FF00109FF
:10CAB00048460DB0BDE8F08F073B032B00F2B08075
:10CAC000264B00F01F00984701278740013FBBB26B
:10CAD00003932B7B03F01F03073B8146032B70D886
:10CAE000DFE803F002275265EB68C3F3473213F423
:10CAF000E05F08BF17B24FEAE40318BF571C07FBFB
:10CB00000833E44303F1080104F007041C4B0491CB
:10CB10003846D5F81CB09847AB7A04998046002B6C
:10CB200053D16B689B680B44C9F1080500206DB2B6
:10CB300072E0EB68C3F3083213F4406F08BF17B21A
:10CB40004FEAA40318BF571CE44307FB083304F063
:10CB5000030403F110016400D8E700BF81750000F1
:10CB60004FE40000B8FF0100F900020037FF0100A8
:10CB7000E9E8000019E40000DBFF010021010200E8
:10CB8000B5EE000069EB0000EB68C3F3C9225B055A
:10CB900058BF17B24FEA640348BF571CE44307FB72
:10CBA000083304F0010403F14001A400AEE7EF688C
:10CBB000C7F38A2318FB03481F4608F58061002449
:10CBC000A4E700210C460F46A0E7184BDBF8000055
:10CBD000174D043198470023DBF800003A464146E0
:10CBE000A8474346A0E703991A78A1400A4022418A
:10CBF000DBF8041031F812103170090A7170DBF89B
:10CC00000810A4EB090464B2002C8A5CB270BCBFAB
:10CC10002C4601330130033602B29245E3DC42E791
:10CC2000044B00934FF4FE72034B51E64FE40000B7
:10CC300019E40000FEFF0100310102002DE9FF4769
:10CC40000646887A01280C4678D148688B4B98476D
:10CC50008B498C4B9847002840F0A98061688A4B2B
:10CC6000022202A8984738B1884B0093884B4FF4B2
:10CC7000A6728849022022E0E369DFF83C92DFF8DF
:10CC80003C8213BB0C20C847E061C047054668B929
:10CC90007F4B8049009340F2531203207E4EB047F1
:10CCA000E2697E487E492B468847FEE7E06948B93D
:10CCB0007C4B00937749764B40F255120320764C1B
:10CCC000A04774E0784B0C2198470820E769C847D3
:10CCD0003860C047054668B96D4B6E49009340F215
:10CCE0005D1203206C4CA0473A686C486C492B4697
:10CCF0008847FEE73B684BB96A4B0093644B40F2B0
:10CD00005F126449644D0320A8474CE002AA03F176
:10CD1000080112F8010B03F8010B8B42F9D1237BB8
:10CD200003F01F00021F022A11D8A37A002B40F043
:10CD3000888063689B682361012005E00028EED1AC
:10CD40004A689268002AEAD104B0BDE8F087C21FA1
:10CD5000032A00F2D480554BDFF85CA1DFF85C9128
:10CD60009847E369804643BB0C20D047E061C84741
:10CD7000054668B9464B474900934FF4C6720320F5
:10CD8000454EB047E269454845492B468847FEE78E
:10CD9000E56975B9434B00933E493D4B3E4F4FF417
:10CDA000C7720320B847424B2146304698470020BF
:10CDB000CAE73D4B0C2128469847022000FA08F0AC
:10CDC000E569D0476860C847074668B9304B3149C4
:10CDD000009340F2971203202F4CA0476A682F4817
:10CDE0002F493B468847FEE7012707FA08F73846F0
:10CDF000D047A860C847804668B9254B25490093AD
:10CE000040F299120320244CA047AA6823482449E1
:10CE100043468847FEE76B680BB1AB682BB9214BE3
:10CE2000009340F29B121A4B6BE7A37A012B49D176
:10CE30002868204BDFF88880042198470026BE42EE
:10CE400001D1002377E70023042202A92868C04704
:10CE50009DF809109DF808306A688908DB0843EAE4
:10CE600041139DF80A10C90843EAC12322F816307D
:10CE7000AB689DF80B209A550136E0E76DE50000A0
:10CE80003800020015630100A1E400003C0002002C
:10CE90005301020037FF0100E9E80000BEED010088
:10CEA000E91700006700020019F00000817500001A
:10CEB0003DC800004FE400002DEA0000E11700002B
:10CEC00019E40000636899680020B84201F1040188
:10CED000B7D011F8036C11F8043C6A68B608DB0897
:10CEE00043EA461311F8026CF60843EAC62322F817
:10CEF0001030AB6811F8012C1A540130E5E7A0F1AD
:10CF00000B03032B9DD9054B214630469847044B14
:10CF1000009340F2D312034BABE600BF3DC80000C4
:10CF200090000200530102002DE9F8430B78DFF86E
:10CF30004480DFF844906FF347130B7007460C4BA7
:10CF40000C480E4698470024054615B92046BDE812
:10CF5000F8832C6834B1324639462846A047012868
:10CF60000446F3D029464046C8470546EDE700BFD2
:10CF7000A9E6000054860020B5E600002DE9F04740
:10CF8000224B0281044608460F4698470023012899
:10CF9000A072E3611DD11E4B384698471D4B0130EE
:10CFA00098471D4B6060394698471C481C4BDFF87A
:10CFB0006C90DFF874A098470026054604F10C0831
:10CFC0004DB91EB9174B2021204698473046BDE881
:10CFD000F0876760E9E72B689BB16A688AB14246CF
:10CFE000394628469847012806460AD10023A361FE
:10CFF000236125606B68214628469847012806462C
:10D00000E4D029464846D0470546D9E705780000D0
:10D01000396301002DEA00002963010054860020D5
:10D02000A9E6000019F00000B5E6000073B5056838
:10D03000AC684CB1069ECDE9003613460A4601465F
:10D040002846A04702B070BD2046FBE710B5044655
:10D05000006858B1C3680BB121469847A37A012BE9
:10D0600004D1034B606898470023636010BD00BF84
:10D07000E5EA000073B50E4B0E4898470E4B044688
:10D080009847054660B90D4B0D490093C92203200E
:10D090000C4EB0470C480D4922462B468847FEE708
:10D0A0001CB10B4B102120469847204602B070BDA2
:10D0B00019E6000054860020E1170000700102000C
:10D0C00037FF0100E9E80000BEED0100E9170000AC
:10D0D00019F0000037B5154B154810219847154B2E
:10D0E00098470446B8B9144A009202204722134BCD
:10D0F0001349144DA847144A2046904798B90F4B3E
:10D100000F49009348220320A847104810490022E5
:10D1100000238847FEE70F4B03600F4B43600F4B24
:10D1200083600F4BC36003B030BD00BF05E6000055
:10D130005486002075D00000B9000200860102006C
:10D1400037FF0100E9E80000E1170000BEED010033
:10D15000E91700005DC700003DCC000071C8000069
:10D160003DC800004368184710B40468A4465DF841
:10D17000044B60471FB51346044C0A4601A9A0475B
:10D1800008B1BDF8040004B010BD00BF69D10000B3
:10D1900003780A78934209BF4B78981A4078C01AEE
:10D1A000704703880A88934209BF4B88981A4088C1
:10D1B000C01A7047531E30B5072B1FD8DFE803F0A5
:10D1C0002304181A1E1E1E1C0323CD0801F007019C
:10D1D0000A44072A445D18D92844C2F11002417854
:10D1E00001EB042189B241FA02F203EA020030BDE8
:10D1F0000723EAE70F23E8E7FF23E6E7012393404D
:10D20000013BDBB2E1E71346DFE7C2F1080214415C
:10D2100003EA0400EBE70000032B30B504D1072A32
:10D220009CBF0B4B9A5C042301F007054FF0FF34C1
:10D23000C1F3CF01C5F10805ED1A04FA03F363F059
:10D24000FF03445CAB402340AA401A43425430BD24
:10D25000D30102002DE9F74F394CDFF8E8A0D4F8EC
:10D26000009027794318804600934FF0020B009BF3
:10D27000434502D103B0BDE8F08F6379A3B9A66836
:10D2800001933A4631464846D047054636B1227B9F
:10D29000019B824202BF6373012363713E44257385
:10D2A000A66008F8015BE2E7012B31D1A6681A46B7
:10D2B00031464846D047637B0133DBB2711C0128FD
:10D2C0006373A16018D10B2B257BEAD10622484657
:10D2D000D04707366073A66010B184F805B0E0E768
:10D2E000019031463A464846D0473E44019B207360
:10D2F0000546A6606371D4E73A4648460191D04797
:10D300000199207339440546A1604FF00003F1E70D
:10D31000022B12D1667B257B013EF6B26673002E8E
:10D32000BFD1A16801913A464846D0470199207380
:10D3300039440546A1606671B3E70025B1E700BF37
:10D34000D4850020B5D1000000880B88C01A704732
:10D35000F0B50C4685B021B10569AB69994246D15B
:10D36000EC69204605B0F0BDAA6800FB03F69119F0
:10D3700092598F88A21ABA42039203F1010338D856
:10D380008B7C13B9CB88134410E0012B03D1CB68FD
:10D390009B5CCA88F7E7022B14D11B480A8A0090CD
:10D3A00089681A4F03A8B84720B90023C5E9064386
:10D3B0001C46D6E7AB6833449A68DB88801A03EBD7
:10D3C0005003F3E7032BF0D10F4B0A8A00938968CF
:10D3D0000E4F022303A8B8470028E6D0AA683244BB
:10D3E0009368C01A4008D368D2881B5CCBE700233F
:10D3F00014206A8A99B2C2F309028A42B4D8AC6195
:10D400000024EC61ADE700BF49D300008D020100AC
:10D410002DE9F04F2DED028B0929684B05698BB082
:10D4200008BF20219847074628B900200BB0BDEC63
:10D43000028BBDE8F08F2B7DD5F804909B0709EB9C
:10D44000C00809D1B8F1000FEFD059F83030286882
:10D45000C3F313031844E9E798F8044098F805303B
:10D4600014FB03F4002CE0D0EB7CC3F38303013BFB
:10D47000032B05D8DFE803F0025053530734E408C8
:10D480004F4E504B30699847A0424BD359F8372044
:10D490002B68ED7C98F80470C2F3130213443269D0
:10D4A000336008EE102A98F805200792C5F383022E
:10D4B000032A4FF0000B1146327108BF042186F891
:10D4C00005B0C6F808B086F80CB086F80DB038463E
:10D4D0003D4E03920491B04704463846B0473B4B5B
:10D4E0000646394620469847B946A04607EB040A47
:10D4F000D04531D1049B17FB03F306939A464FF0B6
:10D500000108079B434532DC2046314CA04730469A
:10D51000A0472B4B186989E70334A408B0E701340E
:10D520006408ADE721462B4B306998472A4B3061A0
:10D530009847044660B9294B294900937222032079
:10D54000284DA84732692848284923468847FEE7DE
:10D550003369002B9AD168E7039B18F8012B244DFF
:10D56000594618EE100AA847049B9B44C0E7174B86
:10D57000494630469847631E0593F319B34608930E
:10D580005146089B9B4506D1069B08F101089A4429
:10D590000FFA88F8B5E705981BF8012B10F8013F42
:10D5A00005905A400270039B114D099118EE100A24
:10D5B000A847049B09991944E3E700BF51D3000031
:10D5C000D48500204DEB0000B5EE000055D20000E0
:10D5D00069EB000015EE0000E1170000DB0102001E
:10D5E0009B010200E9E80000BEED0100E917000020
:10D5F00019D20000092A2DE9FF47DFF83CA107698D
:10D600000C46114608BF2021804699460CBF0126D2
:10D610000026D0470546002800F08680FB683BBB0B
:10D62000002379683A8A01EBC50153434A88C2F363
:10D630000B101B1102460EB102B252000833134404
:10D640001B0923804B79A3800B79638091F9062015
:10D65000E28091F907202281FA7CC2F38302A27250
:10D66000002E63D05B006380304604B0BDE8F087D5
:10D6700049464046D0470028D2D0D8F81020D2F8EA
:10D680000C80D27C53063AD498F80B2012F0030297
:10D690001BD1D8F80090D8F80820DFF8A0A005EB3F
:10D6A0000023ADF80C30224B009322F07F4202237E
:10D6B000494603A8D04703460028B2D0A0EB09038F
:10D6C0005B08D8F80420D356ABE7012AA8D1D8F8D4
:10D6D0000090D8F80820174B009305EB002003902A
:10D6E0000423DFF858A022F07F42494603A8D04720
:10D6F0000346002895D0A0EB09031B09E1E7D8F801
:10D700000420D8F80810525D095C002A88D000294E
:10D7100086D0D8F8003098F80D00013A0B4400FB91
:10D72000023313F9013C7CE706469DE701269BE79F
:10D7300091D10000A3D1000051D300008D0201005F
:10D7400010B5044C206918B1034B9847002323619E
:10D7500010BD00BFD4850020E5EA000010B50D4BD8
:10D760002C21044698470C4B0022C4E9003223893F
:10D77000E26023F47F6323F00F0343F4027343F06A
:10D78000010323814FF4FC63C4E90822238562610D
:10D7900010BD00BF19F00000E0011001F8B504460B
:10D7A0000D4617461E462421034B9847C4E90057EF
:10D7B000C4E90256F8BD00BF19F000002DE9F3419D
:10D7C0003B4B3C4E05463C489847044698B9B04709
:10D7D00020B10024204602B0BDE8F081374B384923
:10D7E00000937C220320374CA0473748374900225A
:10D7F00000238847FEE7364B4FF4B8719847294617
:10D80000344B354D2C2220469847344B4C2104F1A3
:10D81000300098470023C4F86C312B6803B92C60A2
:10D82000234603221E212E48DFF8CC802F682C606F
:10D83000C047E062B047064660B9204B20490093DC
:10D840008D2203201F4DA847E26A1F481F49334617
:10D850008847FEE7E36A002BBBD0B4F86831214E5D
:10D860006FF309030021A4F86831C4F86C1108466D
:10D87000B0470021E0630846B04700212064084615
:10D88000B047194E60640021206CB047606C0021E5
:10D89000B047206C154E0021B047606C0021B047A6
:10D8A000E06B134B9847E06A124B2F60984791E763
:10D8B00019E60000E11700000C860020CF3E0200B0
:10D8C0009C3E0200E9E80000BEED0100E9170000FF
:10D8D00019F0000031EC0000E885002005E60000AA
:10D8E000F54F0000E5300000952E00005D1E0000A1
:10D8F0008527000041FC0000D1FB0000014B1868A7
:10D90000704700BFE885002010B9074B186838B190
:10D91000037A9B0754BFB0F90000B0F902007047CA
:10D920004FF4F070704700BFE885002010B9074B36
:10D93000186838B1037A9B0754BFB0F90200B0F9F8
:10D94000000070474FF48870704700BFE8850020E2
:10D9500010B9044B186818B10089C0F389007047EA
:10D9600082207047E885002008B5014610B90F4BAA
:10D97000196899B10E4B0846984702460D4B084668
:10D9800098470A235A43B2FBF0F01D2809D93128E1
:10D9900009D9462834BF0220032008BD4FF4F07295
:10D9A000ECE70020F9E70120F7E700BFE885002059
:10D9B00009D9000051D90000436800229A61DA6158
:10D9C000704700000146034809B9034B1847034B51
:10D9D000184700BF0C860020A9E60000B5E600004D
:10D9E000406870474368186818B15868003818BF15
:10D9F0000120704708B5074B0246984740B113888D
:10DA000051885268D06813FB01F31B1A58425841E1
:10DA100008BD00BFE5D900000146034809B9034B22
:10DA20001847034B184700BF18860020A9E60000DE
:10DA3000B5E60000034B00221A705A681044586083
:10DA4000704700BFEC850020034B58680121197016
:10DA50001A78002AFBD07047EC85002010B5024BE5
:10DA600004469847001B10BD49DA0000D1E908239D
:10DA70009A421CBF9B0293FBF2F3D1E9060208BF56
:10DA80004FF48063121A534300EBA32000B2704797
:10DA900010B5074C074801232370074B9847074BE5
:10DAA000014618B96068BDE8104018470421F9E73D
:10DAB000F48500203C860020A9E600006DFB0000F4
:10DAC0002DE9F0474F48504F4E4C504D90B0B8475D
:10DAD000A0B94F4D4F4BA868DFF82881DFF82C9193
:10DAE000DFF848A1984706464648B84704467CB93F
:10DAF000494B9847A86010B0BDE8F08790F83C30DB
:10DB00006FF3410380F83C3001462046A847DFE729
:10DB100000232B7094F83C309A076FD443F0020333
:10DB200084F83C30636A002B05DCF34203D4A3681D
:10DB30000BB120469847636A3344002B63622EDBA7
:10DB4000226A9A42D4BF626263622046214650F83C
:10DB5000103F53B39847636813B101B220689847E8
:10DB6000D4E908329A421ADB94F83C30A28EE16A7A
:10DB700013F0010322D1DAB900293CD14022214619
:10DB80006846D0472146254B40469847244B2046BF
:10DB90009847244B9847039B0BB1684698472B78CE
:10DBA00063B34046B8470446A1E71F4B9847D2E706
:10DBB0004FF6FF70824204D0013AA286A28E002A5C
:10DBC000DAD0226B524262620029E8D013B9A26A0D
:10DBD0005242626283F0010294F83C3062F3000327
:10DBE000D4E9060284F83C30DB0758BFA16B216200
:10DBF000C4E90620D3E7002BE3D0BFE72146404627
:10DC0000C847D0E73C860020A9E60000B5E6000042
:10DC1000F48500205DDA000049DA00006DE70000BD
:10DC2000E5EA000091DA00006DDA000031EC000056
:10DC300038B5402109480A4B0A4C0B4D98470B4B0D
:10DC400098470023A06004221E210948A847094BD9
:10DC5000606098470023237038BD00BF3C860020D9
:10DC600005E60000F4850020D1FB000049DA000041
:10DC7000C1DA000091DA000010B50B4B04464021D8
:10DC800098474FF4FA73236200216423C4E9061312
:10DC9000064B23610123A38694F8363043F0010339
:10DCA00084F8363010BD00BF19F000006DDA0000B6
:10DCB0002DE9F84F144BDFF85490DFF85CA0DFF843
:10DCC0005CB0064611480D4698474FF000080446E0
:10DCD00014B94046BDE8F88F21464846D04723682E
:10DCE000B34207460DD16368AB4200D04DB921461F
:10DCF0004846D847064B20469847064B98474FF072
:10DD000001083C46E4E700BFA9E600003C8600208D
:10DD1000E5EA000091DA0000B5E600006DE70000DA
:10DD200073B54168054611B100681D4B98471D4801
:10DD30001D4B984720B11D4B98471D4B01389860EB
:10DD40001C4B184898471C4B04469847064660B938
:10DD50001A4B1B4900936A2203201A4DA8471A4800
:10DD60001A49224633468847FEE7B4B12B6AAB63B3
:10DD70004022174B29462046984794F83630DB0757
:10DD800006D5636823B1206810B1B4F9181098471C
:10DD9000104B02B0BDE87040184702B070BD00BF24
:10DDA000B1DC00003C860020D1E8000049DA000028
:10DDB000F485002019E60000E1170000143F02007E
:10DDC000E43E0200E9E80000BEED0100E9170000B2
:10DDD00031EC000091DA0000F8B5094B094E0A4F0A
:10DDE000044608480D46984700B9F8BD0368A342A9
:10DDF00002D14368AB42F8D001463046B847F3E75A
:10DE0000A9E600003C860020B5E600008A1A002A38
:10DE1000B8BF52424FF47A735A43B2FBF0F0012874
:10DE200038BF01204FF6FF73984228BF184680B2D2
:10DE3000704730B5B0F90430B0F9005040885B1B32
:10DE400003EBD373121A5C10C3F34F03491BD21AAE
:10DE5000C91A12FB02F2644311FB01218C42B4BFC8
:10DE60000020012030BD438801391944C18070472A
:10DE7000B0F90030B0F90420B0F90210D21AB0F9AC
:10DE80000630581A013002FB00007047B1F900302B
:10DE900070B5B2F90050B1F90240B1F90460B1F9BE
:10DEA00006109D42B8BF1D46B2F902300580A3425C
:10DEB000B8BF2346B2F90440B2F906204380B44209
:10DEC000A8BF34468A42A8BF0A46A5428480C280C1
:10DED00004DC9342CCBF0020012070BD0020FCE791
:10DEE000B2F9003010B5B1F90040A342A8BF2346F3
:10DEF0000380B1F90240B2F90230A342A8BF234621
:10DF00004380B1F90440B2F90430A342B8BF2346BC
:10DF10008380B2F90630B1F906209342B8BF1346A8
:10DF2000C38010BD2DE9F04FB1F90090B0F9004069
:10DF3000A14587B08846C0F28880B0F904300193CB
:10DF4000994500F38280B1F902A0B0F902B0DA4538
:10DF50007BDBB0F906309A4577DC002A03DC012030
:10DF600007B0BDE8F08FBDF804000290A7B2013001
:10DF7000C01B9EB2ADF81040C0F3C0341FFA8BFC3A
:10DF800004FA80F0741CA4EB0C04C4F3C03505FA49
:10DF900084F540106D10A842A8BF28469042A8BF43
:10DFA00010461CFA80F417FA80F7002285B2BFB23F
:10DFB00024B204A80393ADF81470ADF812B0ADF814
:10DFC0001640FFF7AFFF039B024640B13D44ADF85A
:10DFD00014501F4B5246494604A89847C0E7761B89
:10DFE000B6B2414604A8ADF81260ADF81630FFF79E
:10DFF00099FF024630B12F44751BADF81470ADF88F
:10E000001250E6E7029B5F1BBFB2019BADF8107098
:10E01000414604A8ADF81430FFF784FF024630B142
:10E020007F1B761BADF81070ADF81260D1E741464A
:10E0300004A8ADF812B0ADF81640FFF773FF002842
:10E040008DD07F1BADF81070C3E7002088E700BFBC
:10E0500033DE0000B0F90020B1F904309A4214DC3C
:10E06000B0F90420B1F900309A420EDBB0F9022079
:10E07000B1F906309A4208DCB0F90600B1F9023075
:10E080009842B4BF00200120704700207047000074
:10E090002DE9FF41B0F90070B1F90030BB420546EF
:10E0A0000C4624DCB0F90210B4F9023099421EDBB0
:10E0B000B0F90410B4F90430994218DCB0F9063014
:10E0C000B4F906108B42CCBF0020012062B16B88EE
:10E0D000164E019203A92046ADF80C70ADF80E3033
:10E0E000B047019A28B9002004B0BDE8F0810020B3
:10E0F000ECE7B5F90480ADF80C8003A92046019245
:10E10000B0470028EFD0EB88019AADF80C7003A956
:10E110002046ADF80E30B0470028E4D0019AADF8A3
:10E120000C8003A92046B047DEE700BF25DF0000D2
:10E13000F0B544880588142A3FD8DFE812F01500AE
:10E140003B0045005A00610069007C0083008500A7
:10E150008C009300A600AD00B300C600CD00D20035
:10E16000D700DC00DF00E20082880F880132521BFA
:10E17000C2F3C03606FA82F68A880132D21BC2F395
:10E18000C03707FA82F25210C2EB66021A80C288C8
:10E190000132121BC2F3C03000FA82F0CA884988EB
:10E1A0000132521AC2F3C03101FA82F25210C2EBAC
:10E1B000600201E000221A805A801A8815445A88A9
:10E1C0001D8014445C80F0BD82880132521BC2F372
:10E1D000C03000FA82F08A8809880132521AC2F3EC
:10E1E000C03101FA82F25210C2EB60021A800022A2
:10E1F000E2E70A888988521A81880A44521BF5E7A7
:10E2000000221A804A88C988521AC1880A4447E005
:10E2100082880F880132521BC2F3C03606FA82F69A
:10E220008A880132D21BC2F3C03707FA82F2521039
:10E23000C2EB6602E5E78E880A88921B8688324424
:10E24000521BDEE70022A1E78E880A88921B86888F
:10E250003244521B9AE700221A804A88C988013A40
:10E26000521AA9E782880E880132521BC2F3C030CD
:10E2700000FA82F08A880132921BC2F3C03606FA95
:10E2800082F25210C2EB6002E6E70A888E8880882C
:10E29000921B0244521BDFE700221A80C28801321F
:10E2A000121B89E782880132521BC2F3C03606FA7C
:10E2B00082F68A8809880132521AC2F3C03101FA03
:10E2C00082F25210C2EB6602E7E70A888988521A86
:10E2D00081880A44521BE0E70A888988013A521A69
:10E2E00084E70A888E88013A921B4FE70A888E8855
:10E2F000013A921B85E7828801327FE782880132EA
:10E30000A7E7828801329BE7830710B58CB21CBF58
:10E3100020F8021B02F1FF3204EB0443102A0146ED
:10E3200000F1200004D801EB42028A420AD110BD5C
:10E3300040E9083340E9063340E9043340E9023359
:10E34000103AEBE721F8024BEFE730B5C1F1FF04DB
:10E35000C0F3451565433F23C1EB411213FB015147
:10E3600000F01F0348F2810504FB0323C0F3C4201F
:10E3700069436B4304FB0020C1F3C5516843C3F3F9
:10E38000C45343EA4113C00D43EAC02030BDC1F17C
:10E39000FF0110B5C0F3451200F01F0348F28104DD
:10E3A0004A434B43C0F3C420624363434843D20D06
:10E3B0006043DB0D43EA4213C00D43EAC02010BDA9
:10E3C000431C184613F8012B2AB13A2AF9D05C2ACB
:10E3D000F7D02F2AF5D070470148024B4421184747
:10E3E0002486002005E6000038B50446406860B188
:10E3F000036963B121689847064B05462068984732
:10E400000023C4E90033284638BD0B25FBE7092566
:10E41000F9E700BFE5EA00007FB505461C460BB1F1
:10E4200000232360686870B1866976B10023039386
:10E4300003AB009313460A462968B0470CB1039B0F
:10E44000236004B070BD0B20FBE70920F9E74368A7
:10E4500010B40A463BB11C6A4CB101681846234609
:10E460005DF8044B18470B205DF8044B70470920FA
:10E47000FAE7000070B5074B074D084E0446064802
:10E48000984700B970BD0378A342FBD001462846E7
:10E49000B047F6E7A9E6000024860020B5E60000B4
:10E4A00000232DE9F341C0E90033044617460E4628
:10E4B000002943D00878234B9847606028B9206032
:10E4C0000325284602B0BDE8F08183682BB1984748
:10E4D00018B9C4E900000125F3E7636858881A4BAE
:10E4E00098471A4B20609847054660B9184B194960
:10E4F00000936F220320184EB0472268174818492E
:10E500002B468847FEE7216811B961600A25D8E7E4
:10E51000D4F80480D8F80C5095B1124B3046984787
:10E520003B4602464046A84705460028C9D00E4B48
:10E53000206898470023C4E90033C2E70B25C0E7F1
:10E540000925BEE775E400002DEA0000E117000090
:10E550006D3F02002C3F0200E9E80000BEED010023
:10E56000E9170000C1E30000E5EA000010B5094B1F
:10E570000446984708B9084804E0235C2E2B02D1D2
:10E580000130204410BD2F2BF5D05C2BF3D0013887
:10E59000F0E700BF39630100D8F701000139031D1E
:10E5A00011F8012F00F8012B9842F9D170470000B3
:10E5B00007B5019229B1006808442AB1044B01A9AA
:10E5C000984703B05DF804FB024B04219847F8E735
:10E5D0009DE5000019F0000007B5019231B1036814
:10E5E0000433C8182AB1054B01A9984703B05DF858
:10E5F00004FB034B04219847F8E700BF9DE50000AA
:10E6000019F000000023C0E901338B071CBF21F083
:10E61000030104310160704770B5044600680D4B7A
:10E6200008309847054690B10146002220460A4E20
:10E63000B04729466268094B20469847616811B186
:10E640002A462046B047A368656003B9A5602846FE
:10E6500070BD00BF2DEA0000B1E50000D9E5000063
:10E6600070B5044600680D4B08309847054690B1D8
:10E670000146002220460A4EB0472946A268094BAF
:10E6800020469847A16811B12A462046B0476368E2
:10E69000A56003B96560284670BD00BF2DEA000083
:10E6A000D9E50000B1E5000000B14068704700B155
:10E6B0008068704707B50023019328B103680433CD
:10E6C000194401A8024B9847019803B05DF804FB78
:10E6D0009DE5000007B50023019320B1036801A860
:10E6E0001944034B9847019803B05DF804FB00BF41
:10E6F0009DE500002DE9F0410E46044640B349B3C4
:10E700004368994203D1BDE8F041134B18470068B4
:10E71000124B083098470546B8B1114BDFF84880D6
:10E720003146204698472A46074601462046C047BC
:10E730003A4629460B4F2046B8472A4631462046DE
:10E74000B847324629462046C0472846BDE8F081F2
:10E750000546FAE70D46F8E719E600002DEA000045
:10E76000D5E60000B1E50000D9E5000070B50D4622
:10E770000446F8B1436899420CD12946174B20460C
:10E7800098470146606008B9A06070BD0022144B34
:10E7900020460CE0836899420ED1124B98470146FF
:10E7A000A06008B96060F0E70F4B00222046BDE88A
:10E7B000704018470029E0D029460A4B2046984768
:10E7C00029460646054B20469847314602460546EF
:10E7D000054B2046984732462946D8E7B5E6000063
:10E7E000B1E50000D5E60000D9E500002DE9F041D3
:10E7F0000C461E461146164BDFF85C80154F154639
:10E80000984796B1002229462046C04729466268AB
:10E810002046B847616811B12A462046C047A36820
:10E82000656003B9A560BDE8F081A268294620466D
:10E83000C047294632462046B847A16811B12A464A
:10E840002046B8476368A560002BECD16560EAE715
:10E850006DE70000D9E50000B1E5000091422DE927
:10E86000F84304460D46174622D01AB3144B1146FE
:10E8700098470646AE421BD0124BDFF84C80DFF8BB
:10E880004C902946204698472A4631462046C047A4
:10E89000324629462046C8472A4639462046C847B8
:10E8A0003A4629462046C04707B9A56006B96560C3
:10E8B000BDE8F88308B18668DCE70646DAE700BF02
:10E8C000D5E600006DE70000D9E50000B1E50000E5
:10E8D00030B1436833B98068B0FA80F040097047BE
:10E8E00001207047002070472DE9F0431F46431E6A
:10E8F000DBB2042BC5B004460D46164617D84DAB07
:10E900000DF11009DFF8308003934C9A4FF48071B9
:10E910004846C047074BD3F80080B8F1000F06D037
:10E92000CDF800903B46324629462046C04745B0C8
:10E93000BDE8F0838487002021F800004FF4B47311
:10E9400090FBF3F202FB130000B20028BCBFC0181A
:10E9500000B259280E4B02DC33F91000704780B228
:10E96000A0F15A02592A03D8C0F1B40080B2F3E7EB
:10E97000A0F1B40292B2592A85BFC0F5B47080B23A
:10E9800033F8120033F81000404200B2704700BF65
:10E99000883F020030B500020023D41804FB04F5C0
:10E9A000A84228BF23465208F7D11A091B01DBB23F
:10E9B0000A804B8030BD0000074A0346106853B1FF
:10E9C00053F8042B03EB5203191D00F580429142CA
:10E9D00034BF184600207047888700208B0718BF77
:10E9E00021F00301026818BF043110B50C1DB4EB0F
:10E9F000520FC2F35E030BD08B4204D0043B42188B
:10EA00005B1A5B005360036861F35F03036010BD32
:10EA10001946F8E7034A044B136047F6F8721A6088
:10EA2000704700BF888700209487002073B5054693
:10EA3000E8B1820718BF20F00305124E18BF043555
:10EA400000242046B047044698B10378DB07F8D489
:10EA50000368B5EB530FF4D80B4B2946984703785E
:10EA600043F0010304F8043B204602B070BD074C9C
:10EA7000FAE7074B00930749074B084DD1220220C4
:10EA8000A847F1E7B9E90000DDE900008C87002024
:10EA90006D4002003E40020052410200E9E80000E1
:10EAA00038B50E4B0E4D1C6804B938BD2046A8473A
:10EAB0002378DA070FD50446F6E70378DB07FAD4A4
:10EAC00023680168C3F35E02043202EB510262F371
:10EAD0005F032360A8470028EFD1E6E7888700207E
:10EAE000B9E90000164A131D984270B5044610D0CB
:10EAF00078B110F8043C6FF3000300F8043C13896C
:10EB000001339BB20F2B138114D80E4D0438A84744
:10EB100000B970BD0378DB07FBD454F8043C0168EE
:10EB2000C3F35E02043202EB510262F35F0344F866
:10EB3000043CECE700231381BDE87040024B18470A
:10EB400088870020B9E90000A1EA000040B1054B28
:10EB5000984204D050F8040CC0F35E0070470020C7
:10EB6000704700BF8C870020164B1A68904213B57F
:10EB70000BD09A6890420AD1012203EBC2039A7922
:10EB80006FF300029A7102B010BD0022F5E70E4A41
:10EB9000002352F83340844202EBC30104D18B7945
:10EBA0006FF300038B71EEE70133102BF1D1074BAC
:10EBB00000930749074B084C40F232220320A0473C
:10EBC000E1E700BF44000020748600208640020078
:10EBD0003E4002005F410200E9E80000114B9A79D3
:10EBE0006FF300022DE9F0419A719A7B0E4CDFF829
:10EBF0003C806FF3000200259A7327462E4620685A
:10EC000040B1C04707EBC50326609A7966F300025E
:10EC10009A71A6800135102D04F10804EFD1BDE8EA
:10EC2000F08100BF4400002074860020E5EA000067
:10EC300070B500F0030501F00306B54204460B462B
:10EC400040F09880002D40F0A88005462B46202AF1
:10EC50001C4601F1200503F1200300F2B080042AD4
:10EC60000E4640F29F8051F8043B44F8043B043ABE
:10EC7000F5E713F8201C04F8201C13F81F1C04F8F7
:10EC80001F1C13F81E1C04F81E1C13F81D1C04F88E
:10EC90001D1C13F81C1C04F81C1C13F81B1C04F886
:10ECA0001B1C13F81A1C04F81A1C13F8191C04F87E
:10ECB000191C13F8181C04F8181C13F8171C04F876
:10ECC000171C13F8161C04F8161C13F8151C04F86E
:10ECD000151C13F8141C04F8141C13F8131C04F866
:10ECE000131C13F8121C04F8121C13F8111C04F85E
:10ECF000111C13F8101C04F8101C13F80F1C04F856
:10ED00000F1C13F80E1C04F80E1C13F80D1C04F84D
:10ED10000D1C13F80C1C04F80C1C13F80B1C04F845
:10ED20000B1C13F80A1C04F80A1C13F8091C04F83D
:10ED3000091C13F8081C04F8081C13F8071C04F835
:10ED4000071C13F8061C04F8061C13F8051C04F82D
:10ED5000051C13F8041C04F8041C13F8031C04F825
:10ED6000031C13F8021C04F8021C13F8011C04F81D
:10ED7000011C203A202A1D46214603F1200304F1FC
:10ED800020043FF676AF6B1E0A44914200D170BD5D
:10ED900013F8014F01F8014BF7E7C5F104050544ED
:10EDA0001E4612B9731E224430E013F8011B04F80A
:10EDB000011BAC42194602F1FF32F1D146E755F88A
:10EDC000201C43F8201C55F81C1C43F81C1C55F84B
:10EDD000181C43F8181C55F8141C43F8141C55F85B
:10EDE000101C43F8101C55F80C1C43F80C1C55F86B
:10EDF000081C43F8081C55F8041C43F8041C203A6E
:10EE0000294624E713F8011F04F8011B9442F9D1A5
:10EE1000BDE700008B07F7B50D4618BF21F00305CD
:10EE2000044618BF043528B110F8043C13F0010F54
:10EE300008BF0024164B204698478542074604D059
:10EE400005D2144B2946201F984726460DE0124B49
:10EE500028469847064658B9104B00931049114B65
:10EE6000114C40F23F120220A047304603B0F0BDE3
:10EE7000002CFAD0002FF8D0BD422A460B4B28BFF9
:10EE80003A46214698470A4B20469847EDE700BF8F
:10EE90004DEB0000DDE900002DEA00006D400200AE
:10EEA0003E40020073410200E9E8000031EC00003E
:10EEB000E5EA0000F7B590B1102812D8364A9379E8
:10EEC00013F0010303D0937BDE070AD4012302EB86
:10EED000C300817941F00101817152F8330003B020
:10EEE000F0BD2E4C00234FF0FF32271D04EBC3066C
:10EEF000B5792946ED0713D437F8335085420FD33F
:10EF000005D141F0010154F83300B171E7E7561C17
:10EF100001D15AB204E004EBC2018988A942F8D8B1
:10EF20000133102BE2D1551C08D004EBC20154F878
:10EF300032008B7943F001038B71D0E7002504EB9D
:10EF4000C50399790A46C90717D442F0010298808F
:10EF50009A710146124B54F83500984744F8350031
:10EF600040B9104B00931049104B114E4FF40472EE
:10EF70000320B04754F83500B1E70135102DDED13C
:10EF80000C4B00930320094B0749094C40F2162211
:10EF9000A0470020A3E700BF4400002074860020A3
:10EFA00015EE0000B24002003E4002008241020025
:10EFB000E9E800001441020010F0030310B409D086
:10EFC000C3F1040303442AB100F8011B984202F183
:10EFD000FF32F8D101EB012404EB014404EB01649E
:10EFE0000346202A184603F1200305D8042A0DD829
:10EFF000084B5DF8044B184743E9084443E90644CD
:10F0000043E9044443E90244203AEAE740F8044B68
:10F01000043AEBE70563010010F003030A460DD143
:10F0200003460021202A184603F1200315D80023A7
:10F03000042A08D940F8043B043AF9E7C3F1040371
:10F040000344002112B90A4B0021184700F8011BA4
:10F05000834202F1FF32F5D1E2E743E9081143E9C7
:10F06000061143E9041143E90211203ADAE700BF2F
:10F070000563010010F003030A460FD103464FF069
:10F08000FF31202A184603F1200316D84FF0FF3332
:10F09000042A08D940F8043B043AF9E7C3F1040311
:10F0A0000344FF2112B90A4BFF21184700F8011B46
:10F0B000834202F1FF32F5D1E0E743E9081143E969
:10F0C000061143E9041143E90211203AD9E700BFD0
:10F0D000056301009A4238BF8854704770472DE994
:10F0E000F74F1746DDE9116212F0020A8046DDE9AA
:10F0F0000C54DDE90F0C9DF838E01FD102F0010936
:10F100004EB1B9F1000F06D0BEF1000F02D112F0DE
:10F110000C0F00D0013E4FF0300B02E005F804B0B8
:10F120000134A44501D9202CF8D14FF0300BB9F1AE
:10F13000000F03D0A64201D9202C37D112F0100FB6
:10F1400019D012F4806F36D1ACB3644501D0B4420B
:10F1500031D1B4F1010C2DD010286AD1023C9006B7
:10F1600031D41F2C0FD87820285501341F2C0AD8F1
:10F17000302028550134202C05D0BEF1000F26D0B8
:10F180002D202855013492073BD03A46254414449B
:10F19000A2423AD1BAF1000F04D0D51BB54205EB1B
:10F1A00007043DD3204603B0BDE8F08F05F804B056
:10F1B0000134BCE764461028D1D00228D6D11F2CD8
:10F1C000E1D86220D0E71F2CDDD85820CCE75007CB
:10F1D00001D52B20D5E71007D5D52020D1E7202059
:10F1E000CDE90013C047DDE9001309F101094E45DF
:10F1F0000BEB0902F3D8321BB44288BF00223A4419
:10F20000C4E7A146A7EB040BF1E702F1010915F8E9
:10F21000010DCDE90013C047DDE900134A46B7E709
:10F2200022462020019300910135C047DDE90013FB
:10F23000B4E70228644699D1C3E700002DE9F04302
:10F2400091B0189D1A9E1D9F0DB927F010077C05DF
:10F2500000D515B317F0200F14BF4FF0410E4FF03B
:10F26000610EAC460DF120080025AEF10A0EBCFB84
:10F27000F6F906FB19C95FFA89F4B9F1090F94BFD1
:10F2800030347444E4B2B44508F8014BBCFBF6F4E6
:10F2900005F1010501D3202D10D11C9C05941B9C68
:10F2A0000697CDE903649DF86440CDE9015408ACAC
:10F2B0000094034CA04711B0BDE8F083A446D6E704
:10F2C000DFF000002DE9F04F2DED048B93B0DDE968
:10F2D00020649A4656EA040302BF289B23F01003D9
:10F2E0002893289B5B05DDE924B908EE100A08EE97
:10F2F000901A09EE102A02D556EA04033FD0289B43
:10F3000013F0200F14BF412361230A3B0DF128089D
:10F310000025099321461B4F5A464B463046B847B5
:10F32000D2B2092A8ABF099B3032D2185E45D2B2C6
:10F3300074EB090408F8012B05F1010501D3202D18
:10F340001AD1289B0693279B0593269B0E4CCDE94B
:10F3500003B39DF88830CDE901530AAB009319EE51
:10F36000102A18EE901A18EE100A5346A04713B050
:10F37000BDEC048BBDE8F08F06460C46CAE70025BD
:10F38000DFE700BF415F0100DFF000002DE9F04F33
:10F3900017461E46AC4AAD4B8946011E91B014BFBC
:10F3A00093469B460025387858B94D452CBF09F146
:10F3B000FF322A464B460020D847284611B0BDE808
:10F3C000F08F252807F1010706D06C1C4B462A4612
:10F3D0000A91D8472546D2E0002306E02D2A16D010
:10F3E000302A0CD143F001030746384610F8012BB0
:10F3F0002B2A0FD0F2D8202A0FD0232A10D0A2F126
:10F400003004092C2CD84FF000080A2410E043F0F7
:10F410000203E9E743F00403E6E743F00803E3E708
:10F4200043F01003E0E704FB0822A2F1300807468E
:10F43000384610F8012BA2F1300CBCF1090FF2D9BB
:10F440003A782E2A5AD17878A0F13004092C07F1A5
:10F45000010243F4806348D800244FF00A0E14E000
:10F460002A2A0AD156F8048BB8F1000FBCBF43F02A
:10F470000203C8F100080746E2E74FF00008DFE7A3
:10F480000EFB0400A0F130043A46174617F8010BB2
:10F49000A0F1300CBCF1090FF2D917463A4612F828
:10F4A000010B6C2833D02BD8682837D06A283FD07E
:10F4B00017F801EBBEF1780F11D8BEF1630F3AD8FF
:10F4C000BEF1620F00F0A280BEF1630F00F0FC807D
:10F4D000BEF1250F03D0BEF1580F00F093806C1CD5
:10F4E0004B462A460A91704673E72A2805D156F8FA
:10F4F000044B023724EAE474D0E717460024CDE732
:10F50000742801D07A28D3D143F480730BE0787843
:10F510006C28F9D143F440730237C9E7787868283A
:10F5200003D043F080031746C2E743F0C003F3E77C
:10F5300043F40073F7E7AEF1640C45485FFA8CFCC6
:10F54000012202FA0CF202401BD1BEF1730F00F04F
:10F55000FB80BEF1700FC2D143F021030593082355
:10F56000CDE903431023CDE9012356F8043B009372
:10F570002A46384C0A914B465846A04705460A99F8
:10F5800011E7BEF1780F3FD0BEF16F0F00F044815C
:10F59000BEF1690F23F010034FF00A0202D0BEF152
:10F5A000640F34D1580548BF23F00103BEF1690F41
:10F5B00003F4007C02D0BEF1640F4FD1BCF1000F08
:10F5C00028D0073626F00706B24676685AF8080BA8
:10F5D0000694CDE9078300230593F30F002E0293D1
:10F5E0000492034602DA434266EB4606CDE9003652
:10F5F000194C0A914B462A465846A0470A99054697
:10F600005646D0E643F02003102200E0022223F009
:10F610000C03C7E7D80506F1040A01D5306802E0FB
:10F6200058060CD53078CDE90224CDE904830028B2
:10F630004FEAD0730193B8BF404200902DE0180606
:10F64000ECD5B6F90000EEE7D5F00000DDF00000E3
:10F65000210812003DF20000C5F20000BCF1000FCD
:10F660000FD0CDE907830023CDE9042306F1070A73
:10F670002AF0070A06940293FAE80223CDE9002350
:10F68000B6E7D80506F1040A0ED5CDE90483CDE925
:10F690000224CDF804C033680093604C0A914B46B5
:10F6A0002A465846A047A9E7580607D53078CDE93D
:10F6B00004830023CDE902240193BEE7306813F0F0
:10F6C000800F18BF80B2F2E713F0020426D04FF08B
:10F6D000010A6B1C0A930B9116F8040B4B462A4641
:10F6E000D8470B9974B30A9A544621E00A914B46C5
:10F6F0002020D8470A9905EB0A020AF1010AC245FF
:10F70000F4D3B8F1000F08F1FF3308BF002308F16C
:10F71000010A1D4408BF4FF0020ADAE7A246EAE7F1
:10F720000B914B462020551CD8470B9901342A4693
:10F730004445F5D30A9AA8EB0A03D04538BF002305
:10F740001A440A920A9D2EE63246002C52F8046BA7
:10F750000A9214BF20464FF0FF303044324692F8F0
:10F7600000C0BCF1000F01D0904211D1A2EB060AFB
:10F7700013F480620B9202D0A24528BFA24613F078
:10F7800002030C931CD1AAEB05032A460E9309E051
:10F790000132E4E7531C0D930F914B462020D847CC
:10F7A0000D9A0F990E9BD3184345F3D3A8EB0A0388
:10F7B000D04538BF00230AF101021D4403EB020AC1
:10F7C000AB1B0D9305E01C460E914B462A46D847CD
:10F7D0000E990D9B9D1916F8010B28B10B9B002B60
:10F7E000F2D0631E002CEED10C9B9BB12A46AAEBF3
:10F7F000050406E00B914B462020561CD8470B9978
:10F800003246A3189845F5D8A8EB0A03D04538BF6F
:10F8100000231D440A9EC6E50822F8E63DF20000DA
:10F8200010B4024CA4465DF8044B60478DF3000011
:10F8300008B50548054B18219847054B00221A705A
:10F8400001225A7008BD00BF0086002005E60000B6
:10F85000B4C70020F7B5364B364898470546E0B1A7
:10F86000344E354C2B7D03F00703032B29462ED84D
:10F87000324B30489847324B04469847054608BB00
:10F88000304B31490093DB220320304EB0473048E3
:10F89000304922462B468847FEE72F4B254898479C
:10F8A000274B04469847054660B9264B26490093E6
:10F8B000D3220320254EB0472548264922462B4611
:10F8C0008847FEE7ECB90024204603B0F0BD30467F
:10F8D000A04705460028C5D1204B16489847184B2D
:10F8E000044698470028EDD1164B17490093E522AE
:10F8F0000320164EB0471648164922462B46884725
:10F90000FEE74FF4FA732360237D154D032262F363
:10F910000203002723754FF0FF3301262361A76000
:10F92000104B2E709847E7606060AE70CCE700BF68
:10F93000A9E6000000860020B5E60000F5E600001C
:10F94000E1170000C241020092410200E9E8000014
:10F95000BEED0100E917000019E6000061E60000B5
:10F96000B4C7002049DA000070B501460446074BD1
:10F970000748084D98470126074B2E7020469847A8
:10F98000064B1B68A34208BFEE7070BD6DE7000018
:10F9900000860020B4C70020E5EA00007086002041
:10F9A00038B5124B044640689847236898421BD3E9
:10F9B0000F4B104D98470023EB70AB70A36860604D
:10F9C00043B92369002B0CDC236943B90A4B204659
:10F9D000984704E020469847EB78002BF1D00120AF
:10F9E00038BD013B2361EFE70020F9E75DDA000055
:10F9F00049DA0000B4C7002069F900002DE9F84F8A
:10FA0000DFF85CB19BF80440012034B99BF8012079
:10FA10008BF804001AB98BF80420BDE8F88FDFF8E2
:10FA20004481DFF838A1DFF84091C047CBF80800E7
:10FA3000002250468BF803208BF80220C847434D24
:10FA4000434F2860296889B1424B50469847064683
:10FA50002868027D12F0070108D0A04250D0052985
:10FA600039D1B8479BF80220002A62D03A4CDBF823
:10FA70000800A047DBF80C201044CBF80C00DBF8A2
:10FA80001400A047B0F5FA7F16D3DBF80C206421F0
:10FA90004A434FF4FA71B2FBF1F2D2B2642A9ABF30
:10FAA000C2F16402D2B200228BF810200022CBF8FF
:10FAB0000C20C047CBF814004FF0FF322748CBF89A
:10FAC0001820C847254E234F0546E5B9DBF8180036
:10FAD0008BF80450A1E734B1217D02F0070201F058
:10FAE00007018A42BED9B8470028BBD09BF8022044
:10FAF000002ABBD19BF80320002AB7D12C6897E7D6
:10FB000000242E609EE72A7D53070DD06868A04729
:10FB10002A68904238BF101ADBF8182028BF00204E
:10FB2000824288BFCBF8180029463046B8470546C0
:10FB3000CBE79BF80320002A98D19BF800100029FE
:10FB4000DFD08BF80020144672E700BF70860020DB
:10FB5000A1F90000B5E600005DDA00000086002093
:10FB6000B4C7002049DA0000A9E60000F8B5037D1B
:10FB700003F007038B4204460D4618D00F48104B84
:10FB80000E4E104F9847024632B1137D03F0070323
:10FB90009D420DDBA24203D008480B4B21469847FB
:10FBA0000A4B01221A70237D65F302032375F8BD09
:10FBB00011463046B8470246E6E700BF00860020FF
:10FBC000A9E60000B5E600005DE80000B4C700202B
:10FBD0002DE9FF411E46124B03920F46804698477F
:10FBE000104B044698470399054668B90E4B0F49D8
:10FBF00000934FF4837203200D4EB0470D480E4919
:10FC000022462B468847FEE734B10C4BC4F80880E7
:10FC1000276020469847E660204604B0BDE8F081A2
:10FC200055F80000E1170000D741020092410200A0
:10FC3000E9E80000BEED0100E91700006DFB0000DF
:10FC400010B5044B044698472368C31A013B636010
:10FC500010BD00BF49DA000090F900200378002AA7
:10FC60000FDA03F0E002C02A0DD003F0F002E02A20
:10FC70000BD003F0F800A0F1F00358425841800087
:10FC8000704701207047022070470320704773B50A
:10FC90000023019301B901A90A688556835C002DF0
:10FCA00002F1010403DB18460C6002B070BD03F0E2
:10FCB000E005C02D10D10C60005D00F0C004802C68
:10FCC00001D00020F1E79B0103F4F86300F03F004E
:10FCD000184402320A60E8E703F0F005E02D17D17E
:10FCE0000C60045D04F0C005802DEAD1951C0D6008
:10FCF000455D05F0C0008028E3D1180380B205F00F
:10FD00003F05A401284404F47C6420440332E1E765
:10FD100003F0F805F02D0C60D3D1045D04F0C005AC
:10FD2000802DCED1951C0D60455D05F0C006802E5E
:10FD3000C7D1D61C0E60805D00F0C006802EC0D1F9
:10FD40009B042403AD0100F03F0003F4E01304F42E
:10FD50007C3405F47C651C43054428190432B9E75A
:10FD60000B68F7B5013B0D4F0B6006460C460425AA
:10FD700020683B6830449847236848B92BB1013D5F
:10FD8000013B15F0FF052360F2D1002003B0F0BD68
:10FD9000019301A97B6830469847F7E7540000209B
:10FDA0002DE9F0410024DFF8288007460D4626465D
:10FDB000AE4202D12046BDE8F0813819D8F80030B3
:10FDC0009847012838BF012054FA80F40136EFE744
:10FDD00054000020F7B50024074F019406460D4655
:10FDE000019BAB4202D3204603B0F0BD7B6801A962
:10FDF000304698470134F3E75400002073B50024DF
:10FE0000074E01940546019BEB5C13B9204602B0F6
:10FE100070BD736801A9284698470134F3E700BF15
:10FE2000540000207F2882B011D9B0F5006F10D2A5
:10FE3000830963F03F0300F03F008DF8043060F069
:10FE40007F0000238DF80500ADF80630019802B060
:10FE50007047B0F5803F14D2030B63F01F038DF899
:10FE60000430C0F3851363F07F0300F03F008DF88A
:10FE7000053060F07F0000238DF806008DF8073014
:10FE8000E4E7B0F5881FE1D2830C63F00F038DF82F
:10FE90000430C0F3053363F07F038DF80530C0F301
:10FEA000851300F03F0063F07F0360F07F008DF862
:10FEB00006308DF80700C9E7030612D5C0F3072204
:10FEC000030603EB0243C0F3074203EB022303EBF9
:10FED00010600423C2B202B9000A013B13F0FF0311
:10FEE000F8D17047232916D102785AB9012303703B
:10FEF0000278012A04D1202904BF0223037013468B
:10FF000018467047012A4FF00003F0D0022AEFD1C3
:10FF100003700123ECE70023EAE700002DE9F04F2E
:10FF2000884685B017461E460546002400283ED068
:10FF3000002A3ED003948DF80B40002935D09DF85F
:10FF40003890DFF87CA009F00109DAF8043003A941
:10FF50002846984783460398DAF80420002128446D
:10FF600090470246B9F1000F11D1134B594638465C
:10FF7000984703B2002B14DC039B9845E5D8002C6E
:10FF800001DDA61B34B2204605B0BDE8F08F01901C
:10FF90000A4B59460DF10B009847019A0028E4D00E
:10FFA000EAE73444204404B2E6E70C46EBE70446B3
:10FFB000E9E71446E7E700BF75D10000E5FE000061
:10FFC000540000202DE9F04F8FB099469DF8603025
:10FFD000029104920393074698B1002900F0D28061
:10FFE000039B13F012030FD0002000E001303B5CB4
:10FFF0000A2B00F0C9800D2B00F0C680002BF5D134
:020000021000EC
:1000000080B20FB0BDE8F08F039A8DF82B3012F05C
:100010000202059247F6184218BF91460B930B9BBC
:10002000009307EB030BFB5C002B00F08E80B9F113
:10003000000F40F38A80059A47F61843002A08BF4C
:100040004B460793514B00255B68CDE90C550CA935
:10005000584698470C9B0D93039B019503F00103B1
:1000600080464FF0FF3A2E462A462C4608931BF84E
:10007000043043B9BAF1FF3F52D0009B002B6ED140
:100080001FFA8AF455E0414B0DA95B685846984722
:10009000019B01330693089B024673B109903C4BC8
:1000A00041460DF12B009847099A30B1DDE90C4328
:1000B0000C93069B01939046D9E7364B0298099220
:1000C00041469847064400B20028C8BF049B099ADD
:1000D000B6B2C4BFF618B6B2BAF1FF3F36B205D118
:1000E000049B0799F31A8B42C8BFA246B8F10A0FC6
:1000F00010D0B8F10D0F0DD027480023D9B2415CC4
:1001000021B9BAF1FF3F08BF3546CFE7884503F173
:100110000103F3D1002CADD1BAF1FF3FADD135468B
:10012000019B23B1B8F10D0F02D10A2A00D10C9C1A
:10013000A4B2A9EB05050B9B0FFA85F994B95BB93D
:10014000124B0BA95B68384698470B9B23B90F4BA2
:100150000BA95B6838469847BDF82C0051E700258D
:100160002C46E6E71C443B780B940A2BEDD00D2B74
:10017000EBD03B5D0A2B02D00D2B7FF450AF013446
:100180000B94E2E702983CE7013039E75400002085
:10019000E5FE000075D10000E64102002DE9F04FB8
:1001A00089B0002598469DF85030BDF948B0BDF99A
:1001B0004CA004930446164605804580039129B35C
:1001C00022B3049B13F0020F47F6184318BF9A4658
:1001D000B2F908300693138905935B440793039B98
:1001E00003EB05095B5DA3B955B119F8013C0A2B76
:1001F00001D00D2B04D1059B62885B4413446380BE
:10020000B4F90230002B31D1069B638009B0BDE800
:10021000F08F049B0093424653463146154F4846A3
:10022000B847B4F90230079A1344B3F5004F0146BA
:1002300005440BD3104B114C12931149114B7122F1
:100240000220A44609B0BDE8F04F60476380049BDC
:10025000009348464346DFF830903246C847B4F929
:1002600000309842B8BF18462080B8E7A3EB0B03D4
:10027000CBE700BFC5FF00001D420200E9E8000017
:10028000EE4102005D4202001DFF00002DE9F04733
:10029000089D80460F46144699460CB9264612E042
:1002A0004FEA540A09FB0A7631464046A84700281F
:1002B00008DDE44304F00104AAEB040A06EB090795
:1002C0005446EAE7FCD13046BDE8F087014B1860A0
:1002D000704700BFD0C70020014B1B68D86870472B
:1002E000D0C70020014B1B681B681847D0C70020EF
:1002F000C0F3031310B500F0F001C4B2C0F307124D
:10030000194300F00F0343EA041322F00F02890897
:1003100042EA1020C3F3C40343EA4113C0F3C4000C
:1003200043EAC02010BD000001392DE9F047044622
:10033000272934D8DFE811F028003900BB008200FB
:1003400044004F004703B7000F01560239006F0306
:1003500020029503B700B7007100B7005101B70044
:10036000F701150285032A013B01EF016601D30164
:10037000EB001B033703D700980084028E01B901FC
:10038000F002C701BE02E502994B00219847994B44
:10039000002120469847984B1968984B984720466B
:1003A000974BBDE8F047FF211847914B0021984734
:1003B000904B0021204698478F4B19680431ECE799
:1003C0008B4B002198478B4B0021204698478A4B46
:1003D00019681031E1E7884EDFF81492DFF81482D3
:1003E000864D0021C84700212046C04731680431AE
:1003F0000746A847316818313846A84701212046EA
:10040000C84701212046C047316804310746A84744
:10041000316838460831A847C1E70021DFF8D0919C
:10042000DFF8D081744E754DC84700212046C04783
:1004300031680746A84731686831DDE7DFF8B081E9
:100440006D4E6C4F6D4D0021C04700212046B847CE
:1004500031682431A84701212046C04701212046A8
:10046000B84731682831D6E7DFF88481624E614FA2
:10047000624D0021C04700212046B8473168243131
:10048000A84701212046C04701212046B8473168CE
:100490002831A84702212046C04702212046B847FC
:1004A00031689C31B7E7524B0021984777E7DFF876
:1004B0004091514EDFF83C81504D0021C84700214A
:1004C0002046C047316804310746A847316838469E
:1004D0002031A84701212046C84701212046C047B6
:1004E00031681C3197E7DFF80881434E414F434D97
:1004F0000021C04700212046B84731682031A84775
:1005000020460121C04701212046B847E8E73A4E7E
:10051000DFF8DC80374F394D0021C04700212046ED
:10052000B847316824318146A8473168484694313C
:10053000A84701212046C04701212046B84731681D
:100540002831A84702212046C04702212046B8474B
:10055000316890315FE7284FDFF89480254E274DB2
:100560000021C04700212046B04739684C31A847D8
:1005700040212046C04740212046B047396810310D
:100580000646A84739683046503144E7184B1A4FA1
:100590001A4E00219847174B00212046984739688A
:1005A00004310546B04739687C3128467BE0DFF8E6
:1005B0004080114E0F4F114D4021C0474021204631
:1005C000B84731681831A84741212046C04741212A
:1005D0002046B847316810311DE7054B0021984788
:1005E000044B002120469847034B19686C31D4E630
:1005F000492500008D240000D4C7002019560000B2
:10060000912D0000DFF8A882A64EA74FA74D00212C
:10061000C04700212046B84731680431A84740212F
:100620002046C04740212046B84731681431A847CA
:1006300001212046C04701212046B847316880315A
:10064000A84702212046C04702212046B84731680A
:100650008431E0E6964D934FDFF84C82934E0021B3
:10066000A84700212046C0473968B04740212046AE
:10067000A84741212046A84741212046C047396864
:10068000A831B04743212046A84743212046C04710
:100690003968AC31B04742212046A8474221204664
:1006A000C0473968A431B04779E6814D0021A84799
:1006B00040212046A8477C4B402120469847794B53
:1006C0001968B03169E60021DFF8E481754E764F94
:1006D000764DC04700212046B8473168A7E7714EE4
:1006E000DFF8CC91DFF8C081704D0021C8470021B0
:1006F0002046C047316804310746A847316838466C
:100700008831A84703212046C84703212046C04717
:1007100031688C317FE6664B00219847624B00219F
:10072000204698473BE6624F5E4EDFF87C915F4D76
:100730000021B84700212046C8473168043180466F
:10074000A847316840467431A84740212046B84741
:1007500001212046B84701212046C8473168803131
:1007600059E6534B002198474F4B002120469847AC
:100770004C4B1968783110E64A4EDFF834814A4F05
:100780004A4D0021C04700212046B8473168043156
:100790008146A847316848460831A847316848462D
:1007A0001831A84740212046C04740212046B8477D
:1007B000316804318146A847316848465431A8471A
:1007C00041212046C04741212046B8473168803149
:1007D000A84742212046C04742212046B8473168F9
:1007E000583118E62F4EDFF8C890DFF8BC802F4D47
:1007F0000021C84700212046C04731680431074620
:10080000A847316838464031A84731683846183122
:10081000A84701212046C84701212046C04731682A
:1008200018310746A847316838464431A8470221A5
:100830002046C84702212046C04731684831EAE5D2
:10084000DFF86C80174E184F184D0021C04700216B
:100850002046B84731680431A84701212046C047E7
:1008600001212046B8473168A031A847022120461F
:10087000C04702212046B8473168A031A84703216C
:100880002046C04703212046B8473168A031A84719
:1008900004212046C04704212046B8473168A031D2
:1008A000B9E500BFD4C700208D2400001956000010
:1008B00049250000DFF800827C4E7D4F7D4D0021F0
:1008C000C04700212046B8473168A847422120464A
:1008D000C04742212046B84731688031A8474121AE
:1008E0002046C04741212046B8473168B031A8476B
:1008F00040212046C04740212046B8473168A831F2
:1009000089E56D4B00219847694B002120469847A7
:10091000664B1968A43140E5DFF89C81634E644F53
:10092000644D0021C04700212046B847316804319A
:100930008146A847316848461831A8472046042117
:10094000C04704212046B8473168B831A84720463F
:100950000321C04703212046B8473168B431A84776
:1009600020460121C04701212046B847F6E64F4EF8
:10097000DFF84491DFF838814E4D0021C84700214F
:100980002046C047316804310746A84731683846D9
:100990001831A84703212046C84703212046C047F5
:1009A0003168983137E5444B404F424E002198471B
:1009B0003F4B002120469847396804310546B0472F
:1009C00039680831F1E5DFF8F080384E384F394D9D
:1009D0000021C04700212046B84731680431A847AC
:1009E00003212046C04703212046B84731682C31F7
:1009F000A84701212046C04701212046B847316859
:100A00003031A84702212046C04702212046B8477E
:100A100031683431FFE4DFF8A080244E244F254DA7
:100A20000021C04700212046B84731683831A84727
:100A300001212046C04701212046B84731683C319A
:100A4000E9E41D4B194F1B4E00219847184B00211C
:100A500020469847396804310546B04739687031F7
:100A6000A3E5124EDFF85080114F124D0021C04710
:100A700000212046B847316804318146A8473168D3
:100A800048465C31A84701212046C0470121204645
:100A9000B84731686031A84702212046C04702218B
:100AA0002046B84731686431B5E400BFD4C70020A0
:100AB0008D2400001956000049250000034B1B79C6
:100AC0000BB1034B1847034BFCE700BFD4C7002012
:100AD00095570000315500002DE9F0413A4D3B4B50
:100AE00028683B4E3B4C9C30984728683A4BFF2285
:100AF0002C219C3098472868384B29211A88384B7C
:100B00009C309847286847F6FF7201219C30B04717
:100B100000202F68A0473B2807F19C0747DD0020F5
:100B2000A0476FF0270300F1140292FBF3F212B218
:100B300038461021B04700202F68A0473B2807F116
:100B40009C0737DD0020A0476FF0270300F1140257
:100B500092FBF3F212B238461121B04700202F6801
:100B6000A0473B2807F19C0727DD0020A0476FF036
:100B7000270300F1140292FBF3F212B2122138465D
:100B8000B04700202D68A0473B2805F19C0517DDE4
:100B90000020A0476FF0270300F1140292FBF3F24C
:100BA00012B2284633461321BDE8F04118474FF0F2
:100BB000FF32BDE74FF0FF32CDE74FF0FF32DDE708
:100BC0004FF0FF32EDE700BFD4C70020BD0A01009F
:100BD0007958000051D90000195A000072420200F1
:100BE000495900002DE9F0416B4D6C4B28686C4E63
:100BF0006C4C70309847286847F6FF7201217030BE
:100C0000B04700202F68A04700EB80008000EF284D
:100C100007F1700740F3B2800020A0471423502250
:100C200000FB0322A02392FBF3F212B238461221FA
:100C3000B04700202F68A04700EB80008000EF281D
:100C400007F1700740F39C800020A0471423502236
:100C500000FB0322A02392FBF3F212B238461321C9
:100C6000B04700202F68A04700EB80008000EF28ED
:100C700007F1700740F386800020A047142350221C
:100C800000FB0322A02392FBF3F212B2384610219C
:100C9000B04700202F68A047C0EB00104000EF28AD
:100CA00007F1700770DD0020A0471E23502200FBD3
:100CB0000322A02392FBF3F212B238461421B0476C
:100CC00000202F68A04700EB800000EB8000EF2899
:100CD00007F170075ADD0020A0471923502200FBBE
:100CE0000322A02392FBF3F212B23846C021B04790
:100CF00028682D4FAA8999217030B8472868AA8999
:100D0000C9217030B8472868284B00F1700840F6B8
:100D100088009847CA2102464046B84700202F68FD
:100D2000A04700EB80004000EF2807F170072FDD9F
:100D30000020A0470A23502200FB0322A02392FB9D
:100D4000F3F212B290213846B04700202D68A04738
:100D5000C0EBC000EF2805F170051BDD0020A047A7
:100D60000723502200FB0322A02392FBF3F212B2CE
:100D700028463346C321BDE8F0411847012255E714
:100D800001226BE7012281E7012296E70122ACE70D
:100D90000122D7E70122EBE7D4C70020BD0A0100FA
:100DA0007958000051D9000049590000F1020100B2
:100DB0002DE9F041324C334B2068334F334E344DE4
:100DC0006C3098472068FF222C216C30B84720688F
:100DD000A28929216C30B0472068022230216C3072
:100DE000A84720687F223C216C30B8472068294BF7
:100DF00000F16C074C21A0899847392102463846FA
:100E0000B0472068244F47F6FF7201216C30A84795
:100E10002368002003F16C08B847C0EB0010EF28EE
:100E20002ADD0020B8470F23502200FB0322A02315
:100E300092FBF3F212B250214046A8472068A289E3
:100E400059216C30B04700202468B84700EB80007F
:100E5000EF2804F16C0411DD0020B847052350226F
:100E600000FB0322A02392FBF3F212B220462B4692
:100E70005321BDE8F04118470122DCE70122F5E7E4
:100E8000D4C70020BD0A0100195A000049590000CA
:100E9000795800004BE3000051D90000C0F38522CF
:100EA000C0F3C40343EA4213C0F3C44043EAC02082
:100EB000704700002DE9F047434CDFF8349120687B
:100EC000424E434FDFF82C812430C847206847F654
:100ED000FF7201212430B0472068FF2224302C21EA
:100EE000B847236A256813F0020F14BF39483A48FF
:100EF000C0472435024629212846384DA847236893
:100F000003F1240A236A9A0758D53548C047024698
:100F100079215046A8472068A28949212430A84752
:100F20002068E28940F249412430A8472068002225
:100F30004C212430B84720687F224FF413712430AD
:100F4000B8472068032240212430B0472068962209
:100F5000B0212430B04720684C22B7212430B0475C
:100F600020682830C8472068FF222C212830B84745
:100F7000206847F6FF7201212830B0472068A28917
:100F800029212830A8472068164B00F1280640F692
:100F90008800984742F2290102463046A847236A52
:100FA00020689B0700F128060BD50F48C047024672
:100FB00030462B467921BDE8F04718470B4B1A887D
:100FC000A6E70A4B1A88F3E7D4C700207958000037
:100FD000195A0000D9D7D4004D494500495900009D
:100FE0004F403100F10201004F40410072420200C7
:100FF000BD0A01009D0E01002DE9F0417D4C7E4FA0
:1010000020687E4D9030B84720687D4BFF222C2110
:1010100090309847236A20689A0756BF794BA28977
:101020001A8890302921A847236A26689B0706F171
:10103000900640F1CC807448744B98470246304685
:101040007921A8472068724E724D47F6FF72012140
:101050009030B0472368002003F19008A847C0EB08
:10106000C000EF2840F3B6800020A8470723502295
:1010700000FB0322A02392FBF3F212B2404612219E
:10108000B0472368002003F19008A847C0EBC000D8
:10109000EF2840F3A1800020A8470723502200FB3F
:1010A0000322A02392FBF3F212B240461321B04771
:1010B0002368002003F19008A847C0EBC000EF2888
:1010C00040F38C800020A8470723502200FB032216
:1010D000A02392FBF3F212B240461021B0472368DE
:1010E000002003F19008A847C0EBC000EF2877DD8F
:1010F0000020A8470723502200FB0322A02392FBD5
:10110000F3F212B211214046B04720689430B8473C
:1011100000202768A84700EB80004000EF2807F177
:1011200094075FDD0020A8470A23502200FB03221A
:10113000A02392FBF3F212B238461721B0470020E9
:101140002768A84700EB80004000EF2807F19407CC
:101150004ADD0020A8470A23502200FB0322A023D7
:1011600092FBF3F212B238461821B04700202768EC
:10117000A84700EB80004000EF2807F1940735DD19
:101180000020A8470A23502200FB0322A02392FB41
:10119000F3F212B215213846B04700202468A84760
:1011A00000EB80004000EF2804F1940420DD0020D3
:1011B000A8470A23502200FB0322A02392FBF3F24C
:1011C00012B2204633461621BDE8F04118470D4BB8
:1011D0001A8834E7012251E7012266E701227BE702
:1011E00001228FE70122A7E70122BCE70122D1E714
:1011F0000122E6E7D4C70020BD0A010049590000DA
:10120000195A0000724202004F4031009D0E010049
:101210007958000051D900002DE9F047B64CDFF8AD
:10122000F4822068DFF8F092B44F5C30C047206849
:1012300000F15C0540F68800C8479921024628461F
:10124000B847206800F15C0540F68800C847C9210E
:1012500002462846B8472068A289A94DCA215C30B9
:10126000B84700202668A84700EB8000EF2806F169
:101270005C0640F38D810020A8470523502200FB27
:101280000322A02392FBF3F212B2304690219D4E2E
:10129000B0472368002003F15C0AA8473B2840F3CD
:1012A00079810020A847282300F1140292FBF3F271
:1012B00012B25046C321B0472368002003F15C0AF4
:1012C000A8471D2840F368810020A847142300F197
:1012D0000A0292FBF3F212B25046C221B0472368D1
:1012E000002003F15C0AA84700EB80008000EF2893
:1012F00040F354810020A8471423502200FB03220E
:10130000A02392FBF3F212B250461221B047236899
:10131000002003F15C0AA84700EB80008000EF2862
:1013200040F33E810020A8471423502200FB0322F3
:10133000A02392FBF3F212B250461321B047236868
:10134000002003F15C0AA84700EB80008000EF2832
:1013500040F328810020A8471423502200FB0322D9
:10136000A02392FBF3F212B250461021B04723683B
:10137000002003F15C0AA84700EB80008000EF2802
:1013800040F312810020A8471423502200FB0322BF
:10139000A02392FBF3F212B250461421B047236807
:1013A000002003F15C0AA847C0EB0010EF2840F3CF
:1013B000FD800020A8470F23502200FB0322A0231A
:1013C00092FBF3F212B25046C021B047206847F6B4
:1013D000FF7201215C30B04720686030C047206850
:1013E00000F1600A40F68800C8479921024650463D
:1013F000B847206800F1600A40F68800C847C92154
:1014000002465046B8472068A289CA216030B847D2
:101410002368002003F16009A8471D2840F3C88015
:101420000020A847142300F10A0292FBF3F212B243
:1014300048469021B0472368002003F16009A8477F
:101440001D2840F3B7800020A847142300F10A02AA
:1014500092FBF3F212B24846C321B0472368002042
:1014600003F16009A84700EB800000EB8000EF2843
:1014700040F3A2800020A8471923502200FB03223A
:10148000A02392FBF3F212B2C0214846B047206875
:101490006430C047236803F16408236A9A0740F167
:1014A0008D801948194B9847024640469921B84704
:1014B0002368002003F16408A8471D2840F38180B9
:1014C0000020A847142300F10A0292FBF3F212B2A3
:1014D00040469021B04720680D4BFF222C216430FC
:1014E0009847236803F16408236A9B076BD5064875
:1014F000064B9847024611E0D4C700204959000026
:1015000051D90000795800005B4B46009D0E010048
:10151000195A0000BD0A0100F102010029214046CC
:10152000B847206847F6FF7201216430B0470020B9
:101530002768A847C0EB00104000EF2807F16407B8
:1015400044DD0020A8471E23502200FB0322A023D5
:1015500092FBF3F212B203213846B0470020246810
:10156000A84700EB80004000EF2804F164042FDD61
:101570000020A8470A23502200FB0322A02392FB4D
:10158000F3F212B2204633461421BDE8F047184763
:1015900001227AE601228CE601229DE60122B3E6D1
:1015A0000122C9E60122DFE60122F5E601220AE76F
:1015B00001223DE701224EE7012265E7054B1A882B
:1015C00073E7012284E7034B1A88A7E70122C2E7E9
:1015D0000122D7E7724202002DE9F047684D694FBA
:1015E0002868DFF8BC914030B8472B6A2C6813F0AC
:1015F000020F04F1400400F0B180634B40F6AA20D2
:101600009847024648F289012046DFF898815F4CEE
:10161000C04728684430B84700202E68A047EF280C
:1016200006F1440640F39D800020A047A02300F16E
:10163000500292FBF3F212B230469021544EB04762
:101640002B68002003F1440AA04700EB8000400013
:10165000EF2840F388800020A0470A23502200FB97
:101660000322A02392FBF3F212B250469221B0471C
:101670002B68002003F1440AA04700EB80004000E3
:10168000EF2872DD0020A0470A23502200FB03222E
:10169000A02392FBF3F212B250469321B0472B687D
:1016A00003F1440A2B6A9B074CBF3A483A48C847A3
:1016B000992102465046C04728684830B847002064
:1016C0002F68A04700EB4000EF2807F148074EDDE8
:1016D0000020A0470323502200FB0322A02392FBFB
:1016E000F3F212B238469021B04700202F68A0478D
:1016F0003B2807F148073CDD0020A047282300F1E4
:10170000140292FBF3F212B238460321B0470020D4
:101710002F68A047772807F148072CDD0020A04755
:10172000502300F1280292FBF3F212B21421384642
:10173000B04700202D68A047EF2805F148051CDDC3
:101740000020A047A02300F1500292FBF3F212B256
:10175000284633460121BDE8F04718470F48C847DF
:101760004FE7012268E701227FE7012294E7012287
:10177000B8E70122C8E70122D8E70122E8E700BF65
:10178000D4C70020BD0A0100F102010051D90000B8
:1017900079580000E3DDD600978A8000BDADA10036
:1017A0009D0E0100495900002DE9F04F2DED028BEF
:1017B000A14CA24F2068A24DDFF8B0A283B0B84779
:1017C0002068FF222C21A847236A266813F0020F05
:1017D00014BF9C489C48AB469C4DA847B94602465E
:1017E0009B4F30462921B847236A266898074CBF8B
:1017F00098489948A84748F2890102463046B847B8
:10180000236A266899074CBF92489348A8477921D4
:1018100002463046B84762692068904E48F28E0111
:10182000D047626920687E21D04720680430C847CD
:101830002368002003F10408B0471D2840F36885A1
:101840000020B047142300F10A0292FBF3F212B217
:1018500040460121DFF81882C0472068FF2204308B
:101860002C21D847236803F1040B236A9A0754BF3D
:101870007B486FF07F40A847292102465846B84769
:10188000236803F1040B236A9B074CBF7548764815
:10189000A847392102465846B8472068A28940F235
:1018A00039210430B8472068E28940F239410430D8
:1018B000B8472368002003F1040BB047772840F3B2
:1018C0002A850020B047502300F1280292FBF3F252
:1018D00012B258463021C04720680122332104301B
:1018E000C04720686269043048F28E01D0472368FF
:1018F00003F1040B236A98074CBF56486FF07F40F2
:10190000A84748F2890102465846B84720686269EC
:1019100004307E21D047236803F1040A236A990723
:101920004CBF4C486FF07F40A84779210246504693
:10193000B847236803F1040A236A9A074CBF454855
:101940006FF07F40A84748F2A90102465046B847C9
:10195000236803F1040A236A9B074CBF3D486FF0DC
:101960007F40A847992102465046B8472068DFF8D3
:1019700004A1012290210430C047236800200433D1
:1019800008EE103AD04701284FF0000000F2D3844F
:10199000B047C0EB0010EF2800F3C0844FF0010BFC
:1019A0000020B047772840F3D1840020B04750236F
:1019B000283090FBF3F080B20BEB000212B218EE6D
:1019C000100A1221C04723680020043308EE103AA1
:1019D000D04701284FF0000000F2C884B047C0EBA8
:1019E0000010EF2800F3B5844FF0010B0020B04742
:1019F000772840F3C6840020B0475023283090FB5E
:101A0000F3F080B20BEB000212B218EE100A1321B1
:101A1000C04723680020043308EE103AD04701285D
:101A20004FF0000000F2BD84B047C0EB0010EF287B
:101A300000F3AA8420E000BFD4C70020BD0A010043
:101A4000195A0000F3EFEA005A4B44009D0E0100C2
:101A500049590000423E3B00ECE9E70051D9000043
:101A600073625800E3DDD600978A8000ED5A0000CB
:101A70007958000069D900004FF0010B0020B047F1
:101A8000772840F399840020B0475023283090FBFA
:101A9000F3F080B20BEB000212B218EE100A102124
:101AA000C04723680020043308EE103AD0470128CD
:101AB0004FF0000000F29084B047C0EB0010EF2818
:101AC00000F37D844FF0010B0020B047772840F3EE
:101AD0008E840020B0475023283090FBF3F080B272
:101AE0000BEB000212B218EE100A1121C047236856
:101AF000002003F1040BD04701284FF0000000F252
:101B00008584B047C0EB0010EF2800F373840122F6
:101B100014215846C04720689622B0210430C0479F
:101B200020683922B7210430C04720680C30C847EC
:101B30002068AC4B011D0C309847236A2668980733
:101B40004CBFA948A948A8470C360246292130466F
:101B5000B847236A266899074CBFA548A548A847F7
:101B60000C36024639213046B847236A26689A0760
:101B70004CBFA148A148A8470C36024648F289014B
:101B80003046B847236A26689B074CBF9A489B4853
:101B9000A8470C36024679213046B847236A2668A2
:101BA00098074CBF94489548A8470C36024648F21F
:101BB000A9013046B847236A266899074CBF8E486A
:101BC0008E48A8470C36024699213046B84720680F
:101BD0000830C847236A2668DFF850929A074CBF3E
:101BE00087488848A8470836024641F2290130460E
:101BF000B8472068A28940F229110830B847206808
:101C0000332100F10806A089C84741F22911024694
